:020000040800F2
:100000000000011011E3030835E602083DF800087E
:1000100015E4030815E4030815E4030800000000D4
:1000200000000000000000000000000081EC020859
:100030007DEC02080000000079EC0208DDF1000808
:1000400015E4030815E4030815E4030815E40308A0
:1000500015E4030815E4030881D70108F9D701085E
:10006000BDD7010845D70108FDF80008F5AB000829
:10007000E5AB0008D5AB0008C5AB0008B5AB000880
:10008000A1AB00088DAB000815E4030815E40308D4
:1000900015E4030815E4030815E40308C1F8000893
:1000A00015E4030815E4030815E4030815E4030840
:1000B00011E9000801E90008F1E8000815E4030867
:1000C00015E4030815E4030815E4030815E4030820
:1000D00015E4030835F2000815E4030829F20008C6
:1000E00085F8000815E4030899ED020815E40308F3
:1000F00015E4030815E4030815E4030879AB0008C8
:1001000015E4030815E4030815E4030815E40308DF
:100110001DF2000815E40308D98D0308BD8D0308FE
:1001200065AB000851AB00083DAB000829AB0008E7
:1001300015AB000815E4030815E4030815E40308EB
:1001400015E4030815E4030815E4030839E602087A
:1001500001AB0008EDAA0008D9AA000811F20008B6
:1001600015E4030815E4030815E4030815E403087F
:1001700015E4030815E4030815E4030815E403086F
:0801800015E4030815E403086F
:08018800A8DE030001000000E5
:1001900016000800B8280020CC280020000000002D
:1001A0002C060008270004009C2E0020082F0020A9
:1001B000000000003406000801010400542F002054
:1001C0008C4200200000000000000000080209002E
:1001D0004C4200209042002000000000ADD10108F8
:1001E00002000C00584200209C4200200000000049
:1001F00000000000F701060040420020A842002055
:1002000000000000380600080300010068440020D8
:100210006C440020000000000000000003123300C6
:100220008B480020584800200000000040060008CD
:1002300025005A00A4470020FE47002000000000CF
:1002400000000000F6110C00984700208C470020A9
:10025000000000007406000815007000AC46002085
:100260001C47002000000000000000002A00600081
:10027000EC4500204C46002000000000C52C03087F
:100280002C001000C4510020B451002000000000D8
:10029000D95F02082B002400F8510020D45100201F
:1002A00000000000A95F020829005000EC50002067
:1002B0001C520020000000000000000009020100A4
:1002C000DA540020305500200000000080060008AD
:1002D0000102050084540020345500200000000075
:1002E00035820208000205006C5200203C550020B7
:1002F000000000000000000004008000F463002003
:10030000746400200000000000000000F9010400F7
:10031000E4580020F464002000000000F5D8000834
:10032000FD011E00C4580020F864002000000000F9
:1003300085D80008060016004455002018650020E6
:1003400000000000592D03081F000E0084660020E5
:100350005868002000000000820600080502010025
:100360006C6600206868002000000000900600080D
:100370001E000400186A0020006C0020000000002D
:100380009206000822000C0098690020046C0020EE
:10039000000000009606000814000200687F00209C
:1003A0006C7F002000000000A2060008100003007F
:1003B000587F0020707F002000000000A406000885
:1003C00028001000487F0020747F002000000000FB
:1003D000953D020823001000387F0020847F002014
:1003E00000000000AD3D020819000500307F00202C
:1003F000947F002000000000A8060008F81101000A
:100400002C7F00209C7F002000000000AE0600082A
:1004100000010400287F0020A07F002000000000D1
:10042000B00600081B00F40030800020B88E0020C9
:1004300000000000A9C902080E0202002C80002062
:10044000AC8F002000000000B40600082F0011004F
:100450005C8E0020B08F002000000000B60600086F
:1004600005100600AC8E0020C48F002000000000A4
:10047000C8060008F5216C00A47F0020CC8F002066
:10048000000000009106030803010A0068900020A4
:100490007490002000000000CE0600080120080033
:1004A000609600208096002000000000D80600081A
:1004B0001A000800489600208896002000000000DE
:1004C000E006000818102C00FC9C0020549D002021
:1004D00000000000B96602080D002C00289D0020D5
:1004E000809D00200000000001B70108FA01020011
:1004F000D0960020AC9D00200000000039D70008F5
:1005000002020300B8960020B09D00200000000009
:10051000000000000C020100A8960020B49D0020FD
:1005200000000000E806000826000E008CA0002055
:100530007CA0002000000000ED6603080B201000E6
:10054000609E00209CA0002000000000EA06000839
:100550000A020A0048A1002058A100200000000063
:10056000FA0600080C002400F0A2002080A300205E
:100570000000000095B601080E20EA00E4A100206A
:10058000A4A3002000000000392D0308130004007C
:100590003CA3002090A400200000000004070008F5
:1005A00002010300CFA1002094A40020000000005D
:1005B000BDB60108FE01090098A70020ECA70020A5
:1005C0000000000025D70008FB01010028B2002030
:1005D000ECB2002000000000DDD60008FC0109009C
:1005E000F4B00020F0B2002000000000A1D6000806
:1005F0000A101200C8B00020FCB200200000000069
:10060000080700083400100018A8002010B30020CC
:1006100000000000ED2C030812200C0008A80020A8
:0C06200020B30020000000001A070008B2
:10062C00C40900001901282820030000240100003F
:10063C0000000000000000000000000000000000AE
:10064C00000000000000000000000000000000009E
:10065C00000000000000000000000000000000008E
:10066C00000000000000010000000000000000007D
:10067C00000000002000000000000000010000004D
:10068C0000050000000000000100C800141E01005D
:10069C0064002C0128000300000105000000280163
:1006AC0000000400900100000000000000000000A9
:1006BC00000000000000000000000000200003010A
:1006CC000000040101006C1600000000E803640047
:1006DC00040A00017E05EA05B405320001002B2155
:1006EC00231E64010100000001000A012900000022
:1006FC004A01B400D60127000800000000300100B8
:10070C00005A0000000090012C01C8006400000099
:0A071C0000010005464F5254000092
:100726000100000050010000070000000200000068
:10073600000000000000000001020304060708098B
:1007460001010000382E0408185F040800000000AC
:1007560000000000482E0408502E04080000000087
:1007660001200000542E04085C2E0408000000003E
:1007760001400000602E0408E04504080000000067
:10078600012000006C2E0408782E040800000000EA
:10079600040000007C2E0408C06404080000000069
:1007A60004000000882E0408845D04080000000090
:1007B600010000000201FF000000803F0000803FB2
:1007C600200204080508040000000000942904081B
:1007D6001025040880290408000000004C020408C3
:1007E60005080A00000000009429040810250408E2
:1007F600B029040800000000FFFFFFFF000101010F
:10080600010000000101D6017D5902080000000028
:1008160000000000E00108000000803F00FFFF002C
:1008260000000000AA5505010000012D202D2D20F5
:100836002D2D2D2D202D2D2D2D000000000000002A
:1008460000000000000000000000AA550B01000097
:10085600AA5507010000AA55090200000000000081
:1008660001000000C012AA5503009F00000001010C
:10087600FFFF000004030904120100020202004007
:1008860083044057000201020301000009024300ED
:10089600020100C032090400000102020100052421
:1008A60000100105240100010424020205240600AB
:1008B60001070582030800FF09040100020A00007F
:1008C6000007050102400000070581024000000004
:1008D600FF0000005925030839E10208112003082A
:1008E60089DE0208F9E2020899DE0208B5DE02088E
:1008F60079DE020869DE0208000000000000000040
:1009060001000000FFFFFFFF0000000001020304DA
:1009160001020304060708090000803F00000000EA
:1009260000000000000000000000803F0000000002
:1009360000000000000000000000000000000000B1
:1009460000000000000000000000000000000000A1
:100956000000803F000000000000000000000000D2
:100966000800000000000001000000000000000078
:100976000000000065E202081DE20208C5EC02085C
:100986000000000041DE020885E002080DE10208D1
:10099600E5DF0208000000000000000035DE020866
:1009A600B5DD0208B1DD0208ADDD0208A1DD0208F1
:1009B6009DDD0208A9DD0208A5DD020829DE020880
:1009C6001DDE0208F5DD020809DE0208E1DD020887
:1009D600CDDD0208B9DD0208285404080000000035
:1009E60000000000D1B60108A08601000400000046
:1009F60000000000000000000000000000000000F1
:100A0600000000000000000000000000506A04081A
:100A16006450040800000000855401087D000000B1
:100A260006000000000000000000000000000000BA
:100A360000000000000000000000000000000000B0
:100A4600DC6404080000000000000000254E0108D8
:100A5600E8030000030000000000000000000000A2
:100A66000000000000000000000000000000000080
:100A760000000000E464040800000000000000001C
:100A86008D2E030810270000030000000000000060
:100A96000000000000000000000000000000000050
:100AA6000000000000000000F064040800000000E0
:100AB6002D5E020825290108204E000005000000D1
:100AC6000000000000000000000000000000000020
:100AD600000000000000000000000000B8550408F7
:100AE600000000000000000039F90008102700008F
:100AF60001000000000000000000000000000000EF
:100B060000000000000000000000000000000000DF
:100B1600F464040800000000000000006DD6000820
:100B2600E8030000050000000000000000000000CF
:100B360000000000000000000000000000000000AF
:100B4600000000000065040800000000000000002E
:100B560089B90108204E00000300000000000000D3
:100B6600000000000000000000000000000000007F
:100B760000000000000000001065040800000000EE
:100B86000000000091B70108204E0000030000009D
:100B9600000000000000000000000000000000004F
:100BA60000000000000000000000000020650408AE
:100BB600000000000000000015520108400D03006F
:100BC600030000000000000000000000000000001C
:100BD600000000000000000000000000000000000F
:100BE600EC540408000000000000000089CE030851
:100BF60010270000010000000000000000000000B7
:100C060000000000000000000000000000000000DE
:100C160000000000805004080000000000000000F2
:100C2600B582020810270000030000000000000043
:100C360000000000000000000000000000000000AE
:100C46000000000000000000C0550408000000007D
:100C56000000000089FE0008A00F0000010000004F
:100C6600000000000000000000000000000000007E
:100C760000000000000000000000000030650408CD
:100C86000000000000000000A5C3020810270000B5
:100C9600010000000000000000000000000000004D
:100CA600000000000000000000000000000000003E
:100CB600F4540408000000000000000011150308A9
:100CC6001A410000010000000000000000000000C2
:100CD600000000000000000000000000000000000E
:100CE6000000000024560408000000000000000078
:100CF6002DAA0208102700000100000000000000D5
:100D060000000000000000000000000000000000DD
:100D16000000000000000000A464040800000000B9
:100D26000000000099A503081A4100000100000018
:100D360000000000000000000000000000000000AD
:100D46000000000000000000000000003C650408F0
:100D56000000000000000000D9A00108400D0300BB
:100D6600000000000000000000000000000000007D
:100D7600000000000000000000000000000000006D
:100D860044650408000000000000000075A001088A
:100D9600400D0300000000000000000000000000FD
:100DA600000000000000000000000000000000003D
:100DB600000000004C650408000000000000000070
:100DC6003D8A0208A0860100030000000000000022
:100DD600000000000000000000000000000000000D
:100DE60000000000000000000000803F000000003E
:100DF600000000000000000001010100C18F03088F
:100E06000000000050080020E8660408000000000A
:100E1600000000000000000000000000185F040849
:100E26000000000000000000BC08002004000000D4
:100E3600946604080D000000E5980308A00C002045
:100E460000000000C86904080D0000000D990308A1
:100E5600940C002000000000086704080800000049
:100E660000000000880C002004000000F86604085A
:100E76000D000000699003087C0C002000000000B3
:100E8600A86504080300000031A40308700C0020C4
:100E960000000000006704080300000031A40308F6
:100EA600640C002000000000AC650408010000008E
:100EB600000000000000000000000000000000002C
:100EC6000E0000000000000000000000000000000E
:100ED600E8660408000000000000000000000000B2
:100EE60000000000185F0408000000000000000079
:100EF600BC080020040000002C6604080300000063
:100F0600F9960308580C002008000000F86604084B
:100F16000D000000699003087C0C00200000000012
:100F2600A86504080300000031A40308700C002023
:100F360000000000006704080300000031A4030855
:100F4600640C002000000000AC65040801000000ED
:100F5600000000000000000000000000000000008B
:100F66000E0000000000000000000000000000006D
:100F760010670408000000000000000000000000E8
:100F860000000000185F04080000000000000000D8
:100F9600BC080020040000003466040803000000BA
:100FA60031A40308AC0C002000000000AC65040866
:100FB600010000000000000000000000000000002A
:100FC600000000000E00000000000000000000000D
:100FD6000000000020700020702D72002D202D2DA5
:100FE600202D2D2D2D202D2D2D0000000000000080
:100FF6000000000000000000000000006AA10020C0
:1010060088136F17010000006CA1002088136F176A
:1010160000000000806504080000000000000000D9
:1010260000000000000000009065040808000000B1
:1010360000000000E8080020040000009C65040889
:101046000800000000000000DC080020000000008E
:10105600A865040804000000399703080000000092
:1010660000000000AC65040801000000000000005C
:101076000000000000000000000000000E0000005C
:1010860000000000000000000000000068A1002031
:1010960088136F17010000006466002088136F171D
:1010A600000000002190030800000000F408002062
:1010B60038A30020010000005429040866660020B9
:1010C60001000000602904085C66002002000000A0
:1010D60068290408167D00200000000000000000BA
:1010E600147D00200000000000000000127D00209A
:1010F6000000000000000000107D0020000000003D
:10110600000000000E7D002000000000000000002E
:101116000C7D0020000000000000000044010020BB
:10112600000000000000000067A10020020000008F
:1011360074290408E46504080000000000000000AB
:101146000000000000000000906504080800000090
:101156000000000078090020040000009C650408D7
:1011660008000000000000006C09002000000000DC
:10117600A865040804000000F58F030800000000BD
:1011860000000000AC65040801000000000000003B
:101196000000000000000000000000000E0000003B
:1011A600000000000000000000000000F4650408D4
:1011B6000000000000000000000000000000000029
:1011C600046604080D00000089980308A809002099
:1011D60004000000106604080D0000004590030896
:1011E6009C090020040000001C6604080D00000095
:1011F6004D980308900900200000000028660408A6
:101206000300000019970308840900200800000065
:10121600346604080300000031A40308AC0C002067
:1012260000000000AC65040801000000000000009A
:101236000000000000000000000000000E0000009A
:101246000000000000000000000000003C660408EA
:101256000000000000000000000000000000000088
:1012660044660408040000005597030800000000C7
:1012760000000000AC65040801000000000000004A
:101286000000000000000000000000000E0000004A
:101296000000000000000000000000009C6604083A
:1012A6000000000000000000000000000000000038
:1012B600B85604080D00000000000000080A0020CF
:1012C60004000000AC6604080800000000000000EE
:1012D600FC09002004000000B866040808000000AD
:1012E60000000000F009002004000000C0660408A9
:1012F6000800000000000000E409002004000000CF
:10130600C86604080800000000000000D809002094
:1013160004000000D0660408080000000000000079
:10132600CC09002004000000D8660408080000006C
:1013360000000000C009002004000000E066040868
:101346000800000000000000B409002004000000AE
:10135600AC65040801000000000000000000000069
:1013660000000000000000000E0000000000000069
:1013760000000000000000000D90030800000000BF
:10138600140A002000000000000000008C0A002063
:1013960000000000000000002C0B00206266002008
:1013A600040000008029040860660020E0150C1780
:1013B600000000005F6600200800000010250408F9
:1013C6005E66002005000000942904080000000065
:1013D600000000007C0B0020000000000000000060
:1013E600F41F0020FFFFFFFFFA00000001000000CD
:1013F600010000003C670408446704083C660408D2
:1014060000000000000000000000000000000000D6
:10141600326704080400000071960308000000000B
:1014260000000000AC650408010000000000000098
:101436000000000000000000000000000E00000098
:101446000000000000000000000000007C8E00206C
:101456000100C409000000007A8E00200100C409C2
:1014660000000000788E00200100C4090000000082
:10147600768E00200100C40900000000728E002054
:101486000100C40900000000748E00200100C40998
:1014960000000000708E00200100C409000000005A
:1014A6006E8E00200100C409000000007AA1002011
:1014B6000100C8000100000078A10020320030754C
:1014C6003200000077A10020055A050072A1002015
:1014D60000FF010076A1002001000000D40C0020CE
:1014E60074A10020020000008026040871A10020DB
:1014F60000FF010075A1002001000000D40C0020AF
:1015060073A10020020000008026040800000000ED
:1015160000000000DC0C0020286600209CFF2C0147
:1015260000000000D80600200A000000B0290408C8
:1015360064A10020E0150C1700000000DA06002068
:101546000800000010250408D90600200500000048
:101556009429040866A1002002000000C829040896
:1015660028A300200100FF7F0100000027A3002020
:1015760002000000D4290408D8A1002003000000BE
:10158600E4290408D7A1002003000000E429040888
:10159600D6A200200000F40101000000D4A2002021
:1015A6000000F40101000000D2A200200000F401B6
:1015B60001000000D0A200200000F401010000009C
:1015C600CEA2002000FF0100EEA20020E803D00713
:1015D6000A000000ECA20020006401000A000000DE
:1015E600E8A2002000640100E7A2002000640100D8
:1015F600EDA20020006401000A000000E6A200201F
:10160600006401000A000000EBA200200064010053
:101616000A000000EAA20020006401000A0000009F
:10162600E9A20020006401000A000000E5A20020F3
:1016360000FF01000A000000E4A2002000FF0100F4
:101646000A000000E0A100200000F40101000000F3
:10165600DEA100200000F40101000000DCA1002052
:101666000000F40101000000DAA100200000F401EE
:1016760001000000E0A200201400E80301000000C1
:10168600DEA20020E803307501000000DDA2002084
:1016960000C80100DCA2002000C80100DBA2002077
:1016A60000C80100DAA20020006401000A00000060
:1016B600D9A2002000FF01000A0000001DA300209F
:1016C60000C801001CA3002000C801001BA30020C5
:1016D60000C801001AA3002000C8010019A30020B9
:1016E60000C8010018A3002000C8010017A30020AD
:1016F60000C8010016A3002000C8010015A30020A1
:1017060000C801006867040800000000000000002F
:1017160000000000000000007867040809000000CF
:1017260000000000800D002004000000806704080F
:101736000900000000000000740D002004000000F5
:10174600046D04080900000000000000680D002078
:1017560004000000682F04080900000000000000D3
:101766005C0D0020040000008867040809000000E2
:1017760000000000500D00200400000090670408DF
:101786000900000000000000440D002004000000D5
:10179600986704080900000000000000380D0020CA
:1017A60004000000A0670408090000000000000013
:1017B6002C0D002004000000AC65040801000000A8
:1017C6000000000000000000000000000000000013
:1017D6000E000000000000000000000000000000F5
:1017E600B4680408000000000000000000000000CB
:1017F60000000000DC5304080700000000000000A1
:10180600A40D002000000000C468040808000000C1
:1018160000000000980D002000000000D0680408B9
:1018260008000000000000008C0D002000000000F1
:10183600AC65040801000000000000000000000084
:1018460000000000000000000E0000000000000084
:101856000000000000000000D86804080000000036
:10186600000000000000000000000000E868040816
:101876000D00000000000000E00D00200000000048
:10188600F06804080D00000000000000D40D0020E0
:1018960000000000F86804080700000000000000CF
:1018A600CC0D002000000000006904080D000000B7
:1018B60000000000C00D00200000000008690408B8
:1018C6000D00000000000000B40D00200000000024
:1018D600106904080700000000000000AC0D00209D
:1018E60000000000AC6504080100000000000000D4
:1018F6000000000000000000000000000E000000D4
:101906000000000000000000000000001869040844
:1019160000000000000000000000000000000000C1
:10192600DC5304080C000000000000007CA100202D
:10193600000000002C6904080C00000000000000F4
:101946007EA10020000000003C6904080C00000095
:1019560000000000B4A10020000000004C6904084B
:101966000C00000000000000A8A1002000000000FC
:10197600606904080C0000000000000080A100203F
:10198600000000006C6904080C0000000000000064
:1019960082A1002000000000746904080C00000009
:1019A6000000000084A100200000000088690408EF
:1019B6000C0000000000000086A1002000000000CE
:1019C600906904080C0000000000000088A10020B7
:1019D60000000000986904080C00000000000000E8
:1019E600C6A1002000000000B06904080C00000039
:1019F600000000008AA1002000000000BC69040865
:101A06000C000000000000008CA100200000000077
:101A1600646404080C000000000000008EA1002091
:101A260000000000C46904080C000000000000006B
:101A360090A1002000000000D06904080C000000FE
:101A46000000000092A1002000000000DC690408EC
:101A56000C0000000000000094A10020000000001F
:101A6600E86904080C0000000000000096A10020B0
:101A760000000000F46904080C00000000000000EB
:101A860098A1002000000000006A04080C00000075
:101A960000000000ACA1002000000000086A040855
:101AA6000C00000000000000AAA1002000000000B9
:101AB600106A04080C00000000000000B8A1002015
:101AC600000000001C6A04080C0000000000000072
:101AD600BAA1002000000000286A04080C000000DB
:101AE60000000000C0A10020000000004C680408AF
:101AF6000C000000000000009AA100200000000079
:101B0600F86604080C00000000000000A2A10020F6
:101B160000000000346A04080C0000000000000009
:101B26009CA1002000000000406A04080C00000090
:101B3600000000009EA10020000000004C6A04087E
:101B46000C00000000000000A0A100200000000022
:101B5600546A04080C00000000000000A4A1002044
:101B660000000000FC5304080C0000000000000008
:101B7600AEA1002000000000606A04080C0000000E
:101B860000000000A6A10020000000006C6A040806
:101B96000C00000000000000B6A1002000000000BC
:101BA600786A04080C00000000000000B0A10020C4
:101BB60000000000806A04080C000000000000001D
:101BC600B2A1002000000000886A04080C00000092
:101BD60000000000BCA1002000000000906A04087C
:101BE6000C00000000000000BEA100200000000064
:101BF600AC650408010000000000000000000000C1
:101C060000000000000000000E00000000000000C0
:101C16000000000000000000986A040800000000B0
:101C2600000000000000000000000000A86A040890
:101C36000500000000000000D6A100200000000002
:101C4600AC65040801000000000000000000000070
:101C560000000000000000000E0000000000000070
:101C66000000000000000000B06A04080000000048
:101C7600000000000000000000000000185F0408DB
:101C860000000000000000000B010020040000001E
:101C9600BC6A04080D000000D5960308340E002027
:101CA60000000000946604080D000000798F030808
:101CB600280E002000000000C86904080D0000007E
:101CC6005D8F03081C0E0020000000000867040852
:101CD6000800000000000000100E002004000000B4
:101CE600F86604080D000000A98E0308040E002003
:101CF60000000000C06A040809000000000000009F
:101D0600F80D002004000000A86504080300000088
:101D160031A40308EC0D002000000000AC650408A7
:101D260001000000000000000000000000000000AC
:101D3600000000000E00000000000000000000008F
:101D460000000000C86A040800000000000000004F
:101D56000000000000000000D86A04080D00000022
:101D6600000000004C0E002000000000E06A04089D
:101D76000A0000000000000040A300200000000050
:101D8600EC6A04080A0000000000000048A30020D6
:101D960000000000F46A04080A00000000000000C9
:101DA60050A3002000000000FC6A040808000000A0
:101DB60000000000400E002000000000046B040834
:101DC60004000000419B0308000000000000000022
:101DD600AC650408010000000000000000000000DF
:101DE60000000000000000000E00000000000000DF
:101DF6000000000000000000106B04080000000056
:101E0600000000000000000000000000246B040831
:101E16000D00000000000000640E0020000000001D
:101E2600346B0408040000008999030800000000D0
:101E3600000000003C6B04080D00000000000000DC
:101E4600580E002000000000506B0408040000003B
:101E5600659903080000000000000000AC65040856
:101E6600010000000000000000000000000000006B
:101E7600000000000E00000000000000000000004E
:101E860000000000586B040800000000000000007D
:101E960000000000000000006C6B04080700000052
:101EA60000000000A00E002000000000786B04086F
:101EB6000800000000000000940E00200000000052
:101EC600846B04080800000000000000880E002053
:101ED60000000000906B04080800000000000000ED
:101EE6007C0E0020000000009C6B04080800000027
:101EF60000000000700E002000000000AC65040821
:101F060001000000000000000000000000000000CA
:101F1600000000000E0000000000000000000000AD
:101F260000000000A86B040800000000000000008C
:101F3600B708002000000000942E04080B000000E3
:101F460000000000180F002000000000B46B040819
:101F56000B000000000000000C0F00200000000035
:101F6600C06B04080B00000000000000000F0020FA
:101F760000000000CC6B04080B000000000000000D
:101F8600F40E002000000000D86B04080B000000CF
:101F960000000000E80E0020000000009C2E04084F
:101FA6000B00000000000000DC0E00200000000016
:101FB600E46B04080B00000000000000D00E0020B7
:101FC60000000000F06B040807000000000000009D
:101FD600C80E002000000000F86B0408070000008F
:101FE60000000000C00E002000000000046C040881
:101FF6000B00000000000000B40E002000000000EE
:10200600106C04080800000000000000A80E002064
:1020160000000000AC65040801000000000000009C
:102026000000000000000000000000000E0000009C
:102036000000000000000000000000001C6C040806
:10204600000000000000000000000000000000008A
:10205600306C04080800000000000000480F002053
:10206600000000003C6C04080800000000000000AE
:102076003C0F002000000000486C04080800000027
:1020860000000000300F002000000000546C04081F
:102096000800000000000000240F002000000000DF
:1020A600AC6504080100000000000000000000000C
:1020B60000000000000000000E000000000000000C
:1020C60000000000000000005C6C04080000000036
:1020D60000000000B4080020000000006C6C04083A
:1020E6000B00000000000000900F00200000000020
:1020F600786C04080B00000000000000840F00202C
:1021060000000000846C04080700000000000000C6
:102116007C0F002000000000906C040807000000FF
:1021260000000000740F0020000000009C6C0408F2
:1021360007000000000000006C0F002000000000F7
:10214600A86C04080800000000000000600F0020D2
:1021560000000000B06C0408080000000000000049
:10216600540F002000000000AC65040801000000C8
:102176000000000000000000000000000000000059
:102186000E0000000000000000000000000000003B
:10219600B86C04080000000000000000B40800202D
:1021A60000000000C46C04080700000000000000E6
:1021B600DC0F002000000000CC6C040807000000C3
:1021C60000000000D40F002000000000D46C0408BA
:1021D6000700000000000000CC0F002000000000F7
:1021E600302F04080700000000000000C40F002084
:1021F60000000000382F040807000000000000005F
:10220600BC0F002000000000402F0408070000005B
:1022160000000000B40F002000000000DC6C040881
:102226000700000000000000AC0F002000000000C6
:10223600E46C04080700000000000000A40F002062
:1022460000000000EC6C040807000000000000001D
:102256009C0F002000000000AC650408010000008F
:102266000000000000000000000000000000000068
:102276000E0000000000000000000000000000004A
:10228600000000003D920308E40F0020D4A10020C6
:102296001B000000F4290408D3A100200A32010023
:1022A600D2A1002001FA0100CEA1002000C8010041
:1022B600CCA10020E803D0070100000046465F4697
:1022C6004F5254494E4946340000000070A1002088
:1022D600000301006FA100200003010061910308C3
:1022E6003D910308C010002005910308C59003081E
:1022F600381100209D91030885910308EC110020F8
:102306005392030835990308F8140020E58E030854
:1023160000000000481500201D9B0308C194030817
:10232600241600207992030800000000D816002029
:102336001D930308ED92030864170020A993030870
:10234600F193030804180020E2A200200103010013
:10235600B99203088D9203081C1900204D930308B7
:10236600AD990308A81900201D940308099A0308CB
:10237600701A0020D8A2002001030100F46C0408A2
:102386000000000000000000000000000000000047
:10239600006D04080800000000000000901B0020EB
:1023A60000000000086D040807000000000000009F
:1023B600881B002000000000186D040807000000BC
:1023C60000000000801B002000000000246D0408AF
:1023D6000700000000000000781B0020000000003D
:1023E600306D04080D000000000000006C1B00208A
:1023F600000000003C6D04080300000031A403083F
:10240600601B002000000000AC650408010000000D
:1024160000000000000000000000000000000000B6
:102426000E00000000000000000000000000000098
:10243600446D0408000000000000000000000000D9
:1024460000000000546D04080A00000000000000AF
:102456005C2D0408000000005C6D04080A00000002
:1024660000000000182E040800000000646D040837
:102476000A000000000000001EA30020000000006B
:102486006C6D04080A000000000000009C1B002080
:1024960000000000AC650408010000000000000018
:1024A6000000000000000000000000000E00000018
:1024B600000000000000000000000000746D040829
:1024C6000000000000000000000000000000000006
:1024D600806D04080300000031A40308D41B00200B
:1024E600000000008C6D04080300000031A40308FE
:1024F600C81B002000000000946D040803000000C3
:1025060031A40308BC1B0020000000009C6D0408D9
:1025160005000000000000006EA100200000000081
:10252600A46D04080700000000000000B41B002092
:1025360000000000B06D0408070000000000000065
:10254600AC1B002000000000AC6504080100000080
:102556000000000000000000000000000000000075
:102566000E00000000000000000000000000000057
:10257600BC6D040800000000000000000000000020
:1025860000000000D06D04080300000031A4030819
:10259600F81B002000000000DC6D040803000000AA
:1025A60031A40308DC06002000000000E46D0408E6
:1025B6000300000031A40308EC1B0020000000000B
:1025C600EC6D04080300000031A40308E01B0020A2
:1025D60000000000AC6504080100000000000000D7
:1025E6000000000000000000000000000E000000D7
:1025F600000000000000000000000000F86D040864
:1026060000000000000000000000000000000000C4
:10261600046E040807000000559A0308541C0020A5
:1026260000000000506A04080300000031A40308FB
:10263600481C002000000000106E04080300000083
:1026460031A403083C1C002000000000186E04089A
:102656000300000031A40308301C00200000000025
:10266600206E040807000000399A0308281C002081
:1026760000000000C42E04080300000031A4030873
:102686001C1C0020000000002C6E04080300000043
:1026960031A40308101C002000000000386E040856
:1026A6000300000031A40308041C00200000000001
:1026B600AC650408010000000000000000000000F6
:1026C60000000000000000000E00000000000000F6
:1026D6000000000000000000F9910308B59103080E
:1026E6005C1C00208D94030800000000101D0020D3
:1026F600A99003088D9003089C1D0020000000008F
:1027060000000000501E002065940308719A03081B
:10271600DC1E0020446E04080000000000000000DB
:102726000000000000000000506E040803000000D6
:1027360031A40308E81F002000000000586E0408BA
:102746000300000031A40308DC1F00200000000085
:10275600F45404080300000031A40308D01F00202D
:1027660000000000646E04080300000031A40308A2
:10277600C41F002000000000706E04080300000063
:1027860031A40308B81F002000000000786E04087A
:102796000200000049A3030800000000000000003A
:1027A600806E04080200000049A30308010000002F
:1027B600000000008C6E04080200000049A3030814
:1027C6000200000000000000000000000E000000F3
:1027D6000000000000000000000000000060024051
:1027E6001060024000000000000B00000000200006
:1027F6000000000000000000006002402860024067
:1028060000000000060C0000000020000000000090
:10281600000000000060024040600240000000002E
:10282600100D000000002000000000000000000065
:10283600006002405860024000000000160E0000D2
:1028460000002000000000000000000000600240C0
:102856007060024000000000200F00000000200011
:102866000000000000000000006002408860024096
:1028760000000000261000000000200000000000FC
:102886000000000000600240A0600240000000005E
:1028960030110000000020000000000000000000D1
:1028A60000600240B860024000000000362F0000C1
:1028B600000020000000000000000000006402404C
:1028C60010640240000000000038000000004000D4
:1028D600000000000000000000640240286402407E
:1028E6000000000006390000000040000000000063
:1028F6000000000000640240406402400000000046
:10290600103A000000004000000000000000000037
:10291600006402405864024000000000163B0000BC
:1029260000004000000000000000000000640240BB
:102936007064024000000000203C000000004000DF
:1029460000000000000000000064024088640240AD
:1029560000000000264400000000400000000000C7
:102966000000000000640240A06402400000000075
:10297600304500000000400000000000000000009C
:1029860000640240B86402400000000036460000C1
:1029960000004000000000000000000001010000EF
:1029A600842200200000000000000000000000005B
:1029B6000000000000000000000000000000000011
:1029C6000000000000000000000000000000000001
:1029D60000000000000000000000000000000000F1
:1029E60000000000000000000000000000000000E1
:1029F60000000000000000000000000000000000D1
:102A0600000000004300000000000000000000007D
:102A160000000000000000000000000000000000B0
:102A2600000000004300000000000000000000005D
:102A36000000000000000000000000000000000090
:102A4600000000004300000000000000000000003D
:102A56000000000000000000000000000000000070
:102A6600000000004300000000000000000000001D
:102A76000000000000000000000000000000000050
:102A860000000000430000000000000000000000FD
:102A96000000000000000000000000000000000030
:102AA60000000000430000000000000000000000DD
:102AB6000000000000000000000000000000000010
:102AC60000000000430000000000000000000000BD
:102AD60000000000000000000000000000000000F0
:102AE6000000000057E6030833E603080000000074
:102AF6001F7004082E670408563704085637040862
:102B0600563704085637040856370408563704085B
:102B1600563704085637040856370408FFFFFFFFE8
:102B2600FFFFFFFFFFFFFFFFFFFF00000100415314
:102B360043494900000000000000000000000000BA
:102B460000000000000000000000000000004153EB
:102B5600434949000000000000000000000000009A
:102B6600000000000000000000000000000000005F
:042B7600010000005A
:10800000012380F8453070474FF400638382704746
:108010004FF40063838270474FF40063838270479C
:108020004FF4805383827047BFF34F8F0549064B4F
:10803000CA6802F4E0621343CB60BFF34F8F00BF06
:10804000FDE700BF00ED00E00400FA0570B4037B1B
:1080500004681F2B08D9203B2021626801FA03F332
:108060001A421CD170BC70472021226801FA03F328
:108070001A42F7D0426914495C2000FB0212516891
:108080005689CD680868296821F001012960828934
:1080900092B222EA06028281A36070BC70474269F4
:1080A00009495C2000FB021251685689CD680868B6
:1080B000296821F001012960828992B222EA060230
:1080C0008281E36070BC70476C5500202B4B19789F
:1080D000002951D02A4B30B41C6898880022626273
:1080E000A5899A80284380B20129A08143D09C6849
:1080F00098896262A589284380B20229A0819A8169
:1081000039D01C69988A6262A589284380B2032904
:10811000A0819A822FD09C69988B6262A58928439E
:1081200080B20429A0819A8325D01C6A988C62624F
:10813000A589284380B20529A0819A841BD09C6A16
:10814000988D6262A589284380B20629A0819A850C
:1081500011D01C6B988E6262A589284380B20729D2
:10816000A0819A8607D0986B998F426284892143B7
:1081700089B281819A8730BC704700BF4C5800207B
:108180005058002010B4037B01681F2B09D9203BF5
:1081900020224C6802FA03F31C4214D15DF8044B10
:1081A000704720220C6802FA03F31C42F6D00C4AF6
:1081B00040680024147002685DF8044B22F001024C
:1081C00002608B607047064A4068002414700268A1
:1081D0005DF8044B22F001020260CB60704700BFE3
:1081E000AC680020F0B5876983B0064617B13B68DC
:1081F000BA885A837069DFF8A4E08389C3244FF4F6
:108200007A734FF0060C6D464FF6FF710EF1010EBA
:1082100003E0013B9BB28B4220D002899207F8D544
:10822000A3B283814FF47A7302E0A3B28B4215D0DC
:108230000289D20703F1FF34F7D5828992B20DB1DA
:108240002A700135BCF1000F0BD00CF1FF3CFF246C
:10825000BEF1000FE1D09EF80040D7E715F04FFBCC
:10826000B76917B13B68BA881A839DF805009DF875
:1082700001509DF802109DF803409DF804209DF8E0
:10828000063041EA052143EA002342EA04220120A4
:1082900031877287B38703B0F0BD00BF90F8030841
:1082A0002DE9F04F87B0029090F85500002840F07B
:1082B0001985029A137C1032022B039204D11046C6
:1082C0006B21802215F036FBB54CB64DDFF8DC9201
:1082D000B548DFF8DCE24FF0640A4FF0100C4FF4C1
:1082E0007A76D9F80430C3F30803002B40F0FC83FE
:1082F000EFF31183002B40F0F7832168826800BF01
:1083000023689942F9D12F6806FB07F39B1AB3FB48
:10831000F7F306FB013101270191D9F80430C3F3CB
:108320000803002B40F0C383EFF31183002B40F0D0
:10833000BE832368816800BF22689342F9D1D5F8D3
:1083400000B006FB0BF2521AB2FBFBF206FB032352
:10835000019A9B1AB3F57A7FDFD3BAF1010AC0D133
:10836000029B1B7C022B04D107226821039815F085
:10837000E1FADFF838928C4EDFF834C24FF0640A2D
:108380004FF010084FF47A77D9F80430C3F308039C
:10839000002B40F01A84EFF31183002B40F015847A
:1083A0002168B26800BF23689942F9D1286807FBA9
:1083B00000F39B1AB3FBF0F307FB0131012001919D
:1083C000D9F80430C3F30803002B40F05383EFF3D4
:1083D0001183002B40F04E832368B16800BF2268F0
:1083E0009342F9D1D5F800B007FB0BF2521AB2FB59
:1083F000FBF207FB0323019A9B1AB3F57A7FDFD3C5
:10840000BAF1010AC0D1029B1B7C022B04D1524657
:108410006B21039815F08EFADFF890916248DFF82F
:1084200090E14FF0640A4FF0100C4FF47A76D9F8CF
:108430000430C3F30803002B40F0AB83EFF3118348
:10844000002B40F0A6832168826800BF2368994210
:10845000F9D12F6806FB07F39B1AB3FBF7F306FB72
:10846000013101270191D9F80430C3F30803002B2F
:1084700040F0E382EFF31183002B40F0DE822368AB
:10848000816800BF22689342F9D1D5F800B006FB9D
:108490000BF2521AB2FBFBF206FB0323019A9B1A62
:1084A000B3F57A7FDFD3BAF1010AC0D1029B1B7CFE
:1084B000022B04D101226B21039815F03BFADFF85F
:1084C000EC903948DFF8E8E04FF00F0A4FF0100C5D
:1084D0004FF47A76D9F80430C3F30803002B40F048
:1084E0003C83EFF31183002B40F0378321688268CF
:1084F00000BF23689942F9D12F6806FB07F39B1A46
:10850000B3FBF7F306FB013101270191D9F80430E1
:10851000C3F30803002B40F07382EFF31183002BA9
:1085200040F06E822368816800BF22689342F9D1CF
:10853000D5F800B006FB0BF2521AB2FBFBF206FBB9
:108540000323019A9B1AB3F57A7FDFD3BAF1010AAC
:10855000C0D1029991F84F200B7C042A34BF182215
:108560001A22022B03D11B21039815F0E3F9DFF83F
:108570003C900D48DFF838E04FF00F0A4FF0100C38
:108580004FF47A76D9F80430C3F30803002B40F097
:10859000C882EFF31183002B40F0C3820AE000BFD2
:1085A000E4A70020E8A7002010E000E000ED00E0D4
:1085B000E0A700202168826800BF23689942F9D1B2
:1085C0002F6806FB07F39B1AB3FBF7F306FB013199
:1085D00001270191D9F80430C3F30803002B40F0C0
:1085E000F281EFF31183002B40F0ED812368816865
:1085F00000BF22689342F9D1D5F800B006FB0BF218
:10860000521AB2FBFBF206FB0323019A9B1AB3F545
:108610007A7FDFD3BAF1010AB4D1029B1B7C022B13
:1086200004D118221C21039815F084F9DFF8E09298
:10863000B648DFF8E0E24FF00F0A4FF0100C4FF4AD
:108640007A76D9F80430C3F30803002B40F02E8368
:10865000EFF31183002B40F029832168826800BF6B
:1086600023689942F9D12F6806FB07F39B1AB3FBE5
:10867000F7F306FB013101270191D9F80430C3F368
:108680000803002B40F08281EFF31183002B40F0B0
:108690007D812368816800BF22689342F9D1D5F8B3
:1086A00000B006FB0BF2521AB2FBFBF206FB0323EF
:1086B000019A9B1AB3F57A7FDFD3BAF1010AC0D1D0
:1086C000029B1B7C022B06D1029B039893F84E2041
:1086D0001A2115F02FF9DFF838928C48DFF834E2D0
:1086E0004FF00F0A4FF0100C4FF47A76D9F804309F
:1086F000C3F30803002B40F0BD82EFF31183002B7E
:1087000040F0B8822168826800BF23689942F9D19D
:108710002F6806FB07F39B1AB3FBF7F306FB013147
:1087200001270191D9F80430C3F30803002B40F06E
:108730001081EFF31183002B40F00B8123688168D7
:1087400000BF22689342F9D1D5F800B006FB0BF2C6
:10875000521AB2FBFBF206FB0323019A9B1AB3F5F4
:108760007A7FDFD3BAF1010AC0D1029B1B7C022BB6
:1087700006D1029B039893F85020192115F0DAF8DE
:10878000DFF88C916148DFF88CE14FF0640A4FF01C
:10879000100C4FF47A76D9F80430C3F30803002B99
:1087A00040F04C82EFF31183002B40F047822168A8
:1087B000826800BF23689942F9D12F6806FB07F34E
:1087C0009B1AB3FBF7F306FB013101270191D9F89E
:1087D0000430C3F30803002B40F09E80EFF31183B5
:1087E000002B40F099802368816800BF2268934283
:1087F000F9D1D5F800B006FB0BF2521AB2FBFBF22E
:1088000006FB0323019A9B1AB3F57A7FDFD3BAF1F3
:10881000010AC0D1029B1B7C022B04D110223721FC
:10882000039815F087F8DFF8E8903848DFF8E4E0BF
:108830004FF00F0A4FF0100C4FF47A76D9F804304D
:10884000C3F30803002B40F0DD81EFF31183002B0D
:1088500040F0D8812168826800BF23689942F9D12D
:108860002F6806FB07F39B1AB3FBF7F306FB0131F6
:1088700001270191D9F80430C3F3080343BBEFF398
:1088800011832BBB2368816800BF22689342F9D112
:10889000D5F800B006FB0BF2521AB2FBFBF206FB56
:1088A0000323019A9B1AB3F57A7FE3D3BAF1010A45
:1088B000C4D1029B1B7C022B04D1039801223821D6
:1088C00015F038F80F2006F0EBFB07B0BDE8F08F8D
:1088D000EFF311888CF3128881680368DB0344BFCF
:1088E000CEF8007081682368DEF800205FFA88F80F
:1088F00088F31188D5F800801A4406FB08F35B1A48
:10890000B3FBF8F306FB0233CBE700BF10E000E057
:1089100000ED00E0E0A70020EFF311888CF312884F
:1089200081680368DB0344BFCEF800708168236868
:10893000DEF800205FFA88F888F31188D5F8008007
:108940001A4406FB08F35B1AB3FBF8F306FB023389
:1089500058E7EFF311888CF3128881680368DB0312
:1089600044BFCEF8007081682368DEF800205FFA0B
:1089700088F888F31188D5F800801A4406FB08F3BC
:108980005B1AB3FBF8F306FB0233E6E6EFF311885C
:108990008CF3128881680368DB0344BFCEF8007053
:1089A00081682368DEF800205FFA88F888F3118870
:1089B000D5F800801A4406FB08F35B1AB3FBF8F302
:1089C00006FB023374E6EFF311888CF3128881689A
:1089D0000368DB0344BFCEF8007081682368DEF8CB
:1089E00000205FFA88F888F31188D5F800801A44CF
:1089F00006FB08F35B1AB3FBF8F306FB023304E64D
:108A0000EFF311888CF3128881680368DB0344BF9D
:108A1000CEF8007081682368DEF800205FFA88F8DD
:108A200088F31188D5F800801A4406FB08F35B1A16
:108A3000B3FBF8F306FB023383E5EFF311888CF305
:108A4000128881680368DB0344BFCEF80070816838
:108A50002368DEF800205FFA88F888F31188D5F8DB
:108A600000801A4406FB08F35B1AB3FBF8F306FB1D
:108A7000023313E5EFF3118E88F31288B16833687F
:108A8000DB0344BFCCF80000B1682368DCF80020A9
:108A90005FFA8EFE8EF31188D5F800E01A4407FBCA
:108AA0000EF35B1AB3FBFEF307FB0233A3E4EFF311
:108AB00011888CF3128881680368DB0344BFCEF809
:108AC000007081682368DEF800205FFA88F888F378
:108AD0001188D5F800801A4406FB08F35B1AB3FB33
:108AE000F8F306FB023333E4EFF311828CF31288C0
:108AF00087680368D90303D50123CEF8003087685F
:108B00002368DEF80010D2B282F311882A68194473
:108B100006FB02F3DB1BB3FBF2F306FB0131FFF7AD
:108B2000FABBEFF311828CF3128887680368D903CC
:108B300003D50123CEF8003087682368DEF80010E3
:108B4000D2B282F311882A68194406FB02F3DB1BB8
:108B5000B3FBF2F306FB01313AE5EFF311828CF33C
:108B6000128887680368D90303D50123CEF8003043
:108B700087682368DEF80010D2B282F311882A6871
:108B8000194406FB02F3DB1BB3FBF2F306FB0131D6
:108B9000BAE4EFF311828CF3128887680368D90373
:108BA00003D50123CEF8003087682368DEF8001073
:108BB000D2B282F311882A68194406FB02F3DB1B48
:108BC000B3FBF2F306FB01314BE4EFF3118288F3C0
:108BD0001288B0683368D90303D50123CCF800307C
:108BE000B0682368DCF80010D2B282F311882A68DA
:108BF000194407FB02F31B1AB3FBF2F307FB013125
:108C0000FFF7DCBBEFF311828CF3128887680368EF
:108C1000D90303D50123CEF8003087682368DEF836
:108C20000010D2B282F311882A68194406FB02F3BD
:108C3000DB1BB3FBF2F306FB013119E6EFF3118204
:108C40008CF3128887680368D90303D50123CEF813
:108C5000003087682368DEF80010D2B282F31188F2
:108C60002A68194406FB02F3DB1BB3FBF2F306FB95
:108C70000131AAE5EFF311828CF31288876803684B
:108C8000D90303D50123CEF8003087682368DEF8C6
:108C90000010D2B282F311882A68194406FB02F34D
:108CA000DB1BB3FBF2F306FB013139E5EFF3118275
:108CB0008CF3128887680368D90303D50123CEF8A3
:108CC000003087682368DEF80010D2B282F3118882
:108CD0002A68194406FB02F3DB1BB3FBF2F306FB25
:108CE0000131C8E405F0DEFD0446002838D00068F4
:108CF000A58802692A407FF4DCAA00F13F4303F50E
:108D00007E039B0A2249E271CA5C02F01F065209E7
:108D100001232021032A03FA06F3A17132D0042A89
:108D20002BD0022A24D0002304A90593049529F00E
:108D300063FF0299174B41F80C3F204632F02EFAA0
:108D4000A388B3FA83F3C3F11F03012212FA03F3DA
:108D50003FF4AFAA10490A6813430B60FFF7A9BAA2
:108D600002990C4B41F80C3F32F018FAFFF7A1BA08
:108D70000A4A516C0B435364D5E7084A116B0B4305
:108D80001363D0E7054A116C0B431364CBE700BFB4
:108D9000742B040801800008003C014000380240A8
:108DA0002DE9F04FAC4A436983B09342019000F043
:108DB000A281AA498B420CBF282130211A88A84CD5
:108DC000DFF8A882A74E22F040021204120C1A808B
:108DD0001A8892B222F03802114319801A8892B28E
:108DE00042F040021A8006F0B5F8DFF884E29E49AE
:108DF000844610274FF47A750120DEF80430C3F35F
:108E00000803002B40F03681EFF31183002B40F074
:108E100031812368D1F8089000BF22689342F8D1CD
:108E2000D8F800A005FB0AF2A2EB0902B2FBFAF2A5
:108E300005FB03239C45E0D0019D2846FFF730FA4F
:108E4000AB6913B11A689B885383019B586940F240
:108E5000E93302E0002B00F046810289013B12F069
:108E6000020F9BB2F6D06A23838140F2E93302E01D
:108E7000002B00F038810289013B12F0010F9BB2F8
:108E8000F6D0838940F2E93302E0002B00F0308114
:108E90000289013B12F0020F9BB2F6D010238381AE
:108EA00040F2E93302E0002B00F022810289013B0D
:108EB00012F0010F9BB2F6D08389019B9B6913B11D
:108EC0001A689B881383DFF8A8916748654F4FF0B5
:108ED000640A4FF0100E4FF47A75D9F80430C3F3DA
:108EE0000803002B40F0E480EFF31183002B40F0E7
:108EF000DF802168826800BF23689942F9D1D8F8E1
:108F0000006005FB06F39B1AB3FBF6F305FB01318A
:108F100001260091D9F80430C3F30803002B63D174
:108F2000EFF31183002B5FD12368816800BF2268B3
:108F30009342F9D1D8F800B005FB0BF2521AB2FBFC
:108F4000FBF205FB0323009A9B1AB3F57A7FE1D36A
:108F5000BAF1010AC1D1019B3F4A5B69934207D034
:108F6000DFF8F8A0534514BF4FF0080A4FF0000A8D
:108F70001A883D4D3B4F22F040021204120C1A8019
:108F80001A8892B222F038024AEA020AA3F800A034
:108F90001A8892B242F040021A8005F0DBFFDFF837
:108FA000D0C081464FF0100E4FF47A760120DCF8E5
:108FB0000430C3F30803002B31D1EFF3118373BBEB
:108FC0002368A96800BF22689342F9D1D8F800A0AD
:108FD00006FB0AF2521AB2FBFAF206FB032399458A
:108FE000E5D003B0BDE8F08FEFF3118C8EF312885B
:108FF00081680368DA0344BF3E60816823683A6889
:109000005FFA8CFC8CF31188D8F800C01A4405FB79
:109010000CF35B1AB3FBFCF305FB023393E7EFF3AE
:1090200011818EF31288D5F808A02B68DB0344BFAA
:109030003860D5F808A023683A68C9B281F311886E
:10904000D8F800101A4406FB01F3A3EB0A03B3FBA4
:10905000F1F306FB0233C2E700380040003C004059
:10906000E4A70020E0A7002010E000E0E8A700202F
:1090700000ED00E0EFF3118987F31288D1F808A022
:109080000B68DB0344BF3060D1F808A02368326866
:109090005FFA89F989F31188D8F800901A4405FB22
:1090A00009F3A3EB0A03B3FBF9F305FB0233C1E6B3
:1090B000EFF311828EF3128886680368D90302D514
:1090C00001233B60866823683968D2B282F3118835
:1090D000D8F80020194405FB02F39B1BB3FBF2F305
:1090E00005FB013114E714F00AFC019B5869C9E63D
:1090F00014F005FCE1E6282160E600BFF8B5057B29
:10910000466903681F2D29D9A5F120045F68202135
:10911000A1400F422A4613D01022A240D960DA6043
:109120005A68E240D10703D5012202FA04F4DC6058
:109130000446304606F084F8227B23681F2A20D993
:10914000A2F1200008215A688140114200D0D96064
:109150000422596882400A4221D1F8BD20211C68AE
:10916000A9400C422A460CD01022AA4099609A606D
:109170001A68EA40D207DBD5012202FA05F59D60A4
:10918000D6E7082118689140014200D09960042177
:10919000186801FA02F2024203D09A60F8BDDA6060
:1091A000F8BDF8BD144B984224D003F58063984273
:1091B00020D0028822F040021204120C02800288A1
:1091C00022F038031B041B0C59B141F480710029B3
:1091D00091FAA1F2B2FA82F108BF4FF0FF310139E2
:1091E000C9000B439BB2038003889BB243F040034A
:1091F000038070474908DCE70038004008B540F2BA
:10920000E93300E0A3B10289013B12F0020F9BB2E7
:10921000F8D089B2818140F2E93300E043B102899C
:10922000013B12F0010F9BB2F8D08089C0B208BD9B
:1092300014F065FBC0B208BD38B504460D4600BF4A
:10924000806806F0A3FA29466068FFF7D7FFA06898
:1092500006F0A2FA00BF38BD66496748674A2DE9A3
:10926000F84F012303700B88128823F040031B047E
:109270001B0C0B800B8823F038031B0452084FEAA9
:1092800013430BD042F48072002A92FAA2F1B1FA91
:1092900081F208BF4FF0FF32013AD2001343554A22
:1092A0009BB2138013889BB243F040031380544B4E
:1092B0001B6813B11A689B88538305214D48DFF85A
:1092C0004881504FFFF79AFF00214A48FFF796FF69
:1092D00006214848FFF792FF00214648FFF78EFF1E
:1092E00098F8004043480421FFF788FF44F001014B
:1092F0004048FFF783FF3B88002B45D0DFF80CA1E7
:109300003C4C08F103094FF0000B07269AF8015076
:1093100040F2E93301E0002B63D02089013B10F0DB
:10932000020F9BB2F7D0A68140F2E93301E0002B97
:1093300057D02089013B10F0010F9BB2F7D0A389D1
:1093400040F2E93301E0002B4FD02089013B10F0BF
:10935000020F9BB2F7D0ADB2A58140F2E93301E034
:10936000002B42D02089013B10F0010F9BB2F7D0B7
:10937000A3893B881AF8010F09F8010F0BF1010BC3
:109380009B45C3DB98F800401A480721FFF736FFDA
:10939000FF211848FFF732FF04211648FFF72EFF80
:1093A00021461448FFF72AFF154B1B6813B11A68B2
:1093B0009B8813830F4A138823F040031B041B0C64
:1093C0001380138823F038031B041B0C13801388AD
:1093D0009BB243F040031380074B00211970BDE896
:1093E000F88F204614F08BFAAAE7204614F087FA8B
:1093F000BFE700BF003C0040815400204002002035
:10940000A0960020F4000020582400207352002071
:10941000A6490A8822F040022DE9F0471204A44F21
:10942000120C3B880A800A8822F0380212045B087A
:109430004FEA124200F0388143F4807090FAA0F1B4
:109440000028B1FA81F108BF4FF0FF310139C9009E
:109450000A439649974D92B20A800A8892B242F026
:1094600040020A80296811B10A6888885083924AAC
:109470001278012A00F04981C0F03081022A40F0C0
:10948000FF808E4E082232704FF4C372DFF848829C
:109490008648A8F80020028822F040021204120C2C
:1094A0000280028822F038021204120C5BB143F4ED
:1094B000807090FAA0F30028B3FA83F308BF4FF04E
:1094C000FF33013BDB001343784A9BB213801388C0
:1094D0009BB243F04003138011B10B688A885A8312
:1094E000724C4FF010094FF0010A40F2E93302E0EC
:1094F000002B00F0CF802289013B12F0020F9BB2BB
:10950000F6D01FFA89F3A38140F2E93302E0002B81
:1095100000F0C0802289013B12F0010F9BB2F6D00F
:10952000A38940F2E93302E0002B00F0B7802289E2
:10953000013B12F0020F9BB2F6D0A4F80CA040F24F
:10954000E93302E0002B00F0A9802289013B12F0F0
:10955000010F9BB2F6D0A38909F10109B9F1200FDF
:10956000C3D1296811B10B688A881A834F4B1A88B6
:1095700022F040021204120C1A801A8822F03802DB
:109580001204120C1A801A8892B242F040021A8019
:1095900018883A8820F040000004000C18801B88CE
:1095A00023F038031B0452084FEA13430BD042F454
:1095B0008072002A92FAA2F0B0FA80F208BF4FF04F
:1095C000FF32013AD2001343384A9BB2138013880A
:1095D0009BB243F04003138011B10B688A885A8311
:1095E000347832480021FFF709FE21462F48FFF763
:1095F00005FE334B2D481C780221FFF7FFFD214665
:109600002A48FFF7FBFD2F4B28481C780321FFF762
:10961000F5FD21462548FFF7F1FD2B4B23481C782B
:1096200004210C43FFF7EAFD21462048FFF7E6FD41
:109630002B6813B11A689B8813831C4A234C138828
:10964000234823F040031B041B0C1380138823F0D2
:1096500038031B041B0C138013889BB243F0400398
:109660001380B8F80020002136F0A3F82378CBB19E
:10967000184B1B78002B4ED000232370BDE8F087D9
:109680000E4E327812F0400F0CBF4FF4C3724FF4FD
:10969000F072FBE6204614F032F942E7204614F05F
:1096A0002EF959E7BDE8F0871946D1E6003C0040A5
:1096B00040020020A0960020B4960020F600002072
:1096C000BB960020BC9600205824002000000020FB
:1096D0005C24002081540020F4000020A0211448C4
:1096E000FFF78CFD00211248FFF788FD00F006030C
:1096F000022B03D000F00500012812D00D4E3B884C
:109700002968082232705B08BEE60A4E4822327091
:109710004FF4F072BAE6FFF79FFD00232370BDE817
:10972000F087044E3B882968482232705B08EFE7D7
:10973000003C0040F60000202DE9F04F85B001907C
:1097400090F85500002840F06F82019C4FF4807122
:109750006069FFF727FDA36913B11A689B885383DB
:10976000019C6B216069FFF749FD80216069FFF76B
:1097700045FDA36913B11A689B8813839E4C9F4DC6
:10978000DFF880929E48DFF880E24FF0640A4FF0E5
:10979000100C4FF47A76D9F80430C3F30803002B89
:1097A00040F0EE81EFF31183002B40F0E981216856
:1097B000826800BF23689942F9D12F6806FB07F33E
:1097C0009B1AB3FBF7F306FB013101270091D9F88F
:1097D0000430C3F30803002B40F0B581EFF311838D
:1097E000002B40F0B0812368816800BF226893425B
:1097F000F9D1D5F800B006FB0BF2521AB2FBFBF21E
:1098000006FB0323009A9B1AB3F57A7FDFD3BAF1E4
:10981000010AC0D1019B9B6913B11A689B885383CD
:10982000019E68217069FFF7E9FC03217069FFF769
:10983000E5FCB36913B11A689B881383642005F0B3
:109840002FFC019B9B6913B11A689B885383019E6F
:109850006B217069FFF7D2FC01217069FFF7CEFC24
:10986000B36913B11A689B881383DFF89891644831
:10987000DFF894E14FF00F0A4FF0100C4FF47A76B6
:10988000D9F80430C3F30803002B40F0B181EFF3A3
:109890001183002B40F0AC812168826800BF2368EF
:1098A0009942F9D12F6806FB07F39B1AB3FBF7F334
:1098B00006FB013101270091D9F80430C3F30803F6
:1098C000002B40F02381EFF31183002B40F01E8129
:1098D0002368816800BF22689342F9D1D5F800B0AF
:1098E00006FB0BF2521AB2FBFBF206FB0323009AB3
:1098F0009B1AB3F57A7FDFD3BAF1010AC0D101997F
:1099000091F84F208B69042A34BF18261A2613B108
:109910001A689B885383019F1B217869FFF76EFCAF
:1099200031467869FFF76AFCBB6913B11A689B88F6
:1099300013830F2005F0B4FB019B9B6913B11A68D8
:109940009B885383019E1C217069FFF757FC1821E7
:109950007069FFF753FCB36913B11A689B881383CE
:109960000F2005F09DFB019A936992F84E6013B1A8
:109970001A689B885383019F1A217869FFF73EFC80
:1099800031467869FFF73AFCBB6913B11A689B88C6
:109990001383DFF870901A48DFF86CE04FF00F0A7D
:1099A0004FF0100C4FF47A76D9F80430C3F3080363
:1099B000002B40F00181EFF31183002B40F0FC807D
:1099C0002168826800BF23689942F9D12F6806FB9D
:1099D00007F39B1AB3FBF7F306FB01310127009154
:1099E000D9F80430C3F30803002B72D1EFF31183CD
:1099F000002B6ED10AE000BFE4A70020E8A70020FA
:109A000010E000E000ED00E0E0A70020236881689E
:109A100000BF22689342F9D1D5F800B006FB0BF2E3
:109A2000521AB2FBFBF206FB0323009A9B1AB3F512
:109A30007A7FD5D3BAF1010AB6D1019A936992F827
:109A4000504013B11A689B885383019D192168699E
:109A5000FFF7D4FB21466869FFF7D0FBAB6913B170
:109A60001A689B881383642005F01AFB019B9B698D
:109A700013B11A689B885383019C37216069FFF7F3
:109A8000BDFB10216069FFF7B9FBA36913B11A6828
:109A90009B8813830F2005F003FB019B9B6913B187
:109AA0001A689B885383019C38216069FFF7A6FBE5
:109AB00001216069FFF7A2FBA36913B11A689B88B3
:109AC0001383019B08215869FFF76CFB05B0BDE8C3
:109AD000F08FEFF311888CF3128881680368DB0341
:109AE00044BFCEF8007081682368DEF800205FFA7A
:109AF00088F888F31188D5F800801A4406FB08F32B
:109B00005B1AB3FBF8F306FB02338EE7EFF3118821
:109B10008CF3128881680368DB0344BFCEF80070C1
:109B200081682368DEF800205FFA88F888F31188DE
:109B3000D5F800801A4406FB08F35B1AB3FBF8F370
:109B400006FB0233D3E6EFF311888CF312888168A9
:109B50000368DB0344BFCEF8007081682368DEF839
:109B600000205FFA88F888F31188D5F800801A443D
:109B700006FB08F35B1AB3FBF8F306FB023341E67E
:109B8000EFF311828CF3128887680368D90303D539
:109B90000123CEF8003087682368DEF80010D2B2C7
:109BA00082F311882A68194406FB02F3DB1BB3FB1E
:109BB000F2F306FB013108E6EFF311828CF3128811
:109BC00087680368D90303D50123CEF8003087687E
:109BD0002368DEF80010D2B282F311882A68194493
:109BE00006FB02F3DB1BB3FBF2F306FB0131F5E6E8
:109BF000EFF311828CF3128887680368D90303D5C9
:109C00000123CEF8003087682368DEF80010D2B256
:109C100082F311882A68194406FB02F3DB1BB3FBAD
:109C2000F2F306FB013145E604F03CFE0446002851
:109C300037D00068A58802692A407FF486AD00F11C
:109C40003F4303F57E039B0A2149E271CA5C02F09F
:109C50001F06520901232021032A03FA06F3A171EA
:109C600030D0042A29D0022A22D0002302A903934B
:109C7000029528F0C1FF0199164B41F80C3F204690
:109C800031F08CFAA388B3FA83F3C3F11F030122E6
:109C900012FA03F33FF459AD0F490A6813430B60FE
:109CA00053E501990B4B41F80C3F31F077FA4CE545
:109CB0000A4A516C0B435364D7E7084A116B0B43B4
:109CC0001363D2E7054A116C0B431364CDE700BF61
:109CD000742B040801800008003C01400038024059
:109CE0002DE9F84FA04F3B7803B1FEE79F4CA04A07
:109CF00001233B702388128823F040031B041B0CB4
:109D00002380238823F038031B0452084FEA1343AF
:109D10000BD042F48072002A92FAA2F4B4FA84F2D0
:109D200008BF4FF0FF32013AD20013438F4ADFF8E9
:109D30004C829BB2138013889BB243F04003138084
:109D4000D8F8003013B11A689B885383894B8A4E28
:109D500001220D468146002184481A70FFF74EFA11
:109D6000824800210446FFF749FA09212046FFF7FF
:109D700045FA49462046FFF741FA013D4FF0000AF7
:109D80004FF00A0B40F2E93302E0002B00F0D280E2
:109D90002289013B12F0020F9BB2F6D0A4F80CB05E
:109DA00040F2E93302E0002B00F0C4802289013B3D
:109DB00012F0010F9BB2F6D0A38940F2E93302E022
:109DC000002B00F0BB802289013B12F0020F9BB2F6
:109DD000F6D01FFA8AF3A38140F2E93302E0002BA8
:109DE00000F0AC802289013B12F0010F9BB2F6D04B
:109DF000A38915F8019F40F2E93302E0002B00F03F
:109E0000A1802289013B12F0020F9BB2F6D00B23F6
:109E1000A38140F2E93302E0002B00F09380228915
:109E2000013B12F0010F9BB2F6D0A38940F2E93357
:109E300002E0002B00F08A802289013B12F0020F21
:109E40009BB2F6D01FFA89F9A4F80C9040F2E933DE
:109E500001E0002B7AD02289013B12F0010F9BB266
:109E6000F7D0A389336833B11A689B8851690B42D4
:109E700014BF538313830AF1010ABAF1360F81D15B
:109E80003A4808210446FFF7B9F9A0212046FFF718
:109E9000B5F9A02540F2E93301E0002B5AD0228920
:109EA000013B12F0020F9BB2F7D0A58140F2E933DB
:109EB00001E0002B4ED02289013B12F0010F9BB232
:109EC000F7D0A38940F2E93301E0002B46D0228984
:109ED000013B12F0020F9BB2F7D00023A38140F2A6
:109EE000E93301E0002B39D02289013B12F0010F48
:109EF0009BB2F7D0A089C0B28306CBD4D8F800308B
:109F000013B11A689B881383184A138823F04003FF
:109F10001B041B0C1380138823F038031B041B0C39
:109F2000138013889BB243F04003002113803970E3
:109F3000BDE8F88F204613F0E2FC3EE7204613F020
:109F4000DEFC56E7204613F0DAFC6FE7204613F0FC
:109F5000D6FC87E7204613F0D2FCB3E7204613F087
:109F6000CEFCC0B2C8E700BF81540020003C0040D6
:109F70004002002089540020B0A70020A0960020B5
:109F800030B4147874B11E23074D13FB010129442A
:109F9000801A83181D2BD8BF0C7012F8014F0131A5
:109FA000002CF6D130BC704774520020F8B5434CF9
:109FB000434A2388128823F040031B041B0C238090
:109FC0002388C1F1030123F0380341EA80071B0411
:109FD0005208FFB24FEA13430BD042F48072002ABA
:109FE00092FAA2F1B1FA81F208BF4FF0FF32013AC2
:109FF000D2001343314A334D9BB2138013889BB276
:10A0000043F0400313802B6813B11A689B88538375
:10A010002A4CBFB2102640F2E93301E0002B45D0B4
:10A020002289013B12F0020F9BB2F7D0B3B2A38199
:10A0300040F2E93301E0002B38D02289013B12F0D5
:10A04000010F9BB2F7D0A38940F2E93301E0002B66
:10A0500030D02289013B12F0020F9BB2F7D0A781CA
:10A0600040F2E93300E02BB32289013B12F0010FEB
:10A070009BB2F8D0A3890136202ECCD12B6813B126
:10A080001A689B8813830D4A138823F040031B042E
:10A090001B0C1380138823F038031B041B0C138044
:10A0A00013889BB243F040031380F8BD204613F0A1
:10A0B00026FCC9E7204613F022FCDCE7003C004008
:10A0C00040020020A096002038B5384B1D780028AB
:10A0D00064D105F0F70536491D700A88354B22F02A
:10A0E00040021204120C1B880A800A8822F03802EF
:10A0F00012045B084FEA12420BD043F48073002B2A
:10A1000093FAA3F1B1FA81F308BF4FF0FF33013B9B
:10A11000DB001343264A284C9BB2138013889BB262
:10A1200043F040031380236813B11A689B8853835C
:10A1300040F2E9331E4801E0002B32D00289013B96
:10A1400012F0020F9BB2F7D00423838140F2E9336F
:10A15000174800E02BB30289013B12F0010F9BB2BC
:10A16000F8D0838912482946FFF748F8236813B1CD
:10A170001A689B8813830E4A138823F040031B043C
:10A180001B0C1380138823F038031B041B0C138053
:10A1900013889BB243F04003138038BD45F0080597
:10A1A00099E7034813F0ABFBDCE700BF582400201D
:10A1B000003C004040020020A09600200C4B98423A
:10A1C00013D0A3F5806398420FD003F580439842E3
:10A1D0000BD003F58063984207D003F58063984263
:10A1E00003D0044B186840087047024B186870474A
:10A1F00000040140E8A80020F0B5774B774A87B00B
:10A200001968914200AF00F0DB800023744A3B6084
:10A210007B60136843F48033136003E03B68B3F55D
:10A22000A04F09D0136803F400337B603B6801330F
:10A230003B607B68002BF1D0694B1B6813F4003343
:10A2400018BF01237B607B68012B7BD0654D644B7D
:10A25000654AEA606549586F654A0860AA605E6BA6
:10A26000644C654A654826F080065E635E6F46F082
:10A2700080765E67196B0C431C63596B5963996B4D
:10A280009963196C41F05B5141F47B1141F41F61FA
:10A2900041F00F011964596C07F118040A4348F2A0
:10A2A000FF715A6444F8101D002621460123FB73F8
:10A2B0003E737E73BE7328F09FFC21464FF6FF73FA
:10A2C0004F48BB6028F098FC4FF6FF7321464D487D
:10A2D000BB6028F091FC21464B4828F08DFC2146BC
:10A2E0004A4828F089FC2146494828F085FC214647
:10A2F000484828F081FC2146474828F07DFC21464B
:10A30000464828F079FC204628F034FA444B454C66
:10A310001B68BA6844484549A4FB03439B09A0FB5A
:10A320000202013B920CB3F1807F0A6007D2404ADF
:10A33000F0200721536085F82300966011601C37D8
:10A34000BD46F0BD264B3B4C1A6C3B4942F0805257
:10A350001A6420688A684D68C96840F440402060EB
:10A36000986898609868120640F40040986042EA45
:10A370008512986842F48002490842F008020139C7
:10A3800042EA014240F4A05098605A601A6842F0D4
:10A3900080721A601A689201FCD52849104A40F26E
:10A3A00005700860996821F003019960996841F08F
:10A3B00002019960936803F00C03082BFAD145E77A
:10A3C00000221A6062B61E4B1B6883F308881D4B7F
:10A3D0001B689847FEE700BFFCFF0120EFBEADDE23
:10A3E0000038024000ED00E00005FA05C0580020EA
:10A3F00000000008FF916700335F07000000024083
:10A400000004024000080240000C0240001002401C
:10A410000014024000180240001C024000200240CC
:10A42000E8A80020D34D621083DE1B43E8A700207C
:10A4300010E000E00070004000000020003C0240FE
:10A440000000FF1F0400FF1F08B5054B1B6803B188
:10A450009847044B044A1A6072B6FDF7E5FD00BF49
:10A460000C4A0020FCFF0120EFBEADDE08B5034B17
:10A470001B6803B1984772B6FDF7D6FD0C4A002061
:10A4800038B5436B044673B1A36DA26BD2B1998A00
:10A490001A88C90592B201D5D20700D438BD4FF64B
:10A4A000F7721A8038BD836D99891A88890692B22D
:10A4B000EBD59206E9D5C26AD2B19888216B80B2F9
:10A4C0009047E1E799891A880D0692B2DFD5100608
:10A4D000DDD5A26A616A8A4219D0A1692569885CC2
:10A4E00098800132B2FBF5F105FB1122A262CEE7A2
:10A4F0009B88E2696169DBB28B54E269E068A36D15
:10A500000132B2FBF0F100FB1122E261BDE7DA6833
:10A5100022F08002DA60BAE72DE9F04F7A4C54F865
:10A52000204083B0002C00F0EA80D4F86090B9F1AC
:10A53000000F00F0E680D9F81050D9F80470734E7F
:10A54000A16004F166012660616104F266264FF4A1
:10A550000071A661E1602161A765A0464DB3DFF8F7
:10A56000B4C14FF0000E61464E68B54201F11C01C6
:10A5700006D00EF1010EBEF1100FF5D14FF0000E16
:10A58000CEEBCE0E0CEB8E01DFF884C10E69DCF849
:10A5900030E04FF00C0A4EEA060E461CCCF830E0D4
:10A5A00081F818A04E76D9F80810E1630437676582
:10A5B00065630546D9F80C001F46164600283CD0B6
:10A5C000DFF850C1002163465A68904203F11C0332
:10A5D00003D001311029F7D10021C1EBC1010CEBEF
:10A5E00081014B4B0A69186BDFF82CE110431863AB
:10A5F0000B200876681C4876186B024399F81F00F8
:10A600001A63830991F80DC08DF8053000220123EB
:10A610004C61C1F808E001A88DF806208DF80730DC
:10A620008DF804C028F05EF8A36DD9F80810D9F8A9
:10A630000C20A26304332164236594F8650004F0C0
:10A6400031F9824694F8640004F02CF9834699F8B5
:10A650001C00002850D1380739D4B2070ED5BAF102
:10A66000000F0BD00B226B1C8AF806208AF80730EB
:10A67000504699F81D20222103F07CFFF30716D4E1
:10A68000E36B83B999F81E208DF8042099F82020F7
:10A690008DF8063001A8930901228DF805308DF858
:10A6A000072028F01FF8404603B0BDE8F08FBBF14B
:10A6B000000FE5D001350C238BF807508BF80630DE
:10A6C000584699F81D20222103F054FFD8E70135A0
:10A6D000EDB2BAF1000F04D00B238AF807508AF8C4
:10A6E000063017F0100F50460CBF1221022199F8C6
:10A6F0001D2003F03FFFC3E730F02EFDABE7A0467F
:10A70000D1E7C846CFE700BF2842002098F80308E9
:10A7100000380240BC200020FD90000800B97047BE
:10A72000F0B595B0064630F01BFFB34DC368026824
:10A730002A600446002B00F03981304604F0B2F85C
:10A74000AE4BC3F8E40118B1292200238271C37112
:10A75000227A2A2103F00EFF286804F075FA30F0FF
:10A76000FBFC2A68138823F001031B041B0C1380D5
:10A770001046FFF723FDA24B984200F219810026F4
:10A78000DFF8B4E29F4F13889F4906F1010CB0FB3C
:10A79000FCF04FF0030CB0FBF1F081B2B1FBFCF127
:10A7A000AEF800104900398098498A429BB200F007
:10A7B000098101F580618A4200F00481B2F1804F85
:10A7C00000F00081A1F580318A4200F0FB8001F5A4
:10A7D00080618A4200F0F68001F580618A4200F0D3
:10A7E000F1808B498A4200F0028101F580618A4242
:10A7F00000F0FD8023F44071844B89B29A421180AD
:10A80000D062168500F0F080824B9A4200F0EC8016
:10A8100001219182E27960200023ADF800009007C9
:10A82000ADF80230ADF804300293ADF80C30ADF85D
:10A830000E30ADF81030ADF8123040F1C78012F094
:10A84000010F0CBF1A4608220423ADF80E20ADF804
:10A85000043000232868617902936A4603F054FCAF
:10A8600060792B680C2816D8DFE810F0FA00150084
:10A87000150015000D00150015001500F10015005C
:10A8800015001500E8001A8B22F400621204120C65
:10A8900042F400621A83B3F844205F4E5F4F6FEAC0
:10A8A00042426FEA524292B2A3F844201A8892B20E
:10A8B00042F080021A80E279198C92074CBF042280
:10A8C0000122824092B289B221EA02011984198CD4
:10A8D00089B20A431A841A88514992B242F001029D
:10A8E0001A80237D086B1C2202FB03634FF0290EA4
:10A8F0001A6900261043086383F818E05E76086B37
:10A9000002430A635A7B9F605E6105A801238DF8AC
:10A9100014208DF815308DF817308DF8166027F05B
:10A92000E1FEE3683F4F18463B6028F00BF83868BB
:10A93000036823F00103036028F004F805A827F05A
:10A94000C3FF2B68627938680A9634331344069340
:10A9500040F22A3309934FF4806322690B93324B00
:10A960000592079340224FF4805305A908920C9357
:10A970004FF480424FF440330D920F930E9627F020
:10A98000B5FF637928683968284C0C2B9CBF284A8E
:10A9900032F81330828988BF334692B213438381E1
:10A9A0000B68012243F010030B60227015B0F0BD5C
:10A9B00000F1B77303F558531E49B3FBF1F3013BA4
:10A9C0009EB2DDE623F070039BB20AE712F0010F9E
:10A9D0000CBF002202224FF48073ADF80210ADF8D4
:10A9E0000C20ADF8103034E70023138610E71380F5
:10A9F000D06216850CE700BF70A300205824002009
:10AA0000FF6BDC0266A3002000350C000000014053
:10AA10000010004000040140BC2000208581000897
:10AA2000003802406CA300202881002068A3002089
:10AA30002C1E0408006CDC0264A300209A8B22F414
:10AA400000621204120C42F400629A8323E79A8B8C
:10AA500022F008021204120C42F008029A831AE74C
:10AA60001A8B22F008021204120C42F008021A8318
:10AA700011E7094B10B507281B68C8BF14381844E4
:10AA80000C46007D03F00EFF20B12146BDE81040CA
:10AA900004F088BE10BD00BF4842002038B50D4B01
:10AAA00007281B68CCBFA0F11404044623440546C4
:10AAB000187D03F0F7FE58B128220134C471827169
:10AAC000012104F0ABFD28460021BDE83840D0E765
:10AAD00038BD00BF484200200348D0F8AC3113B164
:10AAE00000F5D27018477047BC2000200348D0F80A
:10AAF000903113B100F5C47018477047BC20002096
:10AB00000348D0F8743113B100F5B6701847704798
:10AB1000BC2000200348D0F8583113B100F5A870CC
:10AB200018477047BC2000200348D0F83C3113B1CF
:10AB300000F59A7018477047BC2000200348D0F8F1
:10AB4000203113B100F58C7018477047BC200020ED
:10AB50000348D0F804310BB1FC301847704700BFF0
:10AB6000BC2000200348D0F8E8300BB1E030184793
:10AB7000704700BFBC2000200348D0F8CC300BB198
:10AB8000C4301847704700BFBC2000200348D0F8ED
:10AB9000B0300BB1A8301847704700BFBC20002070
:10ABA0000348D0F894300BB18C301847704700BF81
:10ABB000BC2000200248836F0BB1703018477047EB
:10ABC000BC2000200248C36D0BB1543018477047B9
:10ABD000BC2000200248036C0BB138301847704786
:10ABE000BC2000200248436A0BB11C301847704754
:10ABF000BC2000200248836803B11847704700BF9B
:10AC0000BC200020F8B584894FF6FF764FF47A74A3
:10AC100033B319B30F78013101E0B44218D005897C
:10AC2000013CAD07A4B2F8D5BCB284814FF47A746C
:10AC300002E0BCB2B4420BD00589ED0704F1FF3746
:10AC4000F7D58589ADB20AB115700132013BDFE756
:10AC500012F055FE003018BF0120F8BDFF27DEE7D7
:10AC60000120F8BD2DE9F84F7A4B7B4A19887B48C3
:10AC700001231370FEF796FA794B1B6813B11A681B
:10AC80009B88538380217548FEF7B8FA00217348EA
:10AC9000FEF7B4FA724B1B68064613B11A689B881C
:10ACA0001383704C6D48704D0421FEF77BFA2378B6
:10ACB0002F68B34262D0FEF7ABFB6C4E6C4BB6F81C
:10ACC000F221B3F80080DFF8B8C100210D464FF043
:10ACD000050B4FF0060A4FF00709B4181CF80200E4
:10ACE0002379834202F1010705F1050312D006EB37
:10ACF000030E73192071140A83F8F4B183F8F6A1D6
:10AD000083F8F72183F8F89183F8F541013106358E
:10AD10008EF8F401BAB2904501F1010109D9632915
:10AD2000DBDDA6F8F2214DB94B4A00231370BDE8D4
:10AD3000F88F0023A6F8F231002DF5D0454B474897
:10AD40001988FEF72FFA464B1B6813B11A689B88C7
:10AD500053832B46002247494048FFF753FF404B9F
:10AD60001B6813B11A689B88138304213B48FEF7C4
:10AD700019FA394A00231370BDE8F88F3E4B3B4E59
:10AD80001B78002B9AD1D6F8E831FB1AB3F57A7FFD
:10AD900094D9304B31481988FEF704FA304B1B68C0
:10ADA00013B11A689B885383A0212C48FEF726FA1A
:10ADB00000212A48FEF722FA294B1B68814613B16D
:10ADC0001A689B881383DFF8BC8024480421FEF7AF
:10ADD000E9F998F80030182B18D019F0040F11D1A8
:10ADE00009F00503012B1FD04BB923785B0606D56C
:10ADF000D6F8EC212B68DAB19B1A642B1BD8C6F865
:10AE0000E8715BE70023C6F8EC31F8E723781B4ACA
:10AE100003F04003002B09F007010CBF0D201020A8
:10AE200013805180D080D8E723785A06E0D5E6E732
:10AE3000C6F8EC31E3E7FEF7EBFA98F80030182B90
:10AE4000DDD1B6F8F0310D4A01339BB2A6F8F031EE
:10AE50009380D4E74002002081540020003C004051
:10AE6000A0960020F6000020E4A70020582400202F
:10AE7000F40000204C260020B4960020AC96002060
:10AE800074520020A9960020037A022B01D00020E2
:10AE9000704770B5036982B013B11A689B885383F9
:10AEA0000446BB21C068FEF7A9F906236A460021C3
:10AEB000E068FFF7A7FE236913B11A689B88138324
:10AEC0009DF804009DF800609DF801109DF8025067
:10AED0009DF803209DF8053041EA062143EA00234E
:10AEE00042EA05220120E1822283638302B070BD21
:10AEF000037C022B01D00020704770B5836982B0BB
:10AF000013B11A689B8853830446C3214069FEF736
:10AF100075F906236A4600216069FFF773FEA3698D
:10AF200013B11A689B8813839DF804009DF8006094
:10AF30009DF801109DF802509DF803209DF8053002
:10AF400041EA062143EA002342EA05220120218743
:10AF50006287A38702B070BD2DE9F04F044690F8D8
:10AF6000550085B0002840F07F81474D95F84C345E
:10AF7000002B00F08F806069444B984200F0728192
:10AF8000434A90420CBF30223822038823F040030A
:10AF90001B041B0C038003889BB223F038031A4365
:10AFA000028003889BB243F040030380A36994F8B6
:10AFB0004E5013B11A689B88538340F2E93304E082
:10AFC000013B9BB2002B00F0868202899207F7D5E5
:10AFD0001A23838140F2E93304E0013B9BB2002B4A
:10AFE00000F079820289D707F7D5838940F2E933E7
:10AFF00004E0013B9BB2002B00F06A8202899607B5
:10B00000F7D5ADB2858140F2E93304E0013B9BB254
:10B01000002B00F05D820289D107F7D58389A369EF
:10B0200013B11A689B88138303F094FF054603F05D
:10B0300091FF8542FBD06069144B984200F0468234
:10B04000134A904214BF08220022038823F04003D1
:10B050001B041B0C038003889BB223F038031A43A4
:10B06000028003889BB243F040030380237C022BC1
:10B0700000F0B581B4F93A305BB2013300F03881A9
:10B0800005B0BDE8F08F00BF582400200038004014
:10B09000003C00404FF480716069FEF783F8A369BB
:10B0A00013B11A689B8853836B216069FEF7A6F879
:10B0B00080216069FEF7A2F8A36913B11A689B8822
:10B0C0001383962003F0ECFFA36913B11A689B88E1
:10B0D000538368216069FEF791F803216069FEF7E8
:10B0E0008DF8A36913B11A689B881383962003F027
:10B0F000D7FFA36913B11A689B8853836B216069DA
:10B10000FEF77CF803216069FEF778F8A36913B1B4
:10B110001A689B8813830F2003F068FFA36913B19B
:10B120001A689B8853836A216069FEF767F81021CB
:10B130006069FEF763F8A36913B11A689B881383EB
:10B140000F2003F053FFA36913B11A689B88538340
:10B150006C216069FEF752F800216069FEF74EF835
:10B16000A36913B11A689B8813830F2003F03EFF75
:10B17000A36994F8506013B11A689B88538319210E
:10B180006069FEF73BF831466069FEF737F8A3695E
:10B1900013B11A689B8813830F2003F027FFA3695C
:10B1A00013B11A689B8853831B216069FEF726F848
:10B1B00018216069FEF722F8A36913B11A689B8809
:10B1C00013830F2003F012FFA36913B11A689B8841
:10B1D00053831C216069FEF711F810216069FEF7A6
:10B1E0000DF8A36913B11A689B8813830F2003F02D
:10B1F000FDFEA36913B11A689B88538337216069E8
:10B20000FDF7FCFF10216069FDF7F8FFA36913B19A
:10B210001A689B8813830F2003F0E8FEA36913B11B
:10B220001A689B88538338216069FDF7E7FF012185
:10B230006069FDF7E3FFA36913B11A689B88138364
:10B240000F2003F0D3FE04216069FDF7ABFF01205E
:10B2500003F0CCFE012385F84C346069A04B984282
:10B260007FF48EAE302290E603F01CFB05460028EA
:10B2700000F025810068AE88026932407FF475AE27
:10B2800000F13F4303F57E039B0A9649EA71CA5CCD
:10B2900002F01F07520901232021032A03FA07F3B2
:10B2A000A97100F00781042A00F0FF80022A03D16F
:10B2B0008D4A516C0B435364002302A903930296F9
:10B2C00027F09AFC2146894B41F80C3F28462FF085
:10B2D00065FFAB88B3FA83F3C3F11F03012212FAAF
:10B2E00003F33FF442AE82490A6813430B603CE625
:10B2F00094F9383001337FF4C3AE0A237D4D7E4F7D
:10B300007E4C7F4E0193322030F004FBDFF8F49145
:10B310004FF4FA7A4FF0100803F01CFE4FF47A71E4
:10B3200086460120D9F80430C3F30803002B40F00F
:10B330009E80EFF31183002B40F099802B68D4F8A6
:10B3400008C000BF2A689342F8D1D7F800B001FBCB
:10B350000BF2A2EB0C02B2FBFBF201FB0323A3EB0B
:10B360000E03B3F57A7FDDD3BAF1010AD4D10720F9
:10B3700030F032F9DFF88C914FF47A7A4FF0100800
:10B3800003F0E8FD4FF47A7186460120D9F80430C5
:10B39000C3F30803002B4CD1EFF31183002B48D1EA
:10B3A0002B68D4F808C000BF2A689342F8D1D7F8B8
:10B3B00000B001FB0BF2A2EB0C02B2FBFBF201FBB3
:10B3C0000323A3EB0E03B3F57A7FDFD3BAF1010AAF
:10B3D000D6D1019B013B019395D1FFF735F8A369C5
:10B3E00013B11A689B885383C321FDF707FF062317
:10B3F00002AA00216069FFF705FCA36913B11A686E
:10B400009B8813839DF80A609DF80B309DF80850C7
:10B410009DF809109DF80C009DF80D2043EA0623C5
:10B420001BB241EA052142EA002263872187A287F5
:10B4300022E6EFF3118C88F31288D4F808B0236861
:10B44000DB0344BF3060D4F808B02B6832685FFA81
:10B450008CFC8CF31188D7F800C01A4401FB0CF364
:10B46000A3EB0B03B3FBFCF301FB0233A9E7EFF300
:10B47000118C88F31288D4F808B02368DA0344BF2B
:10B480003060D4F808B02B6832685FFA8CFC8CF31B
:10B490001188D7F800C01A4401FB0CF3A3EB0B038F
:10B4A000B3FBFCF301FB023359E70F4A116B0B436B
:10B4B000136301E70C4A116C0B431364FCE621464D
:10B4C0000A4B41F80C3F2FF069FE4EE50022BCE527
:10B4D00012F015FAA3E512F012FA606986E500BFD2
:10B4E00000380040742B0408003802400180000836
:10B4F000003C0140E4A70020E8A7002010E000E0A5
:10B50000E0A7002000ED00E0F8B5654C0601A719A2
:10B510000546387A2FF020FE3B7A03F01F015B09C5
:10B520000122032B02FA01F26DD0042B66D0022B0C
:10B530005CD0A3190135187903F0B4F9EDB20746D0
:10B5400010B11223C5718371A319587903F0AAF9B8
:10B5500010B11323C5718371A319987903F0A2F96F
:10B5600010B11423C5718371A5190A21EA793846EF
:10B5700003F000F8687903F095F9EA790A2102F0FE
:10B58000F9FFA87903F08EF9EA790A2102F0F2FFB7
:10B59000A359444A934247D0434A934250D0434A26
:10B5A000934259D0424A934262D0424A93426BD06E
:10B5B000414A93422CD03444227BE2B9012002223A
:10B5C000198801F4415141F445710A4302431A803C
:10B5D0009A8B22F400621204120C07219A831982BA
:10B5E0001A8892B242F040021A80F8BD334B596A71
:10B5F0000A435A629DE700200246E1E72F4B196992
:10B600000A431A6195E72D4B196A0A431A6290E7BB
:10B6100002F564424FF40010536A43F4001353627E
:10B6200027F098F8A359C6E702F584324FF480500A
:10B63000536A43F48053536227F08CF8A359BAE756
:10B6400002F500324FF48040136A43F480431362E2
:10B6500027F088F8A359AEE702F5FE324FF4004018
:10B66000136A43F40043136227F07CF8A359A2E75E
:10B6700002F582324FF40050536A43F40053536290
:10B6800027F068F8A35996E702F568424FF4801056
:10B69000536A43F48013536227F05CF8A3598AE796
:10B6A000D49600200030014000380040003C0040AB
:10B6B0000034014000500140005401400038024075
:10B6C0001549164B16484A6810B4CC681549B2FBA8
:10B6D000F4F203FB02F30360D1F88820124B134C01
:10B6E00042F47002C1F888201A68002042F001027A
:10B6F0001A6098601A6822F0847222F480321A600C
:10B700005C601A684FF0006422F480221A60D860EE
:10B710008C605DF8044B70470000002040420F0031
:10B72000E8A8002000ED00E00038024010300024BE
:10B73000044B4FF4F07002210A225860D9609A60DD
:10B74000FFF7BEBF000000202DE9F04F9BB0B0F91D
:10B7500008500D81EDB2442D00AF0C46904600F02C
:10B76000D982064643D9812D00F0128200F29A80D8
:10B77000542D00F0CF8040F2F7816E2D00F09882BA
:10B78000802D40F02581C54B93F800A00AF1020AF4
:10B790001AF0FF0A00F09A80C14BDFF84083C14ED7
:10B7A000DFF83CB39A4403F101090A2516E0322D73
:10B7B00000F0DF82A5F13C00C0B2132840F2DF8226
:10B7C00000232268511C216015702268D14502F1C6
:10B7D00001012160137079D019F8015B0A2DE6D1BF
:10B7E000BBF80030FF2BA8BFFF23DBB2E9E7052D34
:10B7F00000F07E8221D8022D00F0848040F2A181E9
:10B80000032D00F04C82042D40F0E2802A46A64928
:10B81000204612F0B5FCA54B2046197812F0F5FC35
:10B8200022680221531C0125236028462B466C37D1
:10B8300011706381BD46BDE8F08F242D60D040F2C9
:10B840000F81282D00F0ED81382D40F0C1800A686D
:10B85000974B0125511C2160157022680521501954
:10B860002060117022680A2150192060117022682E
:10B870000021501920601170226819785019206039
:10B8800011702268597850192060117022689978D7
:10B89000531923602B46117028466C376381BD46CF
:10B8A000BDE8F08FA02D19D040F22081B82D00F016
:10B8B000F481FE2D40F08C807E4D05F1080635F8B0
:10B8C000021B204612F0A1FCB542F8D101252B46FF
:10B8D00028466C376381BD46BDE8F08F764B08463D
:10B8E000196812F07BFC754B2046196812F076FC43
:10B8F000734B19682046012512F070FC2B46E7E7D0
:10B90000704BF6E7042270492046012512F038FCFE
:10B910002B46C1E70B686D4ADFF8C881581C11211E
:10B920002060197023681278591C21601A702368EE
:10B9300098F85520591C21601A70236898F85420F3
:10B94000591C21601A70B8F85010204612F05DFCA6
:10B9500023680022591C21601A7023682822591C70
:10B9600021601A70B8F85210204612F04EFCA8F16F
:10B97000020508F14E0635F8021F204612F045FC7C
:10B98000B542F8D12268524B0D21501C20605D1841
:10B990001170226813F8011F501C9D422060117025
:10B9A000F7D123680222591C21601A70B8F856108A
:10B9B000204612F02AFCB8F85810204612F025FC58
:10B9C0000125B8F85A10204612F01FFC2B4663E7F9
:10B9D000214628460EF0CEFC034600287FF476AFC1
:10B9E000742D00F0C780772D0DD1326871689142B7
:10B9F0001EBF531C33601178364A08BF19462046D3
:10BA000031F0C2FB62E7F52D01F07283762D00F074
:10BA10008981472D00F02782392D326800F0E882B5
:10BA200000F20682212D01F04383292D40F01C8372
:10BA3000531C336013780A2B01F02F84502B40F0F5
:10BA40002285304612F08CFBDFF89C80A8F80000BD
:10BA5000304612F085FB0125A8F802002B461BE7B3
:10BA6000202DB5D10B681C4D591C6A7821601A70C5
:10BA700023682A78591C21601A702368AA78591CF7
:10BA800021601A702989204612F0BFFB23686A7969
:10BA9000591C21601A702268A979C3E665650020E7
:10BAA000C0F803086C2F00200EA80020A828002052
:10BAB000CFA10020AC960020107AFF1F147AFF1F40
:10BAC000187AFF1F3CA300205C2D0408B8960020C4
:10BAD00001800020A9CD0308609E0020676666668D
:10BAE000942F0020A47F0020542F0020822D7FF46B
:10BAF0006FAF0B68BA4ABB4D1178BB4A581C206027
:10BB000019701189204612F080FBB84B22681B88FF
:10BB1000FF2B02F10101A8BFFF2321601370A96868
:10BB200081F3100189B2204612F06FFB296801F3FE
:10BB30000F0189B2204612F068FBAD4B22681978DC
:10BB400070E6012D7FF444AF0B680022591C216080
:10BB50001A7023685A1C22601D7022682521531C0C
:10BB600023602B46117097E6522D7FF431AF226887
:10BB7000002157E63268716891421EBF531C336042
:10BB800011789C4A08BF1946204631F0FDFA9DE61F
:10BB9000994B1E78033616F0FF063FF497AE974B8D
:10BBA000DFF884821E4403F1010A4FF00A0920E005
:10BBB000B9F1500F00F0DB80B9F1320F00F0F480E2
:10BBC000A9F13C00C0B2132840F2F18000252946BB
:10BBD00023685A1C2260204683F8009012F015FB5F
:10BBE0002946204612F011FBB2453FF46FAE1AF819
:10BBF000019BB9F10A0FDBD1814B9D68196805EBF8
:10BC000085054FF6FF736D009D42A8BF1D46994202
:10BC1000A8BF194625EAE57521EAE171ADB289B2FE
:10BC2000D6E70B68DFF80492764E591C0222216099
:10BC30001A7023684FF006085A1C226083F80080AF
:10BC400023680A22591C21601A70236801255A1999
:10BC500022601D70B9F80010204612F0D6FAB9F82B
:10BC60000210204612F0D1FA23685A19226083F894
:10BC7000008023685022591921601A70236800221D
:10BC8000591921601A703188204612F0BEFA718865
:10BC9000204612F0BAFA2B46FEE55B4B29E60B680C
:10BCA0005A1C0A601D700B685A1C0A601D705EE702
:10BCB0004E4B0A681B884B4DFF2BA8BFFF23511C1E
:10BCC00021601370A96881F3100189B2204612F037
:10BCD0009CFA4E4B2046198812F097FA296801F316
:10BCE0000F0189B22046012512F08FFA2B46D3E5C9
:10BCF0000B224749204612F043FA082245492046C4
:10BD000012F03EFA012507224349204612F038FA84
:10BD10002B46C1E5002A3FF4D9AD404B1360012505
:10BD20002B46B9E53268511C31601278002A01F0C7
:10BD3000BB82102A01F03A83394D1E46194623680A
:10BD4000581C20601A70204612F048FA31462046EE
:10BD500012F044FAE968204612F040FA2046002129
:10BD600012F053FA0021204612F04FFAFFE62D4B55
:10BD700043E73388FF2BA8BFFF23DBB221E51FF089
:10BD8000D3FC00283FF41CAD03780A2B25D8B0F96A
:10BD9000023088FB0312DB17C3EBA2039BB2FF2B1D
:10BDA000A8BFFF23DBB20CE598E8220027E71FF0CD
:10BDB000BBFC00283FF40AAF03780A2B3FF606AF1E
:10BDC000B0F90430B0F9061003EB830383F3500598
:10BDD00021EAE171ADB289B2FAE60023E2E700BFE1
:10BDE00092660020489E0020609E00207C66002015
:10BDF00010800020B5CD030865650020D0F8030849
:10BE0000202F0020542F002098470020588E00201B
:10BE1000642D0408702D04087C2D0408B9A00108C5
:10BE2000A8280020582F0020642F0020287F002001
:10BE3000552D00F0ED80572D40F01681531C3360D6
:10BE400012F8370B07F127010133336013F8015C57
:10BE500001F8015F9342F7D107F128010125FDF7B1
:10BE60003FFF2B4618E5726835687B623046551BEC
:10BE700012F05FF9052D38627B6A01F2018280269B
:10BE8000B346012594E80600521A103AB242B8BFF0
:10BE90001FFA82FB714A396A92683A61521A9345D5
:10BEA000396A7B622046FA6088BF1FFA82FB12F073
:10BEB00095F97B6A002B01F0C281002D41F09E8133
:10BEC0002368C7F800D05D71C0B00533C7F804D04F
:10BED000FB61BBF1000F01F06E833B6A3A6993424C
:10BEE00081F065833E6A7D62AA46A846BC608025D3
:10BEF000FB68A3EB0808594BB8F5807F9B6828BF07
:10BF00004FF4807808EB06029A4288BFA3EB06083C
:10BF100012F0ECFF7C6842462146304613F06CF884
:10BF2000F969B86104EB000C0B787B6164452ED293
:10BF3000DFF830910CF1FF3C04F1FF3E1EF8013FA9
:10BF400009EB830219F823405688ECB100234FF423
:10BF5000004204F1FF3816424FEA520202D008783C
:10BF6000284308706D0806D10AF1010A4D701FFAC6
:10BF70008AFA01318025D34503D8F44532D8984553
:10BF800030DC01339C42E6D1E645D7D1F9617B6ACA
:10BF9000BA6913449BB2D3457B6206D97B6A3A6A7D
:10BFA0009846D6183B699E42A2D3BC68802D1CBF20
:10BFB0000AF101031FFA83FA0AF1020189B220464D
:10BFC00012F023F92368796A01255A192260204664
:10BFD0001D7012F01AF92368534423602B46D7F8DA
:10BFE00000D059E4FB69BC681A463B7D1370DDE75D
:10BFF000531C336013780A2B01F05C81304612F039
:10C00000BAF8304612F0B7F8304612F0B4F85DE4F2
:10C01000531C336092F80080B8F1FF0F01F0CB8120
:10C02000B8F1FE0F01F08081304612F099F83368C4
:10C030007268D21A002A07DD5A1C32601B781BB9BD
:10C04000B8F10C0F41F2F581B8F1270F00F2278506
:10C05000034B012523F818002B461DE44402002061
:10C06000A47F0020E0F8030871680B3D8B1AEF2DC8
:10C0700000F2158501A050F825F000BFAFCD0008F3
:10C080009FCA00089FCA00089FCA00089FCA0008EC
:10C090009FCA00089FCA00089FCA00089FCA0008DC
:10C0A0009FCA00089FCA00089FCA00089FCA0008CC
:10C0B0009FCA00089FCA00089FCA00089FCA0008BC
:10C0C0009FCA00089FCA00089FCA00089FCA0008AC
:10C0D0009FCA00089FCA00089FCA000855CD0008E3
:10C0E0009FCA000833CD00089FCA000879CC000819
:10C0F0009FCA00089FCA00089FCA000851CC0008C8
:10C100009FCA0008F7CB00089FCA0008C5CB0008EB
:10C110009FCA0008B5CC00089FCA0008A3CC00083D
:10C120009FCA0008DBCC00089FCA000851CA00085B
:10C130009FCA00089FCA00089FCA00089FCA00083B
:10C14000CDB800089FCA00080DCB00089FCA0008A0
:10C150009FCA0008B5CA00089FCA00083DC400086D
:10C160009FCA00089FCA00089FCA00089FCA00080B
:10C17000A9CA00089FCA00089FCA00089FCA0008F1
:10C1800085CB00089FCA000839CB00089FCA000869
:10C190009FCA000811CA00089FCA00089FCA000869
:10C1A0009FCA00089FCA00089FCA00089FCA0008CB
:10C1B0009FCA0008A3C900089FCA0008E7C8000872
:10C1C0009FCA000859C800089FCA0008C1C70008D4
:10C1D0009FCA000899C7000885C90008CBC8000895
:10C1E0009FCA00089FCA00089FCA00089FCA00088B
:10C1F0009FCA00089FCA00089FCA00089FCA00087B
:10C200009FCA00089FCA00089FCA00089FCA00086A
:10C210009FCA00089FCA00089FCA00089FCA00085A
:10C220009FCA00089FCA00089FCA00089FCA00084A
:10C230009FCA00089FCA00089FCA00089FCA00083A
:10C240009FCA00089FCA00089FCA00089FCA00082A
:10C250009FCA00089FCA00089FCA00089FCA00081A
:10C260009FCA00089FCA00089FCA00089FCA00080A
:10C270009FCA00089FCA00089FCA00089FCA0008FA
:10C280009FCA00089FCA00089FCA00089FCA0008EA
:10C290009FCA00089FCA00089FCA00089FCA0008DA
:10C2A0009FCA00089FCA00089FCA00089FCA0008CA
:10C2B0009FCA00089FCA00089FCA00089FCA0008BA
:10C2C0009FCA00089FCA00089FCA00089FCA0008AA
:10C2D0009FCA00089FCA00089FCA00089FCA00089A
:10C2E0009FCA00089FCA00089FCA00089FCA00088A
:10C2F0009FCA00089FCA00089FCA00089FCA00087A
:10C300009FCA00089FCA00089FCA00089FCA000869
:10C310009FCA00089FCA00089FCA00089FCA000859
:10C320009FCA00089FCA00089FCA00085BC900088E
:10C330009FCA00082DC7000803C700089FCA00084D
:10C340009FCA00089FCA00089FCA00089FCA000829
:10C350009FCA00089FCA00089FCA00089FCA000819
:10C360009FCA00089FCA00089FCA00089FCA000809
:10C37000A5C6000853C600081BC600089FCA0008CF
:10C3800079C500085FC5000843C500089FCA0008BA
:10C3900029C50008BFC4000897C400088DC4000860
:10C3A00051D000089FCA000821D000089FCA000889
:10C3B0009FCA0008F7CF0008C9CF0008B5CF000812
:10C3C0008DCF00086DCF000843CF000817CF0008BD
:10C3D0009FCA00089FCA00089FCA00089FCA000899
:10C3E0009FCA00089FCA00089FCA00089FCA000889
:10C3F0009FCA00089FCA00089FCA00089FCA000879
:10C400009FCA00089FCA00089FCA0008F7CE00080C
:10C410009FCA00089FCA00089DCE00089FCA000856
:10C420009FCA00089FCA000839CE00089FCA0008AA
:10C430009FCA00089FCA0008E5CD0008531C33605E
:10C44000C14B1278DFF844831A700023C8F800301B
:10C45000304611F06EFE3368D8F80020BB49BC4D61
:10C4600010435A1CC8F8000032601B780B7230462B
:10C4700011F076FE2860304611F072FE686030469A
:10C4800011F06EFEA860304611F06AFE304611F0E1
:10C4900067FEFFF71BBA531C33601078060601F1E4
:10C4A0002D80AC4B1B78DD073FF510AA032828BF71
:10C4B0000020012501F076FB2B46FFF7EDB9531C58
:10C4C0003360304692F800A011F033FE81463046CA
:10C4D00011F02FFE0546304611F02BFE8046304607
:10C4E00011F03EFE304611F03BFE304611F043FEA7
:10C4F000BAF1000F00F0EB87BAF1100F7FF4E6A954
:10C50000954BC3F804909D60B8F1000F01D0C3F8BB
:10C510000C809249924B0222081F01251A701CF0D0
:10C52000E1FB2B46FFF7B8B98A4B1B78D8073FF5DC
:10C53000CDA9012501F0DCFD01F002FC2B46FFF73F
:10C54000ABB9844B1B78DA073FF5C0A9854A13784D
:10C55000012543F0040313702B46FFF79DB97D4B73
:10C560001B78D9073FF5B2A97F4B4FF4C87201255C
:10C570001A802B46FFF790B9092B40F39082DFF821
:10C5800010821346511CD8F80050316013F8021B7A
:10C59000297033605378AB70D31C33609378642B6D
:10C5A00002F10401A8BF64236B713160D378642B5E
:10C5B00002F10501A8BF6423AB7131601379EB71FF
:10C5C000931D33605379642B02F10701A8BF6423E4
:10C5D0002B7231609379EB7002F108033360D379E9
:10C5E0002B71304611F0BCFD726833686881D11A36
:10C5F00000290CDD591CD8F800003160521A002ABD
:10C600001978417203DD9A1C32605B784370012512
:10C6100028F02CFA2B46FFF73FB9544B1868D31C6F
:10C62000014621329D1E356013F8035C0D705D1EBE
:10C63000356013F8025C4D70336013F8015C8D7047
:10C6400003339A4201F10301ECD127F09FFAFFF77F
:10C650003DB9531C336013784249002B00F0218709
:10C660000B7843F00203901C0B70414D30605378FF
:10C670002B75304611F05DFD2860304611F059FDF4
:10C680006860304611F06CFD2881304611F068FD7D
:10C69000384AE8811378012543F0020313702B46D2
:10C6A000FFF7FAB8C3F34705122D00F2F881C5B1C0
:10C6B00007F1680307F1260A03EB4508D146A8F104
:10C6C0004208304611F04CFD29F8020FC845F8D158
:10C6D000294B3AF8022F23F8022FD145F9D1112D19
:10C6E00009D8264A6B00023B13440021223223F86A
:10C6F000021F9A42FBD1224A01231D461370FFF705
:10C70000CBB8531C1F48336001781378002940F0E0
:10C710009D86042202701C4A9B00138002F01AFCC2
:10C720000D4B012518622B46FFF7B6B8DFF8648081
:10C7300000233046C8F8003011F0FBFC0125C8F892
:10C7400000002B46FFF7A8B8687F0020FC9C002063
:10C750005842002060900020A8280020B028002027
:10C760000A690020C69E002042B30020C89E002017
:10C77000EC580020086900204A4F00204C4F002050
:10C78000704F00209C490020588E00203CA30020C0
:10C79000CC9E0020984700201346511C3160CC49A4
:10C7A00013F8020BC8703360CA4953784B71D31C1D
:10C7B0003360C94B9278DA7001252B46FFF76CB8CD
:10C7C000304611F0CDFC304611F0CAFC304611F075
:10C7D000C7FC304611F0CFFC3368C04D1946581CD9
:10C7E0002A68306011F8020B82F82C003160597809
:10C7F00082F83610D91C31609B7882F83730304689
:10C8000011F0B9FC304611F0B6FC304611F0B3FC23
:10C810003046D5F8008011F0A3FCA8F83A00304665
:10C82000D5F8008011F09CFC33687268A8F83800D5
:10C83000D11A01290ADD591C2A6831601B7882F857
:10C840002E30304611F097FC33687268D31A032BF0
:10C8500000F37C862868F8E6531C33609F4DDFF8B0
:10C86000A082137888F805303046D5F8009011F092
:10C8700077FCA9F820003046D5F8009011F070FC44
:10C8800072683368A9F81E00D11A072900F3ED85F4
:10C89000D11A032900F39486D21A002A05DD591C07
:10C8A0002A6831601B7882F8263001F0A1F92FF058
:10C8B00023FC8B4B1B68002B00F0F88528680125B2
:10C8C00026F056FF2B46FEF7E7BF531C3360137864
:10C8D000002B00F049864FF4004001250EF0F2FDD8
:10C8E0002B46FEF7D9BF1346511C3160DFF810828A
:10C8F00013F8021B88F8021033607A4953780B70E2
:10C90000D31C3360784D93782B71131D3360D3782B
:10C91000092BA8BF09233046AB7011F021FC336806
:10C9200072682880D11A012905DD304611F018FC03
:10C9300033687268E8819A4240F08D8501F058F9B9
:10C94000336872689A423EF4C1AF5A1C32601B7859
:10C95000EB7001252B46FEF79FBF1346511C31603B
:10C9600013F8025B3360D31C507833609178002D4C
:10C9700000F0A785012D7EF4A9AF2CF03BFA2B46E1
:10C98000FEF78ABF594B1B7813F0010140F08780F6
:10C99000531C3360107801252CF066F92B46FEF706
:10C9A0007BBF534B1B68002B3EF490AF1CF092FAF8
:10C9B000FF283EF48BAF304611F0D2FB3F2840F207
:10C9C0000D86DFF84081002588F8005033687268D2
:10C9D000A8F80400D21A012A7EF778AF1A46591C2B
:10C9E000316012F8021B88F8021007F1680032600B
:10C9F00000225D7800F8402D1CF03EFA97F82830B0
:10CA0000AB423EF463AF28461CF05AFAFEF75EBF15
:10CA1000384B1B78012B3EF659AF1046531C336040
:10CA2000DFF8E48010F8023B88F802303060D31C55
:10CA300050783360CB1A012B917840F3AC853046A7
:10CA400011F08EFB0125A8F800002B46FEF724BF4D
:10CA50000721B3FBF1F1C1EBC1055B1B1FD1C9B2CB
:10CA600001F1FF395FFA89F900293EF42FAFDFF8B1
:10CA700088A009F101091D46531C336092F900207A
:10CA80001D4B4FF0000893F90210914203F1080387
:10CA900000F0678408F10108B8F1050FF3D14FF0F9
:10CAA000FF352B46FEF7F8BE012512F081FA2B4622
:10CAB000FEF7F2BE114B02F108010132326012F8AA
:10CAC000010C03F8010F9142F7D1FEF7FFBE00BF42
:10CAD000387F00208CA00020487F0020C89E0020C6
:10CAE000607F00202C7F00204455002060900020B3
:10CAF0006490002026A30020289D0020FB9C00209D
:10CB0000C8B0002068900020AC8E00201346501C56
:10CB10003060BB4813F8025B857033605578457010
:10CB20008B423EF4D3AED31C3360B64B92781A7569
:10CB300001252B46FEF7B0BE531C336092F80080EF
:10CB4000B8F1110FABD8931C3360AF4D537805F893
:10CB50001830304611F004FB40F6CA039842A8BFD3
:10CB6000184640F2EE23984205EB4801B8BF18463C
:10CB70000125A0F2EE222B46192092FBF0F24A701A
:10CB8000FEF78ABE1346511CA04D316013F8021BFC
:10CB90002971336053786B71304611F0E1FA3368D4
:10CBA00028805A1C32601B78AB71304611F0D8FADD
:10CBB000336868805A1C32601B78EB7101252B4664
:10CBC000FEF76ABE924D05F14008304611F0C8FAF2
:10CBD0003368A5F88000591C1A46316012F8021B10
:10CBE00085F8821032605B7885F883300435A8457B
:10CBF000EBD1FEF76BBE531C864D336013782B725E
:10CC0000304611F0ADFAA883304611F0A9FA288316
:10CC1000304611F0A5FA32686883531C33601278ED
:10CC2000EA747268D31A032B00F3F9843368D11ABB
:10CC3000052900F3E384D21A002A7EF747AE5A1C76
:10CC400032601B7885F8213001252B46FEF724BE83
:10CC5000531C3360704815780570C91A00297EF797
:10CC600035AE931C33605378003318BF0123012580
:10CC700043702B46FEF710BE304611F071FADFF814
:10CC8000B081C8F80000304611F06AFAC8F8040014
:10CC9000304611F065FA0125C8F808002B46FEF76A
:10CCA000FBBD531C33605B4B12785A7501252B4634
:10CCB000FEF7F2BD511C316015781F2D3FF6EFAE27
:10CCC000052B7FF4ECAE304611F033FA504B43F8AD
:10CCD00025001FF0B7FEFEF7F9BD531C3360137833
:10CCE0000E2B3FF6DCAE911C31605578032D3FF6DC
:10CCF000D6AE4A48062101FB03F1431802F1030EA8
:10CD00005D71C6F800E095784554111D3160D17809
:10CD10005970511D316011799970911D31605179AF
:10CD2000D970D11D316092791A7101252B46FEF719
:10CD3000B3BDDFF800810023C8F80030304611F0A1
:10CD4000F8F9D8F8003001250343C8F800302B4625
:10CD5000FEF7A2BD531C33601578132D3FF69FAE2E
:10CD6000931C336050787A6230F048FA00283FF420
:10CD700096AE7A6A2A4B017803F82510D11C3160EF
:10CD800003EB850391785970111D3160D17899704A
:10CD9000511D31601279DA70002027F0A7FD214B78
:10CDA00080F00100012518702B46FEF775BD1E4A64
:10CDB000102B4FF0000128BF1023116051609160CB
:10CDC000D1601174002B3EF481AD3168013A0B44FF
:10CDD0000131316011F8010C02F8010F9942F7D1CD
:10CDE000FEF774BD114B1B78DB073FF558AE0125EC
:10CDF00000F0F4FE00F0A4FF2B46FEF74DBD00BF8F
:10CE0000587F0020A8280020F851002060960020BC
:10CE100030800020FC9C0020687F0020A447002078
:10CE2000EC5000207D2200205C8E002060900020CD
:10CE3000584200203CA30020304611F091F933689D
:10CE400038851A46591C316012F8021B326087F887
:10CE50002A105A7887F82B20DA1C32609A7887F8E3
:10CE60002C201A1D3260DA7887F82D205A1D326086
:10CE70001B7987F82E3007F1280000233B8611F03C
:10CE8000CBF8CA4ACA4B1268801A4FF0010561F10B
:10CE90000001C3E906012B46FEF7FEBC531C3360BC
:10CEA00013780F2B3FF6FBAD911C3160C3EBC3032E
:10CEB000C0495078C854D01C30600B4491785970E8
:10CEC000111D3160D1789970511D31601179D9707F
:10CED000911D316051791971D11D3160917959716C
:10CEE00002F108013160D2799A71012526F0ACFB7C
:10CEF0002B46FEF7D1BC304611F032F9DFF8C08284
:10CF0000A8F80E00304611F02BF90125A8F80C0006
:10CF10002B46FEF7C1BC1146531C3360A64B11F8DB
:10CF2000020B1870316051785970D11C31609178C2
:10CF30009970111D3160D278DA7001252B46FEF709
:10CF4000ABBC304611F00CF9DFF89C82A8F8100059
:10CF5000304611F005F9A8F81200304611F000F93A
:10CF60000125A8F814002B46FEF796BC1346511C69
:10CF7000316013F8020B3360D31C51783360927820
:10CF800023F0C2FD00287EF4A1AC88E51346511CB5
:10CF900031608A4913F8020B08703360884953786E
:10CFA0008B70D31C3360874B92789A7001252B4687
:10CFB000FEF772BC844B854918684E22012531F07A
:10CFC00067FA2B46FEF768BC1146531C3360804B52
:10CFD00011F8020B1870316051785970D11C316012
:10CFE00092789A70304611F0BBF87A4B0125D880C0
:10CFF0002B46FEF751BC304611F0B2F8DFF8D48171
:10D00000A8F80000304611F0ABF8A8F8020030464E
:10D0100011F0A6F80125A8F804002B46FEF73CBC49
:10D02000DFF8C89199F80030002B3EF44FACDFF8E0
:10D03000C0810025304611F093F826F02FFF99F8B3
:10D040000030A8EC010A01359D42F3DBFEF73EBC3F
:10D050000D2B7FF424AD531C33601578072D3FF65C
:10D060001EADDFF8909130464FF00C0811F078F8C3
:10D0700008FB05F809EB0805A880304611F070F8A8
:10D08000E880304611F06CF8336828811A46591C44
:10D09000316012F8021BA97232605B78EB72304685
:10D0A00011F047F8012549F808002B46FEF7F4BBBC
:10D0B0001346511C3160484D13F8021B69703360F0
:10D0C00053782B70D31C33609378AB70304611F0DB
:10D0D00047F833682881591C1A46316012F8021B40
:10D0E000697132605B78AB7101252B46FEF7D4BBCA
:10D0F000336872689A4240F0EE802D4BFF225A70DE
:10D100004FF0000A354D2AF0BDFE5146202234482A
:10D1100085F800A032F04DFB87F828A097F828305A
:10D12000072B00F29181DFF8D0902D4E524697F8F0
:10D13000283003EB430309EBC3035B7CE3B197F8AF
:10D14000283003EB430309EBC30320215B699BB148
:10D1500097F8283003EB430309EBC303586946F8FB
:10D16000220002F05BFA2B7856F8230002F014FB41
:10D170002A780132D2B22A7097F828300133DBB214
:10D1800087F8283097F82830072BD0D92368591C06
:10D1900021601A70B8F1000F3EF498AB114BC8F83B
:10D1A000003001252B46FEF777BB00BFE4A7002027
:10D1B000A8280020AC460020186A0020C8B0002033
:10D1C000387F0020487F0020C89E0020A426040845
:10D1D000307F002048960020609E0020C14800203B
:10D1E000AC45002019340208445500206565002034
:10D1F00080440020EC4500202CB20020C54B3A6A48
:10D200009B68D4F800905A449342C0F0018111F019
:10D210006DFE5A464946386A11F0EEFE2368034413
:10D22000236086427EF752AB002100E02368013084
:10D230005A1CB04222601970F8D1FEF747BB002D8E
:10D24000DCD15946204610F0E0FF23685A1C2260CA
:10D250001D70B04B26689D683B6A0BEB030295423C
:10D2600080F08B813B6AED1A11F040FE2A46314670
:10D27000386A11F0C1FE236803442360FEF726BB21
:10D28000304610F06DFF326871687B6A91428346C8
:10D290005DD106461D46FEF7F5BD304610F060FF35
:10D2A000DFF8A482FEF7D2BB9B4B9C4D93E8420073
:10D2B000FEF745BD931C3360994B51781970D11C12
:10D2C000316091785970111D3160D2789A700125C2
:10D2D0002B46FEF7E1BA5A1C194632608F4811F806
:10D2E000022B427031605B788370042A03D9FF2AD5
:10D2F0007EF43DAC04E78B490978994205D8022AAF
:10D300007EF435ACFF2B7EF432AC236801255A192C
:10D3100022601D70B8F1000F3EF4D8AA824BC8F805
:10D3200000302B46FEF7B8BA931C33605578022DB7
:10D330003FF6B5AB304610F013FF7C4B03EB4503D3
:10D340004FF0FF35A3F856002B46FEF7A5BA511C47
:10D35000316012781D46131C064618BF0123FEF7E4
:10D3600091BD0AEBC80B30468BF8022010F0F8FE96
:10D3700033682AF838001A46591C316012F8021B2B
:10D380008BF8031032605A788BF80420DA1C326074
:10D390009A788BF806201A1D32600135DB788BF8FD
:10D3A0000530A9457FF468ABFEF790BA5B4D69681C
:10D3B000AE68FEF7C4BC931C33605D4B51781970A6
:10D3C000D31C3360DFF86481937888F85530131DDF
:10D3D0003360D37888F85430304610F0C1FEA8F896
:10D3E0005000304610F0BCFE304610F0B9FE96E812
:10D3F0000C009B1A012BA8F852007EF767AA304652
:10D4000010F0AEFE0125A8F85A002B46FEF744BAEC
:10D410003A6AA3EB020811F069FD42464946386AB0
:10D4200011F0EAFD236803442360002D3EF44EAA68
:10D43000F7E63E4B0030984418BF0120012588F8DC
:10D440005E002B46FEF728BA52469FE604297EF47A
:10D450003DAAFFF760B95A1C32601B78003318BF31
:10D46000012388F80730FFF769BA304610F078FEDC
:10D47000A8F80A00304610F073FEA8F80C003046F9
:10D48000D5F8009010F06CFEA9F822003046D5F8CF
:10D49000009010F065FE33687268A9F82400FFF769
:10D4A000F7B90B7803F0FD03FFF7DDB821482249F7
:10D4B000224A234B036001250B6013602B46FEF7C5
:10D4C000EBB9012526F046FB2B46FEF7E5B9124BDA
:10D4D0001020C3F800905D600DF0C4FF194A137866
:10D4E00043F001031370B8F1000F3EF4EFA90B4BAA
:10D4F0000125C3F80C802B46FEF7CEB900F07F0063
:10D50000032828BF002001252BF090FC2B46FEF7B6
:10D51000C3B900BF44020020E0680020A828002012
:10D52000CFA1002065650020C5A00108A47F0020D0
:10D53000B8960020EC9000204091002040950020FB
:10D540008FD50108C69E0020287F00203046D5F8E0
:10D55000008010F005FEA8F8320030462E6810F06A
:10D56000FFFDB086FFF776B93D4A1368012523F425
:10D57000004313602B46FEF78FB911F0B7FC5A46F3
:10D580003146386A11F038FD2368012503442360D1
:10D590002B46FEF781B9334B1A88012512FB00F2A6
:10D5A0002B4692FBF1F2A8F80020FEF775B97D62D8
:10D5B000AA46FEF701BDDA46C7F824B0FEF7FCBC68
:10D5C000304610F0CDFDA8F80E00304610F0C8FD32
:10D5D00033687268A8F81000FFF75EB9C50800F05C
:10D5E000070301350133EDB2DFF87C802846194688
:10D5F00088F801301EF002F8FFF7E6B95A1C3260D5
:10D600001B78EB72304610F094FD3368E8605A1CCA
:10D6100032601B782B7433687268FFF70CBB30469E
:10D6200010F09EFDA884304610F09AFD33687268B1
:10D63000E884D11A03297FF7FAAA1A46591C3160E7
:10D6400012F8021BA97732605B7885F820303046EB
:10D6500010F086FD336872686884FFF7E8BA00BF8F
:10D66000C09E0020BE7D00206890002038B50B4C85
:10D6700023688BB15A68821A002A054604DA0CE046
:10D680005A68AA1A002A07DB9A68226018461A68A4
:10D6900090472368002BF3D138BD38BD8850002057
:10D6A0000D4B04210022890710B4027203F17804A3
:10D6B00002D51979815401329C4203F1180308D034
:10D6C000072A06DC99798907F3D49C4203F11803F1
:10D6D000F6D15DF8044B7047AC2A040810B4104C26
:10D6E0000423214613F001034FF0000201F1180159
:10D6F00008D10132062A0ED08B7913F0010301F113
:10D700001801F6D002EB420204EBC2025DF8044BB2
:10D7100013790370704703705DF8044B704700BFC6
:10D72000AC2A040801233221312241704271037274
:10D7300003700371704700BF2322032302704370FC
:10D74000704700BF436A8269D154436A0169826BA2
:10D7500001338B4228BF00234362002A2FD0EFF30E
:10D760001182502383F31288836B1968C9072CD464
:10D7700070B45E686EB9456A816A8D4217D084695B
:10D780000C44DC600ED9691A59608562002180F86A
:10D790005C10196841F00101D2B2196082F311885E
:10D7A00070BC70470469611A59608662EEE7012314
:10D7B00080F85C30D2B282F3118870BC7047826D01
:10D7C000D36843F08003D3607047D2B282F31188EC
:10D7D000704700BF426B10B462B1C36CC268446949
:10D7E000D11A013B615C5DF8044B08BF1346C3646A
:10D7F000C8B27047016A4369C4685B5C0131A142E9
:10D8000028BF114601625DF8044BD8B2704700BFD3
:10D81000836B13B190F85C007047836A406A181AF2
:10D82000B0FA80F040097047416A836A99420AD38E
:10D83000CB1A816B026961B14968501E0B44834267
:10D840000AD2C01A704702691144CB1A816B0029B1
:10D85000F2D1501EC01A704700207047436B43B18D
:10D86000C26C5B6893422FBF981AC0689B1AC0189D
:10D870007047C269036A9A422FBFD01AC0688018E5
:10D88000C01A70470A4B30B503F1100493F9002019
:10D890005D78072AC8BF143A811804338D7213F8D3
:10D8A000025C855413F8012C0A75A342EED130BDF9
:10D8B000E4FC030803682DE9F041DF691FB13B4632
:10D8C000BDE8F0411847002A164611DD04460D4612
:10D8D0000E4400E023689B68204698470028F9D052
:10D8E000236815F8011B1B6820469847AE42F1D10A
:10D8F000BDE8F0810023252126220170427083704B
:10D90000C3707047038A2DE9F0478589ADB21D4089
:10D9100029D00F4606464FF000484FF00009B5FAEF
:10D9200085F328FA03F2D24391B21B3B15403182B2
:10D93000042B16D8DFE803F03129211903007B6A94
:10D94000002B32D003F1FF3A1FFA8AFAC7F824906D
:10D950003C6A34B123682046514698476468002CDD
:10D96000F8D1002DDBD1BDE8F0873868716B036812
:10D9700089B29847002DD2D1F5E77868B16B03687A
:10D9800089B29847002DCAD1EDE7B868F16B0368FA
:10D9900089B29847002DC2D1E5E7F868316C036879
:10D9A00089B29847002DBAD1DDE7F36A1FFA83FAEE
:10D9B000CEE700BF30B50446806D61718389A268EF
:10D9C00023F400531B041B0C838185B0A3790092C0
:10D9D00013F0040230D04FF4805213F00203ADF87C
:10D9E00004205CD1ADF806304FF480630022ADF81E
:10D9F000083011F00103ADF80C2028D1ADF80A3041
:10DA000008238D07694648BFADF80A3024F0FAFEB6
:10DA1000A279A36DD10724D412F0080F9A8A1BD1E2
:10DA200022F008021204120C9A829A8992B242F4ED
:10DA300000529A8105B030BD13F00203ADF8042006
:10DA40002AD04FF400551346ADF80650CEE7042314
:10DA5000ADF80A300C23D4E792B242F008029A8261
:10DA6000E3E710498B4215D0A1F548418B420FD016
:10DA700001F580618B4209D00B498B42CCD1052046
:10DA80000121FCF7F6FFA279A36DC5E70320F7E7B4
:10DA90000220F5E70020F3E7ADF80630A6E74FF4E3
:10DAA00000539FE7001001400014014010B50446E8
:10DAB000806DA160838923F400531B041B0C8381B8
:10DAC000A37984B013F00402009135D04FF4805252
:10DAD00013F00203ADF804205CD1ADF806304FF42A
:10DAE00080636279ADF80830D1074FF00003ADF8DC
:10DAF0000A30ADF80C3045BF0423ADF80A300823D6
:10DB00000C236946920748BFADF80A3024F07AFE2C
:10DB1000A279A36DD1071FD412F0080F9A8A16D1EB
:10DB200022F008021204120C9A829A8992B242F4EC
:10DB300000529A8104B010BD13F00203ADF8042026
:10DB400025D04FF400511346ADF80610C9E792B244
:10DB500042F008029A82E8E710498B4215D0A1F5FD
:10DB600048418B420FD001F580618B4209D00C49AE
:10DB70008B42D1D105200121FCF77BFFA279A36D57
:10DB8000CAE70320F7E70220F5E70020F3E7ADF846
:10DB90000630A6E74FF400539FE700BF0010014096
:10DBA00000140140022828BF022010B4084C094B81
:10DBB000207000EB8002C0EBC20207495DF8044B05
:10DBC000013003EB4203C0B20B602FF027BA00BF55
:10DBD00008A80020E4A10020C89E002008B519F084
:10DBE000FDF80FF0FFFFBDE8084019F0DFB800BFF7
:10DBF00038B5484B5A899989914224BF00225A81ED
:10DC0000198ADA89914224BF0022DA81DA78CAB10E
:10DC1000072A41496AD091F85300404D0124002160
:10DC20000A282C709C70D9715DD00C2807D0002A6E
:10DC30006CD0DFED3B7A072A0ED00A2862D0DFEDE8
:10DC4000397A09E0344A92F853000A2856D00C2851
:10DC50005BD1D979DFED347A344C9FED350AA27867
:10DC6000002918BFF0EE407A062A04D8314901EBAA
:10DC7000820191ED040A217979B1013A032A0BD886
:10DC8000F7EE007A87EE800A30F0D6FD23889842BE
:10DC900028BF1846208038BD38BD9B781F4A07EE44
:10DCA000103A1178B8EEC77A67EE277A07EE101AA5
:10DCB000B8EEC77A27EE277AB4EEC70AF1EE10FA6B
:10DCC000EADD80EE277AFDEEC77A17EE903A102B48
:10DCD000A8BF1023012BB8BF0123DBB28B4238BF92
:10DCE0000B46137038BDDFED147AA4E791F85300AA
:10DCF0000A2803D00C28ACD0D9799AE7D979DFED7E
:10DD00000E7AA9E7DFED0D7AA6E7D979DFED047A7F
:10DD1000A2E700BFC8B00020ECA800202C7F0020A4
:10DD20006F1203396F12833A0AD7A3394455002082
:10DD30006F120338E4FC03085304E9380F506E3ABD
:10DD40002DE9F047AC4FAD4E19F048F8BE421ED257
:10DD5000DFF82483DFF824934446258862197DB1D7
:10DD60004A450DD2052D0BD933886188C3F30B03C7
:10DD7000994200F0E380144625886219002DEFD106
:10DD80007168304614360FF0B9FEBE42E4D39C4AA7
:10DD90001378A3F1170102290FD99A4911F833001A
:10DDA000002840F0FA80D8000144497829B196490A
:10DDB00011F833300BB918231370944B5A78022A98
:10DDC00000F2DC809249934802EB420201EB8201AF
:10DDD0001A780160022A00F2DA8002EB82018E4B8F
:10DDE000C2EBC10203EB4203998C5A8C8B4C9142DB
:10DDF000236001D300225A84894B9A78042A00F0C8
:10DE0000ED8032B91A88B2F5F07F84BF4FF4F0721A
:10DE10001A80844DFFF7ECFE2B68834A1A40002AD3
:10DE200000F0E580D80700F1D480590400F1CC80DF
:10DE30001A0700F1BB809B0400F1BF8028F0B8F9FD
:10DE400010B97A480DF05CFC40200FF08DFE4FF4C5
:10DE500000700FF089FE4FF400300FF085FE4FF494
:10DE600000100FF081FE4FF000700FF07DFE4FF0BC
:10DE700080600FF079FE26F0F9FD002130226C4819
:10DE800031F097FC206825F0D7FF6A4B256803F135
:10DE9000500102E0043399427DD01A78002AF9D16A
:10DEA0009C78D8788442F5D26349644B0A7028463E
:10DEB0001D601AF06DFF624A62491079624A634B35
:10DEC0001160C822642111FB0021002259609A6070
:10DED000DA601A615A619A61DA6183F8202083F866
:10DEE000212017F03DFA5A4B9FED5A5A1B885A4A87
:10DEF0009FED5A6A50795A4906EE903AF8EEE66A72
:10DF00001388C5EE265A07EE103A53881279C1EDF0
:10DF1000005A07EE903AB8EEC77A524BF8EEE77A1D
:10DF200018725A7227EE067A67EE867ABDE8F047D5
:10DF300083ED017AC3ED007A18F038BF63799B074F
:10DF40007FF419AF716894F804A030460FF0D6FD45
:10DF50003388BAEB133F04D01436BE42FFF4FCAE54
:10DF600015E773887068AA1FC3F30B039A4204F184
:10DF70000601A8BF1A4630F08BFAEDE700225A706E
:10DF80001A78244822490160022A7FF626AF00222F
:10DF90001A70214B28E7012286E7D8000C18646824
:10DFA000002C7FF401AF17241470FDE62E480FF00B
:10DFB000DBFD2B689B047FF541AF2C480FF0D4FDAF
:10DFC00040200FF0D1FD39E729480FF0CDFD2B6837
:10DFD0002EE728480FF0C8FD2B6826E79A8AB2F58D
:10DFE0007A7FBFF416AF4FF47A729A8211E743F04A
:10DFF00008032B6016E700BF2C06000890010008FC
:10E00000687F0020B81E0408F426040808A8002031
:10E01000F0A20020CC9E0020E4A10020C89E002099
:10E02000445500203CA3002009600002289D0020E8
:10E03000882C0020EC5000207D220020BC2C0020E9
:10E04000609600203E7F0020D02C002088680020B1
:10E050009C2E0020C0C9FB48B828002017B7D13833
:10E06000A02E0020C890002001600002094000029C
:10E070000920000208600002024000080080000839
:10E0800008B518F0ABFE0FF0ADFD18F08FFEFFF7EE
:10E0900057FE0120BDE808402EF0C0BF38B50D4C3A
:10E0A0000D4DAC4206D26168204614340FF026FDB7
:10E0B000AC42F8D310F0B8FD084A094B094C146083
:10E0C000002209491A705A7008480860BDE83840B3
:10E0D0001EF0B8BC900100082C060008C89E002065
:10E0E00008A80020E4A10020CC9E0020F0A200207F
:10E0F00008B5FFF7D3FF18F071FE0FF073FDBDE810
:10E10000084018F053BE00BFF0B50C2934D8DFE842
:10E1100001F0893333335E33333334333333070021
:10E12000048C9689B2F802E01788734D24F4805469
:10E130002404240C0484038C8488818B23F40053EE
:10E1400021F4E6411B0409041B0C46EA0E06090CE7
:10E1500043EA063341EA0721A8429BB2A4B289B23E
:10E1600000F09E8005F58065A84200F099809268D5
:10E170008480818302640384F0BD048C9589B2F8A5
:10E1800002C0B2F800E05C4F24F480742404240C34
:10E190000484038C8688818B23F400731B0421F094
:10E1A00073011B0C45EA0C04090443EA0423090C1F
:10E1B000B8429BB2B6B241EA0E015CD04F4CA042CD
:10E1C00059D0926886808183C2630384F0BD048C39
:10E1D0009589B2F802C0B2F800E0474E24F010046E
:10E1E0002404240C0484038C8788018B23F02003EF
:10E1F00021F4E6411B0409041B0C45EA0C04090C3C
:10E2000043EA041341EA0E21B0429BB2BFB289B285
:10E210005DD03A4CA0425AD09268878001838263D5
:10E220000384F0BD048C9789B2F802E01688324D61
:10E2300024F001042404240C0484038C8488018BBE
:10E2400023F002031B0421F073011B0C47EA0E07A5
:10E2500009043B43090CA8429BB2A4B241EA06015F
:10E2600025D005F58065A84221D09268848001837D
:10E2700042630384F0BDD589148A578A23F400636E
:10E2800043EA05254FF6FF332B40958826F4405688
:10E290003C4343EA052346EA04169BB2B6B290E734
:10E2A000158A24F4804444EA8514A4B25FE7D68931
:10E2B000158A578A23F00803334324F44074968860
:10E2C0003D4323F004032C433343A4B2CDE7D48968
:10E2D000158A568A23F0800343EA04134FF6BF746D
:10E2E0001C40938827F44067354344EA031347EA08
:10E2F00085079BB2BFB28FE70000014000040140D8
:10E300002DE9F04F7822002183B08A488A4CDFF84B
:10E310004C928A4D8A4E8B4FDFF8448231F049FA95
:10E3200089488A49DFF83CE2DFF83CC200221359F1
:10E33000834200F0D480B3F1804F00F0E480AB4220
:10E3400000F0E380B34200F0E280BB4200F0E180E5
:10E35000734500F0E080634500F0DF80434500F046
:10E36000DE80DFF808A2534500F0DB800AF5806A02
:10E37000534500F0D8800AF5806A534500F0D580F7
:10E38000AAF5983A534500F0D2800AF5806A5345C1
:10E390007BD00AF5806A534508BF0D2376D018322A
:10E3A000902AC4D1644C6A4E6A4F6B4D04F19008B8
:10E3B00002E01834A04565D0A379002BF9D0237969
:10E3C0004FEA131909F1FF39B9F1030F03F00F03F5
:10E3D000EFD836F8190040FA03F2D207E9D54FF02A
:10E3E000010A0AFA03F3013B18402FF00DFE17F85B
:10E3F0000930184415EBC002DBD055F83000DFF8C7
:10E4000070E1217A00F13F4303F57E039B0A1EF879
:10E41000033003F01F0E5B09032B0AFA0EFA60D0DB
:10E42000042B67D0022B51D093880093B3FA83F367
:10E43000C3F11F039BB2DA0800EB820203F007036B
:10E44000D2F820E09B004FF00F0C0CFA03FC2EEAF0
:10E450000C0EC2F820E0D2F820E001FA03F343EA00
:10E460000E03136269460023022218348DF804203B
:10E470008DF805308DF806308DF8073024F0BCFBA0
:10E48000A04599D103B0BDE8F08F0C2309EBC3037D
:10E490004FF0010A1B7903F01F0B5B09032B0AFAEB
:10E4A0000BFA0ED0042B07D0022B7FF478AF4B6C05
:10E4B0004AEA03034B6472E70B6B4AEA03030B63FC
:10E4C0006DE70B6C4AEA03030B6468E7DFF87CE056
:10E4D000DEF844304AEA0303CEF84430A4E70023D0
:10E4E000D4E7DFF868E0DEF840304AEA0303CEF80C
:10E4F000403099E7DFF854E0DEF830304AEA0303B1
:10E50000CEF8303090E70123C0E70223BEE70323B3
:10E51000BCE70423BAE70523B8E70623B6E70723D9
:10E52000B4E70823B2E70923B0E70A23AEE70B23D9
:10E53000ACE700BFB4A00020AC2A040800040040EF
:10E5400000080040000C004000000140003802407C
:10E55000402B04083C2B0408B4A50020481E0408E6
:10E560000004014000100040001400400040014041
:10E57000742B040800286AD003682DE9F04F03F1DA
:10E580003F4404F57E045F4EA40A0125345D04F087
:10E590001F066409032C05FA06F559D0042C00F077
:10E5A000AC80022C59D08588B5FA85F0C0F11F00E7
:10E5B00080B2C40803EB840400F00700266A8000E0
:10E5C0000F27874026EA07062662276A01F003061E
:10E5D0008240701E3A430128C1F3810CC1F3001838
:10E5E0002262C1F341113DD90024224601274FF098
:10E5F000030E03E0102A04F1020426D007FA02F009
:10E60000A84302F10102F5D1D3F800C00EFA04F0DC
:10E61000C04300EA0C0CC3F800C0D3F8008006FA2F
:10E6200004FC4CEA080CC3F800C0D3F80CC000EAA4
:10E630000C00D860D3F80CC001FA04F040EA0C00DA
:10E64000102AD86004F10204D8D1BDE8F08F7047D9
:10E650002D4C266C35432564A5E72B4C666C354361
:10E660006564A0E7002002464FF0010E4FF0030959
:10E6700004E00132102A00F102003CD00EFA02F749
:10E6800037EA0504F5D1D3F800A009FA00F4E44311
:10E690000AEA040AC3F800A0D3F800B006FA00FAA8
:10E6A0004AEA0B0AC3F800A0D3F808A004EA0A0A51
:10E6B000C3F808A0D3F808B00CFA00FA4AEA0B0A2B
:10E6C000C3F808A0D3F804A02AEA07075F60D3F8CC
:10E6D00004A008FA02F747EA0A075F60DF683C40D7
:10E6E000DC60DF6801FA00F401323C43102ADC6090
:10E6F00000F10200C2D1BDE8F08F034C266B354318
:10E70000256350E7742B04080038024003682DE9A4
:10E71000F04F03F13F4404F57E04604EA40A012546
:10E72000345D04F01F066409032C05FA06F500F0B9
:10E73000AF80042C00F0A780022C54D08588B5FA55
:10E7400085F0C0F11F0080B2C40803EB840400F020
:10E750000700266A80000F27874026EA0706266200
:10E76000276A01F0030602FA00F0721E3843012AFC
:10E77000C1F3810CC1F300182062C1F3411137D9F4
:10E780000024224601274FF0030E03E0102A04F173
:10E79000020426D007FA02F0A84302F10102F5D1E3
:10E7A000D3F800C00EFA04F0C04300EA0C0CC3F822
:10E7B00000C0D3F8008006FA04FC4CEA080CC3F849
:10E7C00000C0D3F80CC000EA0C00D860D3F80CC02D
:10E7D00001FA04F040EA0C00102AD86004F10204A7
:10E7E000D8D1BDE8F08F2E4C666C35436564A5E743
:10E7F000002002464FF0010E4FF0030904E0013201
:10E80000102A00F102003CD00EFA02F737EA0504A4
:10E81000F5D1D3F800A009FA00F4E4430AEA040AA7
:10E82000C3F800A0D3F800B006FA00FA4AEA0B0ACF
:10E83000C3F800A0D3F808A004EA0A0AC3F808A0A5
:10E84000D3F808B00CFA00FA4AEA0B0AC3F808A099
:10E85000D3F804A02AEA07075F60D3F804A008FAF7
:10E8600002F747EA0A075F60DF683C40DC60DF6868
:10E8700001FA00F401323C43102ADC6000F102008E
:10E88000C2D1BDE8F08F064C266B3543256355E7B2
:10E89000034C266C3543256450E700BF742B0408F5
:10E8A0000038024010B50409013C032C17D80D4B69
:10E8B00033F8142000F00F0042FA00F313F00103C4
:10E8C0000DD0012303FA00F0013810402FF09CFB1B
:10E8D000054A064B125D104403EBC00010BD00203A
:10E8E00010BD00BF402B04083C2B0408B4A5002039
:10E8F00001490248FFF706B804A1002000080040C3
:10E9000001490248FEF7FEBFDCA0002000040040E1
:10E9100002494FF08040FEF7F5BF00BFB4A00020D1
:10E92000F0B50668B30AA3F58013022B50D8384C13
:10E93000E55C022D4CD84379A8009F08002952D0ED
:10E940009C080223B6F80CE0A340441907EB4407E7
:10E9500043EA0E032F4C07F1040E9BB244F8271034
:10E9600044F82E20B381EFF31181502383F31288F2
:10E970004219D200A7183B695BB33B6204334219CA
:10E9800004EBC202576917B11F605369043342197F
:10E9900004EBC202976917B11F60936904334219EF
:10E9A00004EBC202D76917B11F60D3690433002298
:10E9B000C9B21A6081F31188284404EBC004236AA9
:10E9C0005BB9B38923F001031B041B0CB381F0BDB9
:10E9D000F0BD02F120032344D1E7B3899BB243F099
:10E9E0000103B381F0BDB3890A4C4FF0020E0EFA59
:10E9F00007FE9BB223EA0E0300EB050E07EB4E0762
:10EA0000B3813B1D44F8271044F82320ABE700BF37
:10EA10003C290408B4A0002010B5036882480139DD
:10EA2000834282B089B200F0CA80A0F58060834240
:10EA300000F0C58000F58040834200F0B78000F50B
:10EA40008060834200F0B28000F58060834200F075
:10EA5000AD80764C188824686408B4FBF2F4013C5D
:10EA6000A4B282B2B3F1804F0AD07148834207D07A
:10EA700000F58060834203D000F58060834202D1BC
:10EA800022F0700292B26B48834200F0A18000F540
:10EA90008060834200F0A68022F4407200F56C4052
:10EAA00092B283421A80D9621C854FD05E4A93424B
:10EAB0004CD001229A821A8892B242F001021A8046
:10EAC000B3F1804F00F09880594A934200F096804D
:10EAD00002F58062934200F0938002F580629342D7
:10EAE00000F0908002F58062934200F08D8002F584
:10EAF0008062934200F08A8002F57042934200F0F7
:10EB0000878002F57052934200F0848002F58062A3
:10EB1000934200F0818002F5806293427ED0A2F59C
:10EB2000983293427CD002F5806293427AD002F50B
:10EB30008062934208BF0D2215D002A84FF0012336
:10EB400040F8043D23F0CEFD02B010BD01220021AB
:10EB500019869A821A88384892B242F0010283429A
:10EB60001A80ADD10A46354B03EBC20301A85C798C
:10EB70008DF80440012300228DF805308DF8073010
:10EB80008DF8062023F0AEFD1B2C08D02E2CDBD1F7
:10EB90002B4B019301A823F0A5FD02B010BD294B1A
:10EBA000019301A823F09EFD02B010BD1F4C1888F0
:10EBB0002468B4FBF2F4013CA4B282B252E71B4CCD
:10EBC00018882468B4FBF2F4013CA4B282B257E77F
:10EBD00001201A80D9621C8598821A8892B2024359
:10EBE0001A8071E701201A80D9621C8598821A88E0
:10EBF00092B202431A8063E70122B4E70222B2E72D
:10EC00000322B0E70422AEE70522ACE70622AAE71A
:10EC10000722A8E70822A6E70922A4E70A22A2E71A
:10EC20000B22A0E70C229EE700040140E8A8002088
:10EC3000000400400010004000000140481E04088D
:10EC40002C010001190100012B4B98423CD0B0F17E
:10EC5000804F3BD0A3F57C43984239D003F58063C5
:10EC6000984237D003F58063984235D003F580632E
:10EC7000984233D003F58063984231D003F5704356
:10EC800098422FD003F5705398422DD003F580633E
:10EC900098422BD003F58063984229D0A3F598338E
:10ECA000984227D003F58063984207D003F580632C
:10ECB000984208BF0D2202D0002070470C220F4B53
:10ECC00003EBC203187970470022F8E70122F6E748
:10ECD0000222F4E70322F2E70422F0E70522EEE73E
:10ECE0000622ECE70722EAE70822E8E70922E6E73E
:10ECF0000A22E4E70B22E2E700000140481E040874
:10ED00002DE9F04F013085B0C3B203930B46029159
:10ED10008B4C8C4E002B00F09A8032208A4D8B4F0A
:10ED2000DFF82C922CF0F6FD4FF4FA7A4FF0100C2D
:10ED30004FF47A70D9F80430C3F30803002B40F085
:10ED4000DE80EFF31183002B40F0D9802968A268A0
:10ED500000BF2B689942F9D1D7F800E000FB0EF311
:10ED60009B1AB3FBFEF300FB01314FF0010E019142
:10ED7000D9F80430C3F30803002B40F08780EFF389
:10ED80001183002B40F082802B68A16800BF2A68A5
:10ED90009342F9D1D7F800B000FB0BF2521AB2FB44
:10EDA000FBF200FB0323019A9B1AB3F57A7FDFD3B2
:10EDB000BAF1010ABED1039B002B40F0BD804FF495
:10EDC0007A7ADFF88C9150464FF0100CD9F8043065
:10EDD000C3F30803002B75D1EFF31183002B71D11E
:10EDE0002968A26800BF2B689942F9D1D7F800E0E2
:10EDF00000FB0EF39B1AB3FBFEF300FB01314FF057
:10EE0000010E0191D9F80430C3F3080313BBEFF3EB
:10EE10001183FBB92B68A16800BF2A689342F9D11E
:10EE2000D7F800B000FB0BF2521AB2FBFBF200FB6A
:10EE30000323019A9B1AB3F57A7FE3D3BAF1010A4F
:10EE4000C4D1029B013B0293002B7FF466AF05B057
:10EE5000BDE8F08FEFF311888CF31288A168236866
:10EE6000DB0344BFC6F800E0A1682B6832685FFA94
:10EE700088F888F31188D7F800801A4400FB08F35B
:10EE80005B1AB3FBF8F300FB0233D2E7EFF3118810
:10EE90008CF31288A1682368DB0344BFC6F800E046
:10EEA000A1682B6832685FFA88F888F31188D7F870
:10EEB00000801A4400FB08F35B1AB3FBF8F300FB75
:10EEC000023370E7EFF311828CF31288D4F808E074
:10EED0002368D90303D501233360D4F808E02B68F5
:10EEE0003168D2B282F311883A68194400FB02F308
:10EEF000A3EB0E03B3FBF2F300FB01317FE7EFF36B
:10EF000011828CF31288D4F808E02368D90303D562
:10EF100001233360D4F808E02B683168D2B282F361
:10EF200011883A68194400FB02F3A3EB0E03B3FB0C
:10EF3000F2F300FB013118E718462CF04DFB3EE7D9
:10EF400010E000E0E0A70020E4A70020E8A70020F0
:10EF500000ED00E0204B5B68C3F3080330B4BBB99D
:10EF6000EFF31183A3B91D4B1D4C1868A16800BFB6
:10EF70001A689042F9D11B4B1C684FF47A7202FB5D
:10EF800004F3591AB1FBF4F130BC02FB00107047D6
:10EF9000EFF31182102383F3128811498C680B68F8
:10EFA00013F4803F104B02D0012018608C680B498D
:10EFB000D2B20D68186882F311880A4B19684FF4B1
:10EFC0007A72284402FB01F31B1B30BCB3FBF1F344
:10EFD00002FB0030704700BF00ED00E0E4A7002016
:10EFE00010E000E0E8A70020E0A700202DE9F84F9E
:10EFF0008046FFF7AFFF254E2549DFF8A0E0254A00
:10F00000254D844610274FF47A740120DEF8043031
:10F01000C3F30803D3B9EFF31183BBB90B68D2F87C
:10F0200008A000BFD1F800904B45F7D1D6F800B04A
:10F0300004FB0BF9A9EB0A09B9FBFBF904FB0393E9
:10F04000A3EB0C034345E1D3BDE8F88FEFF3118A3E
:10F0500087F31288D2F808B01368DB0344BF286036
:10F06000D2F808B00B68D5F800905FFA8AFA8AF3F4
:10F070001188D6F800A0994404FB0AF3A3EB0B0314
:10F08000B3FBFAF304FB0933DAE700BFE8A700207B
:10F09000E4A7002010E000E0E0A7002000ED00E081
:10F0A0002DE9F04FDFF830C1474A4849484E494DF5
:10F0B0008046102718F1FF38C0F08480DCF8043057
:10F0C000C3F30803002B5CD1EFF31183002B58D15D
:10F0D0000B68946800BF08688342F9D1D6F80090A5
:10F0E0004FF47A7000FB09FEAEEB040EBEFBF9FE96
:10F0F00000FB03EEDCF80430C3F308034FF47A742A
:10F100000120FBB9EFF31183E3B90B68D2F808A033
:10F1100000BFD1F800904B45F7D1D6F800B004FB02
:10F120000BF9A9EB0A09B9FBFBF904FB0393A3EB69
:10F130000E03B3F57A7FBDD2DCF80430C3F30803C5
:10F14000002BDFD0EFF3118A87F31288D2F808B0D2
:10F150001368DB0344BF2860D2F808B00B68D5F809
:10F1600000905FFA8AFA8AF31188D6F800A09944D1
:10F1700004FB0AF3A3EB0B03B3FBFAF304FB093321
:10F18000D5E7EFF3118487F31288D2F8089013685B
:10F19000D80303D501232B60D2F808900B682868A8
:10F1A000E4B284F31188D6F800A04FF47A7400EB2F
:10F1B000030E04FB0AF3A3EB0903B3FBFAF304FB0E
:10F1C0000E3E97E7BDE8F08F10E000E0E4A70020D6
:10F1D000E8A70020E0A7002000ED00E030B4EFF346
:10F1E0001183102282F312880649074C0A680748E7
:10F1F000013200250A602560DBB2026883F31188C2
:10F2000030BC7047E4A70020E0A7002010E000E039
:10F21000014B5869FBF734B928420020014BD868EC
:10F22000FBF72EB928420020014B9868FBF728B95C
:10F2300028420020014B1868FBF722B92842002021
:10F2400070B4EFF31186502383F31288836B1A682E
:10F25000D20720D45D686DB9446A826A944217D09F
:10F2600081691144D9600ED9A21A5A6084620022C1
:10F2700080F85C201A6842F00102F1B21A6081F352
:10F28000118870BC704701698A1A5A608562EEE77E
:10F29000012380F85C30F3B283F3118870BC7047AF
:10F2A00003685B6A03B11847704700BF03681B6AB5
:10F2B00003B11847704700BF03682DE9F041DF69CB
:10F2C0001FB13B46BDE8F0411847002A164611DD44
:10F2D00004460D460E4400E023689B68204698478C
:10F2E0000028F9D0236815F8011B1B6820469847B1
:10F2F000AE42F1D1BDE8F08103689B69184700BFB9
:10F3000003685B69184700BF03681B69184700BFA3
:10F310000368DB68184700BF03689B68184700BF95
:10F3200003685B68184700BF03681B68184700BF85
:10F3300038B50C46097849B1054601342B68284692
:10F340001B68984714F8011B0029F7D138BD00BF8E
:10F35000064B53F820302BB11A689B8851690B4239
:10F3600001D1138370475383704700BFB0A70020BB
:10F37000026802F13F4303F57E032DE9F04F9B0A3B
:10F38000544DEB5C03F01F055B090124032B04FAC9
:10F3900005F400F09980042B00F09180022B3ED000
:10F3A00001F00306731E012BC1F3810CC1F3001899
:10F3B0008588C1F3411137D90024234601274FF036
:10F3C000030E03E0102B04F1020426D007FA03F029
:10F3D000A84303F10103F5D1D2F800C00EFA04F0FE
:10F3E000C04300EA0C0CC2F800C0D2F8008006FA54
:10F3F00004FC4CEA080CC2F800C0D2F80CC000EAC9
:10F400000C00D060D2F80CC001FA04F040EA0C0005
:10F41000102BD06004F10204D8D1BDE8F08F2E4B40
:10F420005D6C2C435C64BBE7002003464FF0010E8B
:10F430004FF0030904E00133102B00F102003CD02F
:10F440000EFA03F737EA0504F5D1D2F800A009FA5D
:10F4500000F4E4430AEA040AC2F800A0D2F800B0BB
:10F4600006FA00FA4AEA0B0AC2F800A0D2F808A08D
:10F4700004EA0A0AC2F808A0D2F808B00CFA00FAA6
:10F480004AEA0B0AC2F808A0D2F804A02AEA070741
:10F490005760D2F804A008FA03F747EA0A07576052
:10F4A000D7683C40D460D76801FA00F401333C438C
:10F4B000102BD46000F10200C2D1BDE8F08F064BE2
:10F4C0001D6B2C431C636BE7034B1D6C2C431C64AE
:10F4D00066E700BF742B0408003802402DE9F04FA6
:10F4E0004A484B494B4B4C4C4FF0010A4FF0020934
:10F4F0004FF004084FF0080C4FF0100E2027402664
:10F50000802530F8022B12F0010F03D01960A3F808
:10F5100004A0083312F0020F03D01960A3F804907E
:10F52000083312F0040F03D01960A3F804800833E5
:10F5300012F0080F03D01960A3F804C0083312F0CA
:10F54000100F03D01960A3F804E0083312F0200F65
:10F5500002D019609F80083312F0400F02D019606A
:10F560009E80083312F0800F02D019609D8008330E
:10F5700012F4807F05D04FF4807B1960A3F804B0AB
:10F58000083312F4007F05D04FF4007B1960A3F814
:10F5900004B0083312F4806F05D04FF4806B19600B
:10F5A000A3F804B0083312F4006F05D04FF4006BD9
:10F5B0001960A3F804B0083312F4805F05D04FF44B
:10F5C000805B1960A3F804B0083312F4005F05D023
:10F5D0004FF4005B1960A3F804B0083312F4804FB5
:10F5E00005D04FF4804B1960A3F804B00833D20B58
:10F5F00004D04FF4004219609A80083301F580610D
:10F60000A1427FF47EAFBDE8F08F00BF402B04081D
:10F6100000000240B4A5002000100240002855D090
:10F62000026802F13F4303F57E032DE9F04F9B0A88
:10F63000544DEB5C03F01F055B090124032B04FA16
:10F6400005F444D0042B00F09780022B44D001F045
:10F650000306731E012BC1F3810CC1F300188588CA
:10F66000C1F341113DD90024234601274FF0030E79
:10F6700003E0102B04F1020426D007FA03F0A8439C
:10F6800003F10103F5D1D2F800C00EFA04F0C04333
:10F6900000EA0C0CC2F800C0D2F8008006FA04FCA4
:10F6A0004CEA080CC2F800C0D2F80CC000EA0C000A
:10F6B000D060D2F80CC001FA04F040EA0C00102B24
:10F6C000D06004F10204D8D1BDE8F08F70472E4B12
:10F6D0001D6C2C431C64BAE72B4B5D6C2C435C64A3
:10F6E000B5E7002003464FF0010E4FF0030904E098
:10F6F0000133102B00F102003CD00EFA03F737EA79
:10F700000504F5D1D2F800A009FA00F4E4430AEAAE
:10F71000040AC2F800A0D2F800B006FA00FA4AEAD9
:10F720000B0AC2F800A0D2F808A004EA0A0AC2F83C
:10F7300008A0D2F808B00CFA00FA4AEA0B0AC2F89C
:10F7400008A0D2F804A02AEA07075760D2F804A05C
:10F7500008FA03F747EA0A075760D7683C40D460C5
:10F76000D76801FA00F401333C43102BD46000F158
:10F770000200C2D1BDE8F08F034B1D6B2C431C630C
:10F7800065E700BF742B04080038024010B103681D
:10F7900082885A83704700BF10B1036882881A8339
:10F7A000704700BF18B10368828809B95A8370474F
:10F7B0001A8370470E4B1B8801463BB90D4B0E4A0E
:10F7C0001B7810680BB981F00101EBE70B4B5A690C
:10F7D0001AB118B91A68106058747047084A186846
:10F7E0001188084A92FBF1F20121026059747047B6
:10F7F000BCA70020BEA70020C0A70020C4A70020EF
:10F80000DCA7002020A1070010B40A4B0A4A1C788C
:10F8100001238340234052F8200029B9B3FA83F131
:10F8200049095DF8044BBDE7191C18BF01215DF8BB
:10F83000044BB7E7ACA70020B0A7002008B5012112
:10F840000220FFF7E1FF094B1B7803F00503052BAE
:10F8500008D000210120FFF7D7FF00210846FFF75D
:10F86000D3FFFEE724F02EFCF3E700BF2442002084
:10F8700030B1036882881B691A4214BF012000203E
:10F88000704700BF2DE9F0410B4E346873691C408E
:10F890000FD0DFF828800127B4FA84F3C3F11F03E7
:10F8A00007FA03F558F8230003689847AC437561DD
:10F8B000F2D1BDE8F08100BF003C01403CA7002030
:10F8C0002DE9F0410B4E346873691C400FD0DFF80E
:10F8D00028800127B4FA84F3C3F11F0307FA03F564
:10F8E00058F8230003689847AC437561F2D1BDE82E
:10F8F000F08100BF003C01403CA700202DE9F04111
:10F900000B4E346873691C400FD0DFF82880012744
:10F91000B4FA84F3C3F11F0307FA03F558F8230080
:10F9200003689847AC437561F2D1BDE8F08100BF30
:10F93000003C01403CA700202DE9F04FBC4B1E7855
:10F940008BB0002E40F08180BA4BBB4C1D78BB4F72
:10F95000DFF80CB305F00105A4F10A0954F80A0C0C
:10F96000B8B14FF0CC0808FB0698FFF7D9FC80B17E
:10F9700054F80A0CFFF7CCFC14F8023C024683B999
:10F9800024283BD075B354F80A0CFFF7C9FC0028B3
:10F99000EED10136032E04F1CC04DFD10BB0BDE86B
:10F9A000F08F012B2ED0022B33D0032B40D0042B11
:10F9B00000F06981052B00F05781062BE3D114F884
:10F9C00001ECBEF1000F00F0D881BEF1010F00F094
:10F9D0001B8201360023032E04F8023C04F1CC0400
:10F9E000BCD1DBE7232A54F80A0C00F08281944B47
:10F9F00093F82A309342B8D1FAF726FD012304F890
:10FA0000023CC0E74D2800F06781002304F8023C67
:10FA1000B9E700233C2804F8023C00F057813E2857
:10FA2000B1D10122032304F8012C04F8023CAAE717
:10FA3000C028EAD80021042304F8050C04F8040CBB
:10FA400004F8061C04F8023C9DE77E4B1868002869
:10FA5000A4D00DF0B5FFDFF80CA27B4DDFF8F891D4
:10FA6000DAF80000FFF75CFC002897D0DAF8000015
:10FA7000FFF74EFC09281BD03F2819D02B68002B1C
:10FA800067D1042800F0BA810C2800F0CA807F28D2
:10FA9000E6D0A0F12002D2B25E2AE1D80BB920282C
:10FAA000DED05A1C09F803002A600FF0ADFBD7E73F
:10FAB0002C68002C5AD1654FA34607F52078BBF17E
:10FAC000000F08BFBB4610374745F8D1BBF1000F08
:10FAD00000F04E81103FDBF800003A68065D135DD0
:10FAE0009E42204402EB040140F04081661E4E44D9
:10FAF00022460BB9FD2A5CD906F8013F01322A6083
:10FB000010F8013F11F801EF9E45F2D00AB15F45B0
:10FB100012D04F480FF080FB5F4508D35BF8100B05
:10FB20000FF07AFB09200FF06FFBBB45F6D949486F
:10FB30000FF072FB2A680024944291D2661E4E4454
:10FB400016F8010F0FF060FB2B6801349C42F7D3CD
:10FB500086E70C2865D00A2834D00D2832D07F28BB
:10FB600000F0BE80FF2B3FF67BAF92E7374E0027B9
:10FB700006F52078BB4602E0103646450DD02246F9
:10FB8000316848460EF078FA0028F5D1B346002FC8
:10FB9000F2D1374610364645F1D13B465F469B468B
:10FBA000002B98D1002F3FF45BAF29480FF034FBB6
:10FBB000B4E7511C202009F80200296009F801303F
:10FBC0000A46A4E70FF0A9FB232123482FF008FEE3
:10FBD000002800F01181A0EB0900286090B1431EBD
:10FBE00019F80310202940F02C8109EB030243B1DE
:10FBF00012F8011D202903F1FF304FD10346002BDD
:10FC0000F6D12B604FF48072002148462FF0D1FDD1
:10FC1000074B1B78002B3FF4C1AE0E480FF0FCFAE7
:10FC20001EE70E480FF0F8FA0A480FF0F5FA17E74A
:10FC300080540020609000209A610020D828002085
:10FC4000289D0020C4480020A44500201816040860
:10FC5000882D0408902D0408A4440020982D040841
:10FC600010FD0308A044002014F8063C14F8051CFD
:10FC700099426FD814F8043C83427FF4C6AE062341
:10FC800004F8023C9BE614F8043C04F8030C5A40C8
:10FC9000052304F8042C04F8023C74E62B606A4C3B
:10FCA000002204F5207809F8032002E010344445CE
:10FCB0004CD02168484612F087FB0028F6D0444516
:10FCC00044D2E368984700232B609BE7032204F8A3
:10FCD000013C04F8022C56E6022304F8023C52E6EA
:10FCE000013B002259482B6009F803200FF094FAD9
:10FCF000B6E6574B5749DB78574ADFF888E1106082
:10FD0000003318BF01230B70544B554ACEF8003016
:10FD1000544B7A604FF0400E012187F80CE03860B8
:10FD2000B8607D73504819700FF042FF4F480FF0D4
:10FD300073FA4FF400600BF0C5FB4D4B93F82A307B
:10FD4000232B3FF459AE14F8023C36E649480FF035
:10FD500063FAB8E714F8041C08EB030051400133C0
:10FD600004F8041C04F8063C82720CE62246CDE638
:10FD70004148103F0FF050FAD0E69BE80F000DF11C
:10FD8000280C0DF1080888E80F004CF824ED14F851
:10FD9000053C14F803AC0694624623444FF0010C72
:10FDA000414606A8ADF822E00793ADF820A08DF8F3
:10FDB00024C0FBF7C9FC40B1029A304B0392414684
:10FDC000A4F10A0002930CF0FFF8DDF80480002390
:10FDD00004F8023CB8F1000F3FF4DBAD54F80A0C14
:10FDE0000CF07AF9013654F80A0CC047032E04F1DE
:10FDF000CC047FF4B3ADD1E52868EFE6204811F0DC
:10FE0000A3FB0BB0BDE8F08F14F8053C14F8032CED
:10FE10000694234407936E2A4FF000030893099336
:10FE2000ADF820207FF4D5AD06A80EF0A4F906A801
:10FE30000EF096F906A80EF093F906A80EF090F9C8
:10FE4000C7E503462BE700BF18160408C02D0408B9
:10FE500008A8002028300020A0440020DC28002032
:10FE6000B5D8000880540020C42D0408902D040843
:10FE7000289D0020A42D0408882D04084CB30020E0
:10FE8000A4440020C44800202DE9F04F2DED028B42
:10FE900093B0054627F014FA994B1E7826B113B09B
:10FEA000BDEC028BBDE8F08F964B1B685805F6D56C
:10FEB000DFF89C82D8F80020002A00F01E81924CC6
:10FEC000D4F8283103F5F43348339D42C0F015814E
:10FED0008E4F94F82C313968C4F828510133DBB2C5
:10FEE000890784F82C3101F1ED8513F0070901F041
:10FEF0002B85282B864B029301F026875E209047A6
:10FF0000844B1B78002B6BD07F4C834AD4F8343160
:10FF1000EB1A934201F2D683DFF838A29AF80080F8
:10FF2000B8F1000F33D1DFF80092D9F80000FFF7E5
:10FF3000F7F9C0B201280ED90228784F41F0C487E2
:10FF40003B78002B42F01D81D4F83C31EB1AB3F51D
:10FF50007A6F82F07B8172480768002F40D09AF850
:10FF60000030BBB96F4BD9F800001B689B781E3B73
:10FF7000012B4FF0020142F21481043027F058F8AF
:10FF8000012200238AF8002084F8483126E06448E2
:10FF900007682FB3D4F8443140F6B732EB1A9342D6
:10FFA0001ED994F84031002B01F08487013BDBB26D
:10FFB00084F84031002B01F0F28517F8011B94F80A
:10FFC0004821076094F8493157480A4401330068D2
:10FFD00084F8482184F84931FFF7A6F9C4F8445160
:10FFE000524A029B12781B68012A03F101030A930B
:10FFF00001F092824E4B1B787BB1DFF85C81D8F820
:020000040801F1
:10000000003053B1029B404CD3F800B0D4F85C31BF
:10001000ABEB0303632B01F2BC81DFF8408198F85E
:1000200000A0BAF1020F01F096853C4F97F87430AA
:10003000032B01F050843F4B1B7873B13E4E336865
:100040005BB1314CFEF786FFD4F86831039044F67B
:100050001F62C31A934200F22581384B1B78002B94
:100060007ED1374B1B7843B1274CD4F8B83203F517
:100070000043E8339D4281F0C582324B1B78002B50
:100080003FF40DAF204E304C304D06F2C1272068B2
:10009000FFF746F900283FF402AF2068FFF738F970
:1000A0002B7880465A1E33B120682A70FFF738F942
:1000B0000028F2D1F3E603223946781E2FF05FFBC9
:1000C00096F8C03296F8C12286F8C38283F47F4343
:1000D00083F0FF039B1A1FFA88F89BB2B8EB132F2B
:1000E000D5D196F8C222DBB29A42D0D1781E1BF04D
:1000F0009BFB2B7818442870C9E7054B0293FFE659
:1001000080540020ECB0002028290020709E0020A0
:10011000E4A700207A9F00203F0D0300200000206C
:10012000E09E0020DC9E0020D89E00207B9F0020C7
:10013000889F0020909F0020949F002000A0002016
:1001400011A000209A9F0020A09F0020A49F0020C3
:10015000E89E0020E49E002050680020725000209D
:10016000444C2278002A41F0CE81DFF8349199F88E
:100170000040002C72D1404E3078002841F08C872E
:100180003E4C3F4ED4F8B02231783E4B93FBF1F316
:1001900013449D42FFF465AF94F8B4323A4AC4F870
:1001A000B052D75CFB0702F16781B80702F1B0805B
:1001B000790702F16D803A0745D5344B344F0B93E4
:1001C0000DF14809A3F13D0249F8202D0021A3F1CA
:1001D000400203F8401C02231121517093704846DD
:1001E00039680DF0D7FF484679680DF0D3FFFB89D9
:1001F000284903EBC3039B00053381FB0321DB1775
:10020000C3EBA10189B248460DF0DBFF3B8A03EB4B
:100210008303590089B248460DF0D3FF1E4B1B786B
:100220009B0743BF398901F57A7189B24FF47A711E
:1002300048460DF0C6FF0A9B3A7D591C0A91484674
:100240001A7026F0E3FF94F8B4323178013393FB4F
:10025000F1F201FB123384F8B43202E70F4E376E2D
:10026000002F41F02585054B89F80070C3F8B05286
:10027000F7E600BF6C9F002008A00020282900207E
:1002800010A00020A08601000CA000202C9F0020C0
:10029000EC58002067666666C69E002018A0002005
:1002A00009A0002094F86E31002B41F08084DF4BD0
:1002B0001B6803F00802002A48F603414AF60B4087
:1002C0004BF60F4249F6074704BF02460F4613F0AC
:1002D000040F4FF0190118BF17469B0684F86E11E2
:1002E00003D547F4804747F020070BF051FCC7F3D4
:1002F0000909002842F0C781CD4B9B79002B42F0C1
:100300004F82984664204FF0FF3A4FF0000C0A9756
:100310000B97ADF834C0CDF83AC0CDF83EC0CDF85B
:1003200042C0CDF83090ADF83680ADF838A08DF8E9
:1003300046000AAF0FCFDFF808E384F805C0AEE847
:100340000F0097E80F00AEE807002EF8023B714659
:100350004FF0010C1B0CFE271F20C82201F81E398C
:10036000A770A27184F807C0E07094F87E01207134
:1003700080F0F10383EA0313DAB2130983F0E70391
:1003800043EA022383EAC2031BB283EA0312D2B216
:10039000C3F3072383EA121343EA022383EAC20367
:1003A0001BB283F0C80282EA0212D2B2C3F307235F
:1003B00083EA121343EA022383EAC2031BB283EAED
:1003C0000C0787EA0717FFB2C3F3072282EA171266
:1003D00042EA072200EB0C0382EAC7070EEB0C008F
:1003E00084F87E31278011F8013B7B4083EA0313B8
:1003F000DBB21A0982EA172242EA032282EAC30325
:100400001BB29FB281422780EDD183F07C0383EA47
:100410000313DBB24FEA131E8EEA172E8EEA032E69
:100420008EEAC30E0FFA8EFE1FFA8EF9DFF814C2A1
:10043000A4F800905FFA8EFE4FEA192984F82890FC
:1004400084F827E00CF5D37804F1220ADCF80000E8
:10045000DCF80410DCF80820DCF80C3047460FC745
:100460000CF1100CD445B846F0D1DCF8000038602F
:10047000704F9CF8043088F8043007F1270884F89E
:10048000CDE184F8CE9117F8011F3068FEF74CFFDC
:10049000B845F8D194F86F21002A41F0F4836649F9
:1004A000029B08781B680A2184F86F11002801F06C
:1004B0002C85DFF894E10128BEF80010059142F286
:1004C000FE810228BEF8028002F0F580BEF804101A
:1004D0000491032802F00E820428BEF806A002F060
:1004E00004820528BEF8087002F0FB810628BEF8D9
:1004F0000AC002F0F3810728BEF80C1001D0BEF844
:100500000E2094F87EB10A938BF0300383EA031334
:10051000DBB24FEA131E494884F804B08EF07A0E1D
:100520004EEA032E00888EEAC303DFF820E1C0EB19
:1005300000208EFB009E8644C0171BB2C0EB6E20CD
:100540000690C3F3072E83EA0310059BC0B24FF059
:10055000000963F30F098EEA101305934FF0000EA4
:10056000049B68F31F4967F30F0E4FF00008002744
:1005700063F30F0861F30F07059BCDF82C906CF324
:100580001F4E62F31F474FF0000C9DF81820CDF866
:1005900034E06AF31F48CDF830800E978DF83CC0E8
:1005A0008DF83D2043EA00230DF1280883EAC007B7
:1005B000B8E80F003FB287F0C80989EA0919DFF8E7
:1005C00080E084F805C05FFA89F9C7F30727AEE831
:1005D0000F0087EA191747EA092398E8030083EA1E
:1005E000C9031BB283F023074EF8040B87EA0717F1
:1005F000FFB2C3F3072282EA1712704642EA0722CB
:1006000082EAC70720F814190BF1010B4FF0230CF5
:10061000FE211622C82384F87EB1278084F807C003
:100620000EF1020EA170E270A37111E0709E002025
:10063000609E0020CF2A0020344F0020588E0020DA
:10064000302900202A2900206E8E002003082080F7
:1006500010F8013B7B4083EA0313DBB21A0982EAFC
:10066000172242EA032282EAC3031BB29FB27045FB
:100670002780EDD183F0F40383EA0313DBB24FEA62
:10068000131E8EEA172E8EEA032E8EEAC30E0FFA81
:100690008EFE1FFA8EFCCA4FA4F800C04FEA1C2938
:1006A0005FFA8EFE84F81EE084F81F907968BA68BD
:1006B0003868FB6807F5D37CACE80F0038697969C6
:1006C000BA6904F2C518ACE8070004F2A71784F869
:1006D000C59184F8C4E117F8011F3068FEF724FEC5
:1006E000B845F8D194F87231002B41F0DC82B54B5B
:1006F0001B681922980684F8722140F1F482B24BEB
:10070000B24F1B78990741F147863B7D042B8CBF84
:100710004FF003084FF00208FEF71CFC3B8A3A89B1
:100720000A9003EB83035B00ADF842304FF47A701C
:100730003B680C93B7F80EE0397D7B688DF84480F8
:1007400000FB02F24FF0000C4FF0FF300DF12809D2
:10075000ADF840E0CDF82CC00E920D938DF8451009
:100760000F90C846B8E80F00DFF86CE2AEE80F0063
:1007700098E80F00AEE807007246182122F81C39ED
:10078000E17194F87E1184F805C081F0780383EA62
:100790000313D8B2030983F0F60343EA002383EA84
:1007A000C0031BB283EA0310C0B2C3F3072383EA7A
:1007B000101343EA002383EAC0031BB283F0C8008E
:1007C00080EA001C5FFA8CFCC3F3072080EA1C104F
:1007D00040EA0C2080EACC0000B280F0180383EAE3
:1007E000031C5FFA8CFCC0F3072383EA1C1343EA63
:1007F0000C2383EACC03C82001F1010A4FF0FE0864
:100800004FF01E0CA0710EF1020E217184F87EA132
:10081000238084F8028084F803C0184612F8011B74
:10082000414081EA0111C9B20B0983EA102343EA6E
:10083000012383EAC10109B288B272452080EDD15B
:1008400081F0180181EA0111C9B24FEA111B8BEA4C
:10085000102B8BEA012B8BEAC10B0FFA8BFB1FFAD3
:100860008BF3574A23805FFA8BFB1B0A0492059394
:1008700084F8273084F826B0964602F5D37A04F13E
:100880002208DEF80000DEF80410DEF80820DEF8AA
:100890000C30D446ACE80F000EF1100EC645E2460F
:1008A000EFD1DEF80000CCF80000DFF830819DF8D1
:1008B000143084F8CCB108F1260A84F8CD31C3464F
:1008C0001BF8011F3068FEF72FFDDA45F8D1FEF75F
:1008D00041FB3F4B3F4AB3F90410B7F808E03B68CF
:1008E0000B930A907B680C9382FB01274FF47A707C
:1008F000C9174FF0000C00FB0EF0C1EBA701ADF8DB
:100900003CC0ADF83EC0ADF840C0ADF842100D900F
:100910000E90CE46BEE80F002F4F84F805C00FC7DB
:100920009EE807004FF0210C87E807001C23C8222F
:100930004FF0FE0EE370A27184F807C084F802E065
:1009400094F87E11217181F06A0383EA0313DAB20D
:10095000130983F0D50343EA022383EAC2031BB2DF
:1009600083EA0312D2B2C3F3072383EA121343EAE2
:10097000022383EAC2031BB283F0C80282EA021296
:10098000D2B2C3F3072383EA121343EA022383EAB2
:10099000C2031BB283EA0C0282EA0210C0B2C3F3A4
:1009A000072282EA101242EA0022013182EAC002E2
:1009B0000C3784F87E112280A7F11C0110460FE04D
:1009C0002A290020709E0020C69E0020EC5800209E
:1009D000749E00206766666630290020CF2A0020BA
:1009E00011F8013B434083EA0313DBB21A0982EAA0
:1009F000102242EA032282EAC3031BB298B2B94230
:100A00002080EDD183F0680383EA0313DBB24FEA61
:100A1000131B8BEA102282EA032B8BEAC30B0FFA1B
:100A20008BFB1FFA8BF3DA4F23804FEA132C5FFA0C
:100A30008BFB04F1220384F825C084F824B007F569
:100A4000D37A0593FB6838687968BA68D646AEE809
:100A50000F00059B10379F42F246F3D13B88CD4FE4
:100A6000AEF80030C24684F8CAB184F8CBC11AF897
:100A7000011F3068FEF758FC5745F8D194F87EC145
:100A8000C54A84F804C08CF0EB0383EA0313D9B29F
:100A90000B0983F0C50343EA012383EAC1031BB2B8
:100AA00083EA0310C0B2C3F3072181EA101141EABF
:100AB000002181EAC00109B20CCA81F0C80787EAA7
:100AC0000717FFB24FF0000EC1F307210B93CDF8CB
:100AD00030E081EA17130A9299E8070043EA0723F6
:100AE00083EAC7030FFA83F9AC4B84F805E089F079
:100AF000310783E8070087EA0717FFB2C9F3072326
:100B000083EA171343EA072383EAC703277A607A45
:100B1000A27AE17A94F80CE094F811901BB25F404D
:100B200087EA0717FFB2C3F3072383EA171343EAE1
:100B3000072383EAC7031BB2584080EA0010C0B203
:100B4000C3F3072383EA101343EA002383EAC003B5
:100B50001BB25A4082EA0210C0B2C3F3072282EAF3
:100B6000101242EA002282EAC00212B2514081EA27
:100B70000111C9B2C2F3072383EA111343EA012327
:100B800083EAC1031BB28EEA030E8EEA0E1E5FFAE1
:100B90008EFEC3F3072383EA1E1343EA0E23677B0B
:100BA000A07BE17B227C83EACE031BB25F4087EA15
:100BB0000717FFB2C3F3072383EA171343EA072398
:100BC00083EAC7031BB2584080EA0010C0B2C3F3E7
:100BD000072383EA101343EA002383EAC0031BB20E
:100BE000594081EA0111C9B2C3F3072383EA111303
:100BF00043EA012383EAC1031BB25A4082EA02128C
:100C0000D2B2C3F3072383EA121343EA022383EA2F
:100C1000C2031BB289EA030989EA09195FFA89F953
:100C2000C3F3072383EA191343EA092383EAC903B9
:100C3000A17CE27CDFF870911BB2594081EA01117E
:100C4000C9B2C3F3072383EA111343EA012383EAFA
:100C5000C1031BB25A4082EA0212D2B2C3F3072385
:100C600083EA121343EA022383EAC2031BB283F02E
:100C7000270787EA0712D2B2C3F3072787EA1217BA
:100C800047EA022787EAC2073FB20CF10103BAB272
:100C90005FFA87FA4FF0310CFE200C2184F87E3188
:100CA000C8234FEA122E228084F807C0A070E1709A
:100CB000A37184F814A0049F84F815E07968BA68D9
:100CC000FB683868B7F810C0A9E80F0029F803CB13
:100CD00084F8BBE184F8BAA118F8011F3068FEF768
:100CE00023FBC145F8D194F87671002F40F0D687E8
:100CF0002B4B94F87E81B3F90010B3F90220B3F9BD
:100D000004309FED286ADFF89490677107EE103A7F
:100D1000029B1B680A9388F06A0383EA031306EEBA
:100D2000901AD9B20B0983F0D50343EA012383EA71
:100D3000C1031BB283EA03115242C9B207EE902AE3
:100D4000C3F3072383EA111343EA0123F8EEE77A9A
:100D5000F8EEE66AB8EEC77A83EAC1031BB267EE23
:100D6000867A66EE866A27EE067A002083F0C80C43
:100D7000CDED0C7ACDED0B6A8DED0D7A0E900F90C6
:100D800010908CEA0C1E0DF1280A5FFA8EFE0DE021
:100D90002A290020F32A0020E068002030290020C2
:100DA000749E002088C3E43AD02A0020C3F3072CA5
:100DB000BAE80F008CEA1E1C4CEA0E2C8CEACE0C12
:100DC0000FFA8CFCA9E80F008CF01E0E9AE80700C1
:100DD0008EEA0E17FFB2CCF3072E8EEA171E4EEAEC
:100DE000072E89E807008EEAC70E1C21FE274FF068
:100DF000050A4FF01E0CC82208F10103A770E1702C
:100E000084F876A184F807C0A9F11001A27109F154
:100E10000C0784F80480A4F800E084F87E3111F80F
:100E2000013B83EA0E0383EA0313DBB21A0982EA69
:100E30001E2242EA032282EAC3031BB21FFA83FE88
:100E4000B942A4F800E0EAD183F0270383EA031350
:100E5000DBB21A0982EA1E2282EA032282EAC30373
:100E60001BB21FFA83FCDFF8E083A4F800C05FFA2E
:100E700083FE4FEA1C2C84F825C084F824E008F592
:100E8000D37904F1220AD8F80000D8F80410D8F871
:100E90000820D8F80C304F460FC708F11008D0458D
:100EA000B946F0D1DF4FB8F80030A9F8003007F1AB
:100EB000240884F8CAE184F8CBC117F8011F306810
:100EC000FEF732FAB845F8D194F877A1BAF1000FDD
:100ED00040F0DE86D44B1B68052284F877219A0601
:100EE00041F10D80D14BDFEDD26ADA891B8907EE23
:100EF000902A07EE103AF8EEE77AB8EE477A67EEF6
:100F0000A67A94F87EC1CB4BCB4AB3F90410B2F960
:100F10000620CA4FCA48CDED0B7A8CF0220383EA33
:100F200003135FFA83FE4FEA1E1383F0590343EA6B
:100F30000E23B2F5FA6F83EACE031BB2A8BF4FF4BB
:100F4000FA6283EA0318B2F57A7F5FFA88F8C3F38E
:100F5000072EB8BF4FF47A72A2F57A728EEA181E85
:100F6000642303FB02F34EEA082E87FB03278EEA75
:100F7000C80EDA17C2EBA71280FB01300FFA8EF70A
:100F8000CB174FF0000BC3EBA00387F0C8080DF19F
:100F900028098DED0C7AADF83A20ADF83830CDF84F
:100FA00028B0CDF834B0CE4688EA0818BEE80F0065
:100FB0005FFA88F8C7F3072787EA181747EA082770
:100FC00087EAC8089F4FDEF800E084F804C00FC726
:100FD0000FFA88F888F04A0383EA0310C0B2C8F316
:100FE000072383EA10133A460CF1010143EA002378
:100FF00083EAC00342F810E900204FF04A084FF09E
:10100000FE0C4FF0140E84F87E11C821607123800D
:10101000043784F8078084F802C084F803E0A171E3
:10102000184612F8011B414081EA0111C9B20B09AF
:1010300083EA102343EA012383EAC10109B288B29B
:10104000BA422080EDD181F0140181EA0111C9B2C8
:101050004FEA111E8EEA102E8EEA012E8EEAC10E84
:10106000794B0FFA8EFE1FFA8EFC1F464FEA1C2B9F
:101070005FFA8EFE84F81DB084F81CE05968386869
:101080009A68DB68A4F800C007F5D37CACE80F00D1
:1010900038697969B7F818800497ACE8030004F25E
:1010A000A717ACF8008084F8C3B1B84684F8C2E151
:1010B00004F2C31B18F8011F3068FEF735F9C34569
:1010C000F8D1624B624A1B781278013B12F00100A2
:1010D000DBB214BFC0214021172B03D85D4A134453
:1010E00093F80CA05C4B1A8893071ABF002341F0B9
:1010F0001001012312F4027F18BF022312F0100F17
:1011000018BF062312F0200F18BF1023002841F04B
:1011100093804FF0030894F87EC10A938CF0460345
:1011200083EA0313DAB2130983F0920343EA02233A
:1011300083EAC2031BB283EA0310C0B2C3F30722DF
:1011400082EA101242EA002282EAC00212B282F05F
:10115000C80E8EEA0E1E00235FFA8EFE0320C2F335
:1011600007228DF82CA08DF82F8082EA1E128DF8B0
:101170002D308DF82E108DF8300042EA0E2899E8B7
:10118000070088EACE0E0FFA8EF8DFF8B8A0E371F8
:1011900088EA0819AAE803005FFA89F9C8F3072862
:1011A00088EA191848EA092181EAC90994F80880EF
:1011B0008AF800200FFA89F988EA090282EA0218FF
:1011C0005FFA88F8C9F3072282EA181242EA082275
:1011D000607AA17A94F80B90637182EAC80212B225
:1011E000504080EA0010C0B2C2F3072282EA101217
:1011F00042EA002282EAC00212B2514081EA0111A1
:10120000C9B2C2F3072282EA111242EA012282EA3B
:10121000C10212B289EA020989EA09195FFA89F959
:101220001CE000BFCF2A0020709E0020EC58002058
:101230000AD7233C749E00206E8E0020D34D62108E
:1012400067666666302900202A290020687F002012
:101250006090002020FD0308C49E0020C2F30722F6
:1012600082EA191242EA092294F80C80607BA17B81
:1012700084F804C082EAC90212B288EA020888EA45
:1012800008185FFA88F8C2F3072282EA181242EAC5
:10129000082282EAC80212B2504080EA0010C0B2AE
:1012A000C2F3072282EA101242EA002282EAC00256
:1012B00012B2514081EA0111C9B2C2F3072282EA97
:1012C000111242EA012282EAC102E17B94F81090F5
:1012D00013B281EA030282EA0212D2B2C3F30723F5
:1012E00083EA121343EA022383EAC2031BB289EAA8
:1012F000030282EA0212D2B2C3F3072383EA121373
:1013000043EA022383EAC2031BB283F0320282EA79
:101310000212D2B2C3F3072383EA121343EA022371
:1013200083EAC2031BB29AB24FF0FE085FFA83FE53
:101330000920C8210CF1010C84F802804FEA122820
:10134000E070A17184F87EC1228084F8128084F854
:1013500011E0049B186859689A68B3F80CB00AF554
:10136000CC7CACE807000AF5D47A8CF80290ACF893
:1013700000B084F8B88184F8B7E117F8011F30682D
:10138000FDF7D2FFBA45F8D1039BC4F86831FEF7E8
:1013900064BEDFF824A3B84FDFF8209341201AF091
:1013A000C3FCBAF9023087FB0320DB17C3EBA000B4
:1013B00080B21AF09DFCBAF9003087FB0320DB17DE
:1013C000C3EBA00080B21AF093FCBAF9043087FB9B
:1013D0000320DB17C3EBA00080B21AF089FC99F858
:1013E0000010D8F80000FDF79FFF94F860A11AF0F4
:1013F000010700F0E183A14B1B68980672D5A04B52
:10140000A04F1B78990740F1C9863B7D042B8CBF08
:1014100003230223472003931AF086FC38681AF04E
:1014200033FC78681AF030FCB7F80EA0964AD8F86A
:101430000000A2FB0A3ACAF3471A5146FDF774FFAF
:101440003A8999F8001064208AEA010A00FB02F048
:1014500089F800A01AF018FC039B3F7DD8F8000023
:1014600043EA8707FFB23946FDF75EFF99F800307F
:10147000D8F800005F40394689F80070FDF754FF46
:1014800094F860A1BAF1000F2CD1804F4F201AF0D0
:101490004BFC38681AF0F8FB78681AF0F5FB5046F8
:1014A0001AF0F2FB0121D8F80000FDF73DFF744B64
:1014B00099F800201B78D8F8000003F0010782F0AB
:1014C0000102394689F80020FDF72EFF99F8003017
:1014D000D8F800007B40194689F80030FDF724FF5A
:1014E00094F860A16A4AC4F85CB10AF10103DBB266
:1014F000A2FB0312D20802EB8202A3EB420384F8A0
:101500006031FEF78ABD634B63491868FDF7D4FE6E
:1015100000232370FEF729BE604F386800283EF490
:1015200069AD4FF0000ADFF898815D4CAB46554637
:10153000FDF7F6FEF8B1F5B94FF00109AA46386893
:10154000FDF7E6FE83B27E2B00F01A8398F80120A7
:10155000002A49D194F84C11B1B11B2B84F84C21CD
:1015600000F0E8820D2B45D0386888F80190FDF72F
:10157000D7FE0028E3D1AA4650460AAA49495D464B
:1015800025F0F6F9FEF736BD7D2B00F0AE8494F819
:10159000502122B180F02003DBB284F8501194F87E
:1015A0004B21062A10D8B4F84E1138681944A4F813
:1015B0004E11A118013281F8543184F84B21FDF706
:1015C000AFFE0028BBD1D6E7B4F84E2188F80190D1
:1015D00013449BB21A0A52FA83F3FF2BA4F84E313C
:1015E000386802D1304DA3E73868FDF799FE00282E
:1015F000A5D1C0E73868A4F84E21FDF791FE002878
:101600009DD1B8E794F8BC32C4F8B852012B40F22F
:10161000558494F8BD222549981801EB80010132C8
:1016200002F001024E6A84F8BD22BEB1204F0B9732
:101630000DF14809123FA52349F8207D802284F846
:10164000103115232946484684F8112184F81231B7
:10165000B047002840F0B38394F8BC32154A0133F8
:1016600082FB0312A2EBE37202EB42029B1A84F8A4
:10167000BC32FEF702BD00BF67666666709E002042
:10168000C69E0020EC5800201F85EB51E06800202A
:10169000CDCCCCCC04A000202C9F0020D49E0020D8
:1016A00028290020722A00207C2A002020FD03081F
:1016B0004D2A002056555555749E00205468002030
:1016C000200000208F4A904B92F80BE0029AD4F849
:1016D000381110681B888D4A401A4FF47A71DFB2B6
:1016E00001FB0EF11B0A9777177588424FF0000730
:1016F000D37753759770177180F0CD8384498548EF
:101700000B688968DFF828E2834F9EF800E097F8BD
:10171000149080FB03C8DB1780FB010CC817C3EBD8
:10172000A80111770912C0EBAC005177F4214FEA00
:10173000202C7A4B82F82000917601203021D0763F
:1017400082F82210752078211EF0020F82F821C045
:1017500083F81A9082F8230082F8241000F098830E
:10176000D7F800C06E4AD7F804E0DFF8C8B1DFF858
:10177000C88182FB0C014FEAEC7082FB0EA2C0EB29
:10178000A1504FEAEE71C1EBA2520BFB00C10BFB63
:1017900002EB01EB41010BEB4B0B49004FEA4B0B0A
:1017A000039288FB012A88FB0B284FEAA842069285
:1017B000039AB7F80E803F8902EB820202EB8202A5
:1017C00007F5FA7707924FEAAA4ACA17BFB20597F8
:1017D000AAEB02073A464FFA87FA524F00EB800015
:1017E00008EBC80807FB121200EB8000069F4FEAC7
:1017F0008808CDF810800AEB800A4FEAEB78494858
:10180000A7EB080100FB11B003900798464FDFF8E3
:101810001C81DDF814B083F815B049B201EB8001EA
:1018200006910499B9F1050F87FB01074FEADC7CAB
:101830004FEAE179C9EBA71983F809C0039FDFF8E4
:10184000FCC0BDF81810CDF810904FEADE7E88FB82
:1018500002091FFA8AFA88FB070883F80EE04FEAAC
:10186000E770BCF800E0049FDFF8D4C083F80AA05A
:101870004FEAE272C2EB6912C0EB68104FEA1A2914
:101880004FEA1B284FEA112B4FEA222A1A73BCF8A1
:1018900000C083F80B90D97383F810B04FEA202969
:1018A000C7F307214FEA1E2B34BF3222332283F8BD
:1018B0000DA0587483F8129083F81680DF711972A6
:1018C00083F813E083F814B0DA7683F81CC0C4F808
:1018D0003451FEF721BBDFF86C90D9F80000FDF71A
:1018E0000FFD00283EF4A7ABD9F800000121FDF759
:1018F00003FD0222002387F8742088F80030FEF7E9
:101900009ABB00BF846600207C660020A89F002050
:10191000489E002067666666EC580020D49F002031
:101920006BCA5F6B40420F00D34D62101F85EB51B5
:10193000C69E0020806967FF83DE1B43D09E002087
:101940005A8E0020885100205E209047D8F8003041
:1019500002209847FF2019F0E7FE0378FF2B00F0E4
:101960001A8490F901304FEAE3795FFA89F9D8B225
:1019700025F0B2FB484625F0AFFBD8F800305E20DA
:101980009847D8F8003003209847FF2019F0CCFE84
:101990000378FF2B00F0FB83B0F90830D8B2C3F313
:1019A000072925F099FB484625F096FBD34B1B7879
:1019B000042B7DD0DFF880B3B4F82E119BF8002003
:1019C000DFF868A391FBF2F302FB13139BB2BAF8A2
:1019D0000010A4F82E314FEA03191FFA89F9642385
:1019E00003FB01235200B3FBF2F349EA0329C3F3DB
:1019F00003225E20D8F800301FFA89F949EA02096B
:101A00009847D8F80030062098475FFA89F025F00B
:101A100063FB4FEA192025F05FFBB949B4F82E218A
:101A20004B7ABAF800A00132012BA4F82E2100F065
:101A30005E864A7B0AEB8A031FFA83FA002A40F08B
:101A4000F683D8F800305E209847D8F800303A2066
:101A50009847AC4BA3FB0A394FEA59191FFA89FB87
:101A60005FFA8BF025F038FB4FEA1B2025F034FBA2
:101A7000D8F800305E209847D8F800303B209847CF
:101A8000642303FB19A39BB29F48053380FB03200B
:101A9000DB17C3EBA000C0B225F01EFB002025F031
:101AA0001BFBDFF8989299F80630002B40F08A83F0
:101AB0003B689F0600F13A8294F82C31D8F8002058
:101AC000FEF717BADFF878929FED908A4FF0240A5C
:101AD0005E2090475046D8F8003098478C4BF9EC80
:101AE000016A9B8A07EE103AF8EEE66AB8EEC77A0A
:101AF0000AF1010AC6EE877A5FFA8AFA67EE887AF7
:101B0000FDEEE77ACDED027ABDF908B05FFA8BF011
:101B100025F0E2FACBF3072025F0DEFABAF1270F21
:101B200002D0D8F80020D3E794F82C31D8F8002060
:101B3000FEF7DBB93868FDF7F3FB00287FF414AD3E
:101B4000386884F84A9188F80190FDF7E9FB00288D
:101B50007FF4F5AC0FE5FDF7FDF96E4B1B68A0EBCC
:101B6000030B40F6B8339B4500F2B4816A4B1A79F7
:101B70003A2A00F0CD84002388F80030FEF75BBAE3
:101B8000386884F84AA184F84BA184F84C9188F80D
:101B900001A0FDF7C5FB00287FF4D1ACEBE494F87D
:101BA000481194F849315D484A1CFEF70FBA013BD1
:101BB00084F86E31FEF76EBC594B1B88DA0513D4DE
:101BC000D80600F1FD82990600F17C855A0600F1E5
:101BD000A785180700F1A785D90700F1DE8513F066
:101BE000020F0CBF04270C274E4B4F4A1B78D278AC
:101BF00003F001030AB143F00203532003931AF0E8
:101C000093F84A4A128802EB820202EB82029000A9
:101C100080B21AF06DF800201AF06AF8444A45497B
:101C20001288D8F80000C2EBC212520081FB0231C8
:101C300011444FEAE27ACAEB612A5FFA8AFA514606
:101C4000FDF772FB99F80020039BD8F800001F43B2
:101C50008AEA020A002189F800A0FDF765FB3946EF
:101C6000D8F80000FDF760FB99F80030D8F80000C4
:101C70007B40DBB2194689F80030FDF755FB94F83C
:101C800060A1FFF7FFBB013A84F86F21FEF72ABD80
:101C90000AF1FF3A84F877A1FFF776BB013F84F899
:101CA0007671FFF711B9013B84F87231FFF71BB869
:101CB0000024DFF8908027464FF0500A02E0DBB2A4
:101CC00083F3118816F804B0601C5946304419F0AB
:101CD000D9FE002840F023810BF101031C44EFF3EF
:101CE00011838AF31288326E9442E8DB0022DBB261
:101CF000326683F31188FEF7B6BA00BF1080002069
:101D0000846600201F85EB516766666600007A4492
:101D10007C9E00207850002060500020D89E00203B
:101D2000C49E002060900020886800207C6600200F
:101D3000588E00200308208092660020609E0020BC
:101D4000AC9E0020417203084FF0000A5E201F681D
:101D500084F82CA19047D8F80030DFF83093172092
:101D60009847504625F0B8F9BC4BA3FB07239B0BC3
:101D7000A9FB03125209C2EB0212A3EB8203D8B2F1
:101D800025F0AAF9D8F800305E209847D8F800303E
:101D900018209847B24BA3FB07239B09A9FB03120A
:101DA0005209C2EB0212A3EB8203D8B225F094F9D8
:101DB000504625F091F9D8F80020FEF79FB80A9E0A
:101DC000BE4240F2AA843D46002141F2210015F8AE
:101DD000013B81EA03235A0013F4004F80EA020119
:101DE00092B289B208BF11464A0080EA020311F498
:101DF000004F99B293B218BF0B46590013F4004F2D
:101E000080EA010289B292B208BF0A46530012F476
:101E1000004F80EA03019BB289B208BF19464B000C
:101E200011F4004F80EA03029BB292B208BF1A4637
:101E3000530012F4004F80EA03019BB289B208BF3D
:101E400019464B0011F4004F80EA03029BB292B294
:101E500008BF1A46530080EA030112F4004F9BB2F8
:101E600089B208BF1946B542B1D148460CF0CDF948
:101E70007C490A9D7C486D1A152DA8BF15252A4658
:101E80002CF006FB794A94F8BC321570FFF7E6BBDC
:101E90002D22DA761BE5764B02991B780968C4F887
:101EA0003811013B012B3FF629AC10210223917020
:101EB000137123E425F0F2F8FEF790B86D4A02EBB7
:101EC0008302566AFFF7B1BB25F0D8F801233B70B7
:101ED000FEF741B8684AB2F8623100210133A2F836
:101EE000623188F80010FEF7A6B8386884F850917F
:101EF000FDF716FA00287FF422ABFFF73CBBDFEDBD
:101F00005F7AB0EE677AFEF7FCBF0146844607466B
:101F100082460490804605900246FEF7F2BA41469A
:101F20003A2019F00BFD0743FFB2D5E6DFF860A1B8
:101F30009AF80030980700F15782514F4FF000098E
:101F4000CB46D8F800305E209847D8F80030012002
:101F50009847584625F0C0F8484625F0BDF8D8F80F
:101F600000305E209847D8F80030092098470020BC
:101F700025F0B2F8002025F0AFF87B8A97F814908E
:101F8000B3F5967F0AD994F82C2102F00F02072AA4
:101F900004D842F20F79994528BF9946D8F8003005
:101FA000DFF8F0B05E209847D8F800300520984759
:101FB0009BF80830002B00F09183A9F1200307EE75
:101FC000903A9FED307AF8EEE77AF6EE006A67EE27
:101FD000877ABEEE007AF5EEC07AF1EE10FA58BFBD
:101FE000B0EE667A77EE877AFDEEE77ACDED027A8B
:101FF000BDF908905FFA89F025F06EF8C9F3072063
:1020000025F06AF89AF800200023920708930993B4
:1020100000F1CB8094F83031012B00F0C680BBF981
:102020000030DFED196A07EE103ABBF9023007EE17
:10203000903AB8EEC77AF8EEE77A27EE267A67EE9E
:10204000A67ABDEEC77AFDEEE77A0AA88DED0A7A88
:10205000CDED0B7A25F062F82EE500BF73B2E745AF
:10206000D34D6210382A0020404E0020554E0020EB
:102070001080002020FD0308282900200000000017
:10208000EC580020E4380E3F0050C3478988888808
:10209000C69E002084660020C149C24B0093A1F176
:1020A0003F07C14BC14A099101F8404C0AA8C049F9
:1020B00008970CF081F9089F7B1C08933C70089BE3
:1020C0002922591C08911A70089BEA22591C089170
:1020D0001A70089BC822591C08910AA81A702BF084
:1020E00079FA00F101080AA9424608982CF0D0F9C3
:1020F000089A02EB08030133089302F80840089B92
:102100005A1C08921C70089B5A1C08921C70089B51
:102110005A1C08921C70089B5A1C08921C70089B41
:102120005A1C08921C70089B5A1C08921C70089B31
:102130005A1C08921C70089B5A1C08921C70089B21
:102140005A1C08921C70089B5A1C08921C70089B11
:102150005A1C08921C70089B5A1C08921C70089B01
:102160000122991812A808911A7050F8283DDB1B1B
:102170003B7025F04BF88F4B3470C3F8B052FDF72D
:1021800070BFC4F83C5187F80080FDF7E4BE4FF003
:102190000009484605E44846FFF7EABB0123FFF77C
:1021A00039B9FDF7A9F8FDF7EBBE97E80C0001215E
:1021B00008A884F830110892099324F0AFFF7BE45B
:1021C000342711E5D8F80030DFF818A2DFF810B294
:1021D0005E209847D8F8003028209847DAF8003079
:1021E0008BFB032BDB17C3EBAB0B5FFA8BF024F0FD
:1021F00073FFCBF3072024F06FFFD8F800305E2088
:102200009847D8F8003004209847B9F80830002BD8
:1022100040F05B82DAF8083083F310095FFA89F046
:1022200024F05AFFC9F3072024F056FF40E49BF83E
:1022300000309AFBF3FA04E45F4AD278002A0CBF1C
:102240004FF004084FF00508FEF765BF0123D9F8E9
:1022500000003B70FDF75CF80746D9F80000FDF779
:1022600057F87B067DF477AE8A2800F085828E28A9
:102270007DF471AE9AF80030002B7DF488AE4F48A3
:102280004F4B03602D2384F840310768FDF767BE8C
:10229000434B0B93A3F1400900222121A3F13D0AF6
:1022A00003F8402C89F8021089F80120CDF828A005
:1022B00022F06AFB434B444A1B88444900280ABF6A
:1022C00011464FF003084FF004085A0500F121822F
:1022D000D80700F12B8203F002033D4A002B1CBFFC
:1022E0004FF00308114642463A482CF0D1F80AEB69
:1022F000080312A8384A013340F8203D9B1A0022F7
:102300000AF8082089F8013024F080FFFDF753BF58
:10231000234A324B0B920DF14808A2F13D0048F8D8
:10232000200D1988DFF8BC90A2F1400300204FF087
:102330000A0E02F8400C082283F801E040469A7029
:102340000BF03FFFD9F800302549DA1781FB031362
:10235000C2EBA30399B240460BF033FF09F026FC11
:10236000D9F808900A9B4FEA1942591C0A911A7031
:102370000A9B4FEA1922591C0A911A700A9B5A1C8F
:102380000A9283F800900A9B5A1C0A9218704046E1
:1023900024F03CFFFDF70CBF4FF00108FEF7BCB97D
:1023A0002C9F00200EA80020182E0408202E0408C0
:1023B0002C2E04082829002088680020E09E002098
:1023C000A89F0020C49E0020FC2D0408042E0408B1
:1023D000142E0408EF9E0020ED9E00207C66002055
:1023E00067666666489E0020D24FD8F80030DFF856
:1023F00074935E209847D8F8003011209847FA89E6
:102400004FF4F36B0BFB02F289FB0239D217C2EBDC
:1024100069395FFA89F024F05FFEC9F3072024F0E0
:102420005BFED8F800305E2098471920D8F80030BD
:102430009847FB89C04A0BFB03F382FB0301DB17C0
:10244000C3EB611382FB0321DA17C2EB6112642133
:1024500001FB1233D8B224F03FFE002024F03CFEF2
:102460009AF80030B7F8089099077FF567AD5FFAE2
:1024700089FB4FEA192964E5DFF8EC929FEDAF8AFA
:10248000B9F90230AE4A0B9207EE903AF8EEE77ACD
:102490000DF1480867EE887AA2F14003FDEEE77A75
:1024A000A2F13D0148F8201D02F8400C0822CDEDB4
:1024B000027A5A701E229A70BDF8081040460BF03E
:1024C00080FEB9F9003007EE903AF8EEE77A404620
:1024D00067EE887AFDEEE77ACDED027ABDF8081056
:1024E0000BF06FFEB9F9043007EE903AF8EEE77A98
:1024F000404667EE887AFDEEE77ACDED027ABDF8C8
:1025000008100BF05EFE404624F080FEFDF74DBE45
:1025100099780393184615F09DFC00287FF42BABA7
:102520008849894F894A8A4C0988DFF84092936824
:10253000F9611168B4F86221F863C7F86CB0FB6404
:10254000F962D9F80000FA65FBF788F9834600289C
:102550007DF46CAD5146D9F80000FCF7CDFE039B2D
:1025600094F86421DB780493642A4FF0040387F81D
:10257000743040F01C8194F86531DFF8F4A1072B2A
:1025800008BF84F865B194F86521069207EB021B39
:10259000DBF80410059108462BF01CF8DBF8083036
:1025A00003935FFA80FB18462BF014F8C3B20BEBD1
:1025B0000300069A0599059308308AF8070022F06F
:1025C0000F008AF80A0002F00F0203EBCB008AF832
:1025D0000D208AF80E005A460AF10F002BF058FF22
:1025E000059B03990BF109001A460AF106031844EA
:1025F0002BF04EFF9AF8073003F1010BD3B1013BEA
:102600005FFA83FC0CF1080CDFF868E1D4440AF1AE
:102610000700002310F8011B59408B00CA0883EA09
:10262000410302F018024B404EFA02F25340844537
:10263000DBB2EFD1474A04980BF802302BF004FFCD
:1026400094F865310022013384F8653184F86421FF
:102650009AF802305BB11AF80610D9F80000FCF7BE
:1026600063FE01369AF80230F6B2B342F3D894F81A
:1026700064310322013384F8643187F8742088F8C8
:102680000020FFF72AB92F4B334A1B88927903EBBE
:10269000830303EB83034FEA83081FFA88F8002AB9
:1026A00000F01581294B1B680FFA83FA09F07EFAB6
:1026B00040B2FDF72ABE1146944617469246049250
:1026C000FDF71FBF2427FFF78FBA09F06FFA24F038
:1026D00003FD002024F000FDFFF7EAB95FFA89F05E
:1026E00024F0FAFC4FEA192024F0F6FC8AE4D8F82A
:1026F00000305E209847D8F80030392098475FFABC
:102700008AF024F0E9FC4FEA1A2024F0E5FCFFF7F8
:10271000C8B94FF003081149E5E50021FFF7A5BB53
:102720001027FFF761BA2027FFF75EBA0C494FF078
:102730000408D8E5EC5800201F85EB5158A08B41C8
:102740002C9F00207C66002020000020489E002056
:10275000282900200A590020609E0020082E040825
:102760000C2E040889B5F814749E002088510020AE
:10277000045900200007090E614B1B689F067DF578
:10278000EAAB9AF80030002B7DF401AC5D485E4B5B
:1027900003602D2384F8403177E50827FFF724BA3A
:1027A0005A4B8046B3F900A06420FDF7AEBD97F800
:1027B0007530DFF868A1564905961A0704BF013342
:1027C000DBB2072B28BF01234FEA031B07EB0B02E9
:1027D000107C00228AF80A2011F800C05FFA8BF200
:1027E00003920AF10D02039E07EB0B013043BCF18B
:1027F000010F1070C96802F101000ED9ACF1020698
:10280000F6B206F1020E9644024602F8011B72452A
:102810004FEA1121F9D101363044BB4421F0600266
:1028200001339BF81110DBB20A43082B027000F150
:1028300001024FD04FEA031B07EB0B00344E007C24
:10284000344916F800C0039E511A06F1100E01EB30
:102850000C0606965FFA8EF60396069E132EC2DDD0
:10286000059EDFF8BCE0C9B28A1DD2B242F040003A
:102870008AF8070002F1010BCAB14A1DD2B2083230
:10288000524403920EF1010C00221CF8010B50403F
:10289000820082EA4002C10842401F4801F018014C
:1028A00040FA01F14A4003996145D2B2EDD1049852
:1028B0000BF80E2087F875302BF0C6FDC8E61146E0
:1028C00094461746924604929046FDF71ABE4FF082
:1028D000FF33E9E60F49059E511AC2E71146FDF79D
:1028E00010BE11469446FDF70CBE1146944617469D
:1028F000FDF707BE1146944617469246FDF701BE06
:10290000709E0020E09E0020D49F0020489E002062
:1029100020FD0308115900200007090E045900206A
:102920000A5900202DE9F04F2DED068BB54BB64A24
:102930001C7891B000F59C41203101900691116006
:10294000002C00F09F86B14A01991268914240F232
:10295000E680AF4AAF491668DFF800930292013C67
:102960001C70AD4B009106F480560493002E40F08D
:10297000E480AA4B1B78022B01F00181042B01F0AB
:102980006B81012B01F01F81A54B019A9A42049B98
:102990009B7800F24C85002B40F04D85A14B0393B2
:1029A000029B1E6816F4805740F03A86DFF8B0A20A
:1029B000009BB9F906205D8BAA42B4BF0025012512
:1029C000994B1B68D80040F1C280039B1B7813F021
:1029D000010300F0C3800099498C914241F3C58105
:1029E000002D40F0C280914C94F88C20002A40F0D9
:1029F000BC808F4A8F49106890F82D0000220A6031
:102A00004A608A608C4A002840F0B0801070002B29
:102A100040F0B180894B1A78002A40F0DF8000999D
:102A2000B9F90070488B898BB9F902408742CCBF55
:102A30008026002646F040038F42A8BF33469B08FD
:102A400043F080068442C8BF334643F040068C42C0
:102A5000B8BF33469B08B9F90440B9F9066043F0A2
:102A600080078442C8BF3B4643F040078C42B8BF52
:102A70003B469B0843F080076C4C8642C8BF3B46F0
:102A800043F0400794F88EE08E42B8BF3B469E4527
:102A900001F0E383A4F8902084F89220684984F838
:102AA0008E300E78002E01F0DF825F2B01F08F83D5
:102AB0006F2B00F08B80039B1B78D90700F18E8071
:102AC00094F89210002940F08980B4F99030322BAC
:102AD00040F3848094F88E300120572B84F89200C4
:102AE00001F02987029A1268560741F126825A2B73
:102AF00041F0238294F89430002B42F0C58094F882
:102B0000963083F0010384F89630002B42F0248144
:102B10000C202AF079F9029B4A4E1B6861E03C4B7D
:102B200002931E683B4A3C4B009206F48056DFF845
:102B30002C910493002E3FF41CAF00213A480CF076
:102B400046F800287FF415AF25F0D8F911E7710297
:102B50003FF53BAF039B1B7803F00103334C00228E
:102B600084F88C20002D3FF444AF334A01211170CA
:102B7000002B3FF44FAFF2067FF54CAF324B1B7882
:102B8000DB063FF547AF002F7FF444AF21F0FCFE9A
:102B900000287FF43FAF2A4B1B78002B02F07B808C
:102BA0002A4B9B78002D42F0E6803BB1284A294B06
:102BB00012681B689B1A002BC2F2D68010201B4C97
:102BC0002AF022F9012384F88D3023E7B2F5FA7F49
:102BD00004DB94F89220002A01F00E84029B1B680B
:102BE000184E580700F19B870EAB1B4F00225A600E
:102BF0003D460E9240F6330B4FF0190840F28334F5
:102C000033E000BF84500020484F00208050002057
:102C1000ECB00020FC9C0020886800209C4900202B
:102C2000404B4C0060900020A87D0020EC2B002041
:102C3000C89E0020387D00206C2E0020D754002034
:102C40007D220020C49E0020C69E0020587F0020C8
:102C5000E4A700202CA10020EC5000206E8E002064
:102C60003C5100200435AA4522D0A978EA78914247
:102C700018FB0140F6D26978043118FB024239F999
:102C800011105945A8BF5946B1F5617FB8BF4FF43F
:102C900061718142E6DD9142E4DC29782729E1D89F
:102CA0001846043501930BF083FFAA45019BDCD144
:102CB000CB4A93E803001378CA4A82E80300002B4A
:102CC00040F09386C84B1A78002A00F00286C74B62
:102CD0000193C44801210BF07AFF002840F0938251
:102CE000049BDB78002B40F08E82C14C328822F0AE
:102CF00001039BB29A42338009D0BE4B02201421BB
:102D0000FF2218700E2059709A702AF07DF8022167
:102D1000B4480BF05CFF002800F02587012008F084
:102D2000A1FB33889A0741F1028113F0030FB24BE4
:102D3000B24A19785068069308BF81F00201C1F3C6
:102D400040010592FCF72EFD2421A6480BF03FFF21
:102D500030B9039A1378580744BF23F00403137063
:102D6000236813F00A0F1DD005219E480BF02FFF9A
:102D7000002800F0E0873388590741F1948106214B
:102D800098480BF024FF002800F0D08733885A06BB
:102D900041F17781072193480BF019FF002840F09B
:102DA0006C8723689B0600F16786B6F800B0DFF8F1
:102DB00080828C480C210BF00AFF002800F0E8828A
:102DC0004BF480735B45338009D08A4B0222142177
:102DD0001A700E20FF2259709A702AF015F8884B4D
:102DE0001B78082B00F0E0820E2B00F0DD82029BA6
:102DF0001C68600511D5834B1B79002B00F0E58121
:102E0000142178480BF0E3FE002840F0E38124F021
:102E100057FA09F011FC029B1C68039B93F800B061
:102E2000794B1BF0010B00F02A8201221A70019BE2
:102E3000B9F906101B6875485A894FF0010E914286
:102E400080F800E080F20182714B4FF07E521A60F0
:102E5000704A009BB9F900E0B3F818A092F9043069
:102E6000107892F801C0002BAEEB0A0314BF0122C8
:102E70004FF0FF32002BB8BF5B42B3F5FA7FA8BF1B
:102E80004FF4FA73984280F2DD811B1A07EE903AF4
:102E9000F8EEE77AF245C8ED007A03DDF1EE677AE5
:102EA000C8ED007AB9F902E0AEEB0A03002BB8BF17
:102EB0005B42B3F5FA7FA8BF4FF4FA73984280F2F1
:102EC000BE811B1A07EE903AF8EEE77AF245C8ED9C
:102ED000017A03DDF1EE677AC8ED017AB9F90400F1
:102EE000A0EB0A03002BB8BF5B42B3F5FA7FA8BF83
:102EF0004FF4FA736345CCBFA3EB0C03002302FB32
:102F000003F307EE903AF8EEE77A5045C8ED027AFF
:102F1000BCBFF1EE677AC8ED027A14F4805400F079
:102F20005682B1F5FA6F3C4BA8BF4FF4FA61B1F588
:102F30007A7F1A78B8BF4FF47A71A1F57A71002AB6
:102F400041F01781354ADFF8ECE082FB0130CB1706
:102F5000C3EB6013581C6FF0630C3EF910003EF990
:102F600013E00CFB0313A0EB0E0003FB00F382FB4A
:102F70000312DB17C3EB62139E440FFA8EFE07EEBB
:102F800090EAB8EEE78A88ED038A002C40F0878546
:102F900033885A0640F10E812149224A91ED018A77
:102FA000D2ED019A92ED026A91ED034A92ED030A85
:102FB00091ED029A92ED007AD1ED005AD8ED011A06
:102FC00098ED002A184A194938EE445A79EEC63A63
:102FD00077EE007A65EE233A75EEC96A2EE000BFFF
:102FE00068550020A87D002080540020CC9E002041
:102FF000709E0020C8480020ACA70020B0A7002089
:10300000687F00208466002061900020A42E0020AC
:103010001C2E0020307F0020C42F00201F85EB5184
:10302000C8060020F801002030020020EC2B002010
:1030300094660020689600200000000075EE890A62
:1030400037EE401A66EEA76AB0EE633AA0EE813A18
:1030500013F00303B0EE665A78EE044A79EE867AEE
:10306000A0EE815AF0EE638AA4EEA73AD4EEA78AC6
:10307000A4EEE75A33EE263AF0EE687AF0EE674AAD
:10308000F6EE008A35EE88AAE0EEC14A28EEC33A91
:1030900035EE635A77EE293A77EEE67AAAEE233ACE
:1030A00025EE285A76EE403A34EE49AAE0EE817ACF
:1030B00074EEA64AAAEE235A34EE094A37EE697A2C
:1030C00064EEA84A63EE036AE4EE074A75EEC85A56
:1030D00036EE006A67EEA87AB0EE667A95EE057A6B
:1030E000E5EE056AE5EE867AB1EE648AF0EE665AA0
:1030F000F0EE476AB1EE674AE8EE246A63EE270A0B
:1031000067EEA43AE4EE275AB1EE450AB0EE606AE3
:10311000B0EE631AA4EE277A23EE244AE7EEA76AFC
:10312000A5EE246AA0EE031AE8EE245AB0EE448A13
:1031300031EEA19AE0EE240AA5EE278A66EEA16A96
:1031400072EE028AE5EE033A61EE211A26EE096A72
:10315000A4EEA47AA0EE274A0CBFD8ED022A5FEDB8
:103160004A2A82ED005AA2EE256AE8EEA06AE2EE53
:10317000081A73EEA33A27EE227A34EE044AF0EEF0
:10318000005AE3EEA26AA4EE226AA1EEA57AC8ED87
:10319000016AC1ED376A81ED366A88ED006A81ED1A
:1031A000387A82ED013AC2ED027AC2ED034A0BB9D8
:1031B00088ED027ABBF1000F40F02C812AF052F822
:1031C00011B0BDEC068BBDE8F08F039B1B78D907CF
:1031D0007FF51DAE4FF40F7017F0CAF900283FF4C9
:1031E0001AAE09F03FF84FF40F7017F06DF9002890
:1031F0003FF411AE09F036F84FF40F7017F064F990
:103200000028EED107E69D4C236898077FF56EAD48
:103210003388D90740F1F48723F0020292B29A4230
:1032200032803FF482AD964B022018701421FF22A9
:103230000E2059709A7029F0E7FD338875E5DFEDAF
:10324000917A43E6DFED8F7A24E6B1F5FA6F80F2EA
:103250008D84187A8B1A03FB00F3C2F5FA6293FB94
:10326000F2F3C3F1640307EE903AF8EEE77A9FEDCC
:10327000867A864B67EE877AC3ED007AE8E51B789D
:103280000393002B7FF4D3AD814A1268002A3FF4E8
:10329000CEAD804A804B12F8030C1B780792114682
:1032A000A2F1030A029321F045FB079A002800F0DF
:1032B000B185029A039B002A59D10AF108019AF8B4
:1032C000050021F037FB002841F0C48473499AF8C7
:1032D0000A0021F02FFB002800F0B185029B022B91
:1032E00041F0B4846E499AF80F0021F023FB0028C6
:1032F00041F0C0846B499AF8140021F01BFB0028B0
:1033000000F0B185029B042B41F0B08466499AF825
:10331000190021F00FFB002841F0A48463499AF8BA
:103320001E0021F007FB002800F0B185029B062B50
:1033300041F094845E499AF8230021F0FBFA0028BA
:1033400041F070845B499AF8280021F0F3FA0028D4
:1033500000F0B185029B082B41F0608456499AF831
:103360002D0021F0E7FA00283FF461AD09231A4649
:1033700002EB82029244DFF85CE1474A9AF80100CE
:103380009AF8021013708EF800008EF801104EE5C6
:103390002BF480739BB25B4533807FF416AD474BB3
:1033A0001B78082B7FF420AD328822F040039BB2BB
:1033B0009A4233803FF41BAD314B022214211A7024
:1033C0000E20FF2259709A7029F01EFD0FE5009B18
:1033D0005A8B9142C0F2D183B1F5FA6FD4BFC2EBE0
:1033E0000101C2F5FA614FF47A7303FB01F134482D
:1033F0000378C2F5FA62B1FBF2F1002B3FF4A2AD03
:103400004378304A01FB03F182FB0123C917C1EB6A
:10341000631197E5069B1978059B01F00101186877
:10342000FCF7C0F911B0BDEC068BBDE8F08F13B905
:10343000049A01239370244B049A1D7892F821403A
:1034400003931B2021F0AEFA012C05F001088246FF
:1034500000F0DC8605F00205049A1C4E92F820303C
:103460001B4F01959346052B00F23587DFE813F0DB
:10347000BD00B3003400FB00FD00F000709E002092
:10348000C8480020000000000AD7233C1C2E002062
:10349000649000208E48002096000020984800206C
:1034A0009D480020A2480020A7480020AC480020EA
:1034B000B1480020B6480020BB480020687F0020AB
:1034C000C42F00201F85EB516090002060960020E3
:1034D000C09E002068900020012C04BF05238BF8BB
:1034E0002030B8F1000F13D0009B3088B3F91810CA
:1034F0000022134661F30F0361F31F4361F30F02D0
:1035000060F31F42C9F800300323C9F80420019377
:103510007C4DDBF814102A68914280F0958547F2C3
:1035200030510322CBF81C108BF82020022007F02A
:10353000C9FF24F0E3FC2968DBF81C200A440421BD
:10354000CBF818208BF82010012C40F015872A6842
:10355000DBF81810914280F0BE866B4B187820B9CA
:1035600021F020FA002840F0B6863A6822F00202E4
:103570003A602A687388642101FB03234FF480605A
:103580000022CBF810308BF820208BF8032007F0B6
:1035900069FF9BF8203066E721F00AFA012807D17D
:1035A000584D72882B68642101FB0233CBF8103030
:1035B000BAF1000F02D0B379002B4BD1012C00F0EF
:1035C0008A86504DDBF810102A689142C0F0C986F7
:1035D00001238BF82030012C3AD0F379012B46D00F
:1035E00021F066F99BF820303DE7B8F1000FD3D108
:1035F000019D4FF48060BAF1000F00F03B8307F0AB
:1036000049FF049A00231361002D3FF4C9A92846FD
:1036100029F0FAFB029B1E6816F480573FF4C6A9F6
:103620001D213A480BF0D3FA00287FF4BFA9384B8C
:1036300003F1500A03E004339A4500F052861A78E9
:10364000262AF8D19978DA789142F4D2FFF7B0B906
:103650002C4D8EE721F02CF903224FF47A738BF86E
:103660002020CBF81C30274D60E7264D6CE721F079
:103670001FF9032240F6B8338BF82020CBF81C301A
:10368000204D53E7234F3B78002B4DD0DFF88C8043
:10369000DFF88CB0204BDFF88CA0009345465E46E7
:1036A0004FF47A790DE0009A115D9847032C26DCDF
:1036B00080B93B782AF8020F01349C4205F10405D9
:1036C00034DA072CE1B23046DBF80430EBDD984702
:1036D00000B2EEE738F824206B88801A9B1A09FBA9
:1036E00000F040F6CA0290FBF3F000F57A709042C9
:1036F00040F2EE23A8BF10469842B8BF184600B269
:10370000D7E700BFE4A700207D220020A87D00208D
:10371000EC500020B0510020FC9C0020C45100203F
:10372000344F0020EA2B0020BC4A0092BC4A02928F
:10373000BC491268019842F2010AA1FB001B12EA7F
:103740000A0A4FEA9B1B00F00D83B74DB748B84CEF
:10375000B8492E780078267008701EB1B5490E78E9
:1037600086F00106B44C0F2184F82410002B00F0E1
:10377000DF84B24B009D0B93B5F826C0B5F824E06A
:10378000009DCDF820C018462D8B0078AC4B0C95D1
:1037900094F825500495A3FB00535B0803EB430307
:1037A000C31ADBB202F48052079397F80080DFF867
:1037B000A092DFF8B4C20A900BF59673099104F158
:1037C0002800CDF80CA00D92DDF810A0059304940C
:1037D00000217446002E00F0D683049B33F911209B
:1037E0001FFA82FEA6454FEA410303D3089DAE456A
:1037F00040F20E845CF82120934580F0CD8339F9A6
:103800000320039D002D40F0E1830131414529F85B
:10381000032000F10600DDDB099A049C894B84F843
:1038200024200F2A0CBF0122002284F825A01A7040
:1038300000F08584844B7D497E4ADFF81CB20493F6
:103840001C46042001230B70137007F03BFEDBF8CD
:103850000030A1686268E3605B1A934284BF002372
:1038600084F82130029B3C781E68002C01F0CB804C
:10387000009A764DB2F824E0178B754916F48056FD
:10388000284640F0868432460EE0437803EB8303FB
:1038900003EB830303F2EE239BB20132944221F83F
:1038A000023B00F102000ED015F81230002B00F0A0
:1038B000B483022BE9D001320B8821F8023B9442F9
:1038C00000F10200F0D10B9A137801331370FFF767
:1038D0004DB8DFF898B1DFF898A1574C01920BF181
:1038E0005A0859461BF8010C21F024F810B39BF834
:1038F00004009BF802309BF803E000EB400104EB6E
:103900008101013BD1F8A02003EB430353449342D0
:1039100010D094F8CC2081F89CE04FF0010E0EFA04
:1039200000F022EA0000C1F8A030019BC1F8A430E9
:1039300084F8CC000BF1060BC345D2D1454B464A67
:10394000019319463A4B126809681B78DFF824B1D5
:103950000695089105934FF0FF384FF0000A154681
:103960000796DBF80420002A34D0167896B3DBF8EB
:103970000810691A002911DB2F4C05F5FA7394F829
:10398000CC10CBF80830012000FA0AF0334B21EAC2
:1039900000014FF0FF3084F8CC101860059BCBB1CC
:1039A0009BF8001050780431C9B2002840F016820C
:1039B000009B39F91110188B00F1C804A14240F3A3
:1039C000A1841D4C917894F8CC2042FA0AF2D207D7
:1039D00040F155850AF1010ABAF1040F0BF10C0B05
:1039E000BFD1069D079EFFF774B91D4B03E004335A
:1039F0009D423FF467A919782329F8D19878DA789D
:103A00009042F4D217480BF0E2F800283FF45AA98C
:103A1000142029F0F9F9FFF755B900BFFC9C0020EC
:103A2000ECB00020D34D6210104F0020E4000020C5
:103A30007D680020E5000020EC2B0020A150002034
:103A4000ABAAAAAAB07D002088680020F851002007
:103A50006E8E0020CC9E0020E4A70020E401002010
:103A6000EC500020A87D0020A4500020A547002095
:103A700054FD0308882C0020BF4B1B789C0704D5FD
:103A8000BE4C237D042B00F28484B6F800B01BF0FA
:103A9000300F40F01E82DFF83C83FFF78AB91D210A
:103AA000B7480BF094F820B1EFE30437AF423FF48E
:103AB0006FAA39782629F8D1BA78FB789A42F4D2DD
:103AC000049BDB78002B7FF463AAAD480BF07FF8F2
:103AD000DFEDAC7A002800F0AD8738EE678AAA4A9D
:103AE000AA49FDEEC87ACDED007ABDF900301B037E
:103AF00082FB0302DB17C3EBA212CAF57A731BB277
:103B000003FB02F343F30F33534407EE903AF8EE0E
:103B1000E77A0123C8ED037A0B70FFF739BA9C4CA2
:103B200094F8963053B1039B1B78D90706D5009BB8
:103B3000B9F906205B8B9A4200F3908411219048DA
:103B40000BF045F8002800F0FB8094F89A302BB970
:103B500094F8943013B93223A4F89830012384F8F0
:103B60009A30FFF741B83388FFF756BB1B7AC3F191
:103B7000640307EE903AFFF778BB214637E4009ADA
:103B8000537DD27D013B39F913301AB1C3F53B6344
:103B900008331BB2A3F57A7307EE903A9FED7D7A56
:103BA0007D4AF8EEE77A40F2FF3167EE877AFCEE65
:103BB000E77ACDED037ABDF80C308B4228BF0B4677
:103BC0001380FEF7E1BE724C019AD4F88830D31A04
:103BD000002BFEF6D9AE714A714B527C009933F836
:103BE00012308A7DDFED6F6A9FED6F6AC97D9BB2EF
:103BF00007EE102A07EE903AB8EEC77AF8EEE77AA9
:103C000027EE267A67EE867A069AC4F88820C7EEF1
:103C1000876A40F2FF32FCEEE67ACDED037ABDF81A
:103C20000C30934228BF134609B1D31A9BB25F48A8
:103C30005F4D01785F4C35F81160226825F811302E
:103C4000921B13440131544D236001F00F021B09F4
:103C500002702B80FEF798BEFBF77CF9564B574A53
:103C60001B68C31A93427EF78FAE4B4B00221A801B
:103C7000FEF78ABE07F0F6FBC3E4514AB2F9003002
:103C8000002BB8BF5B42B3F5E17FBFF68AA8B2F95B
:103C90000230002BB8BF5B42B3F5E17FBFF681A8CD
:103CA000484B93ED057AD3ED077AD3ED096A93ED8E
:103CB000030A77EEA67A30EE070AF7EE000AB0EEB6
:103CC000007AE7EEC70A30EE000A0AF0CDFCB6EE45
:103CD000008A20EE488A9FED3C0A38EE000AFDEE8D
:103CE000C07A17EE903A2033402B40F2C5839FED07
:103CF000370ADFF8E480DFED357A88ED000ABDEEA3
:103D0000C87AC8ED017A17EE103A2033402BC8ED7F
:103D1000027A00F24386B0EE480A0AF02BFC0A2031
:103D200088ED030A29F070F8FFF73BB8402007F050
:103D300099FBFFF72FB8042007F094FBFFF71FB89B
:103D400094F89430002B3EF44FAF039B1B7813F094
:103D500001037EF449AF012284F8943084F8952061
:103D6000FEF742BF1A490E78F7E4094C012284F8A5
:103D70008C20FEF7FABE00BFC69E0020EC58002043
:103D8000A87D002000007A44D34D6210982E0020B8
:103D9000EC2B00206F12833F588E002084A7002058
:103DA000A4A700200000C842000080449D490020D4
:103DB000A4490020A0490020C828002060E3160084
:103DC000749E002008020020DB0FC93F00000000A5
:103DD0007D68002094660020C8060020012800F0BD
:103DE0006585B8F1FF3FB94C0BD012780C2A08D08A
:103DF000B74BB84A03EB8603C2F80080B64A5B6C47
:103E0000136094F8CC20012303FA0AF3134384F8D7
:103E1000CC30DFE5511D9AF8050020F08BFD00281D
:103E20003FF454AA029B012B40F014870AF10D01C4
:103E30009AF80A0020F07EFD002840F00787A74985
:103E40009AF80F0020F076FD00283FF453AA029B59
:103E5000032B40F00F87A2499AF8140020F06AFD66
:103E6000002840F003879F499AF8190020F062FD6E
:103E700000283FF453AA029B052B40F0F3869A4991
:103E80009AF81E0020F056FD002840F0E78697497A
:103E90009AF8230020F04EFD00283FF453AA029B1D
:103EA000072B40F0BF8692499AF8280020F042FD87
:103EB000002840F0B3868F499AF82D0020F03AFD93
:103EC00000283EF4B4AF029B092B3EF4B0AFFFF7DD
:103ED0004DBA102007F0C6FA202007F0C3FA864B2F
:103EE000B6F800B0DFF8448200221A708349844A91
:103EF000844C854800230B60844923604FF0000EFA
:103F0000036053609361C2F800E0C2F808E0C2F8B1
:103F100014E0C2F81CE0C1F800E04B60C1F808E012
:103F2000C1F814E08B61C1F81CE0FEF742BF02202B
:103F300007F0B0FA3388FEF7F8BE5D2B00F0A582DB
:103F40005B2B00F064855E2B00F0E785562B00F0BC
:103F50000886972B00F06A86A72B00F0E2856C4E4E
:103F60003288950740F0AA85A3F1B702072A00F22C
:103F7000B682DFE812F0AD02B402B402B4029F02CE
:103F8000B4029802A602002C40D05CF82120934590
:103F90004FEA4103FFF433AC5E4A5E4DD25C05EB61
:103FA000030E002A00F0E880022A4AD19EF8012080
:103FB00002EB820202EB820202F2EE2292B20329AB
:103FC00035DD039D12B2002D3FF41FAC079D20F894
:103FD0001520BAF1000F03D10A9D022D7FF615AC12
:103FE000B0F800A04288B0F804E0524496444A4A2F
:103FF0000FFA8EFE82FB0E52484DA2EBEE7225F8B0
:1040000003E012B24FF0010AFFF7FFBB22464B005C
:10401000059D4CF82150FFF7F4BBD3B2022B04D915
:10402000032B7FF448AC734637E43B4635E4012567
:1040300005FA01FE099D25EA0E0512B20995FFF762
:10404000E0BB39F80320BAE7354A1278002A7FF43A
:1040500066AAB8F1000F3FF462AA012C40F03B8140
:104060009BF82030FFF7FFB931462E480AF0AFFD2C
:10407000002800F0CE8084F8936024F003FAFEF765
:104080001ABD43F04002934232803EF483AE264B89
:10409000022214211A700E20FF2259709A7028F003
:1040A000B3FEFEF777BE43F00402934232803EF443
:1040B00066AE1D4B022214211A700E20FF22597089
:1040C0009A7028F0A1FEFEF75ABE00BFEC2B00202C
:1040D00054FD0308E4010020988E00209D48002034
:1040E000A2480020A7480020AC480020B14800208A
:1040F000B6480020BB4800200A690020F46900206F
:10410000A4690020402E0020002F0020CC69002050
:10411000C49E0020F8510020565555555C2C0020B7
:104120005C2E0020A87D0020C84800209466002056
:10413000BA4ABB4B0B92DFF8189301221A701B216D
:10414000B8480AF044FD00287FF474ABB64BDFF8A2
:1041500004B304931946DBF80030CA688B609B1ADD
:10416000C82B00F25884029B1E6806F48056FFF7A5
:10417000AABB5B78FFF745B9CAB2022A40F2938323
:10418000032A7FF45EAF0C9A0D9D002D08BF2246D6
:1041900015E700220FE0437803EB830303EB83036F
:1041A00003F2EE239BB20132A24221F8023B00F15E
:1041B00002003FF488AB15F812301BB1022BEAD095
:1041C0000B88F0E7D3B2032BFAD83B46EBE7B2F506
:1041D000FA7FFEF603AD94F89230002B7EF4FEAC2D
:1041E000039B1B78012213EA020584F8922000F059
:1041F000C68323F083FE029B8C4E1B68FEF7F1BC46
:10420000012007F047F93388FFF706B80025FFF7CC
:1042100023B9039B864A1B781060DE077EF550ACFD
:10422000844B1B78002B3EF4D9AC049BDB78002B2D
:104230007EF4D4AC94F893300133DBB2032B84F8D2
:1042400093307EF6CBAC7C4B5B7813B9002D7EF4BB
:10425000C5AC23F053FEFEF72EBC784A78491068AF
:10426000B4F99020C66981FB06018911F617701A0E
:1042700000F5FF407F3082423EF710AC891B0A44B4
:1042800012B2A4F89020FEF709BC049BDB78002B47
:104290007FF40FACDFED6B7A694938EE678ACAF5B7
:1042A000FA63FDEEC87A1BB2CDED007ABDF90020AD
:1042B000120381FB0201D217C2EBA11203FB02F32E
:1042C00043F30F33534407EE903AB8EEE78A88ED94
:1042D000038AFFF7EEBB019D002D3EF461ABFFF7B3
:1042E00096B9594A009BD5881B8BB9F90620591BF2
:1042F0008A4240F390802B449A42B4BF00250125A6
:10430000FEF75EBBC8388142504C66DA917894F86B
:10431000CC2042FA0AF2D3073FF55CAB4B420120B6
:10432000099328F07BFE721E099B162A00F2A383D4
:10433000DFE812F08702A002EF01C201AE018101A5
:10434000560166024C0232020C02A103C201850230
:104350008101560166027D0281023D0128010F01A3
:10436000F70020F0A5FA032140F6B8328BF82010B0
:10437000CBF81C20FFF7DAB8AB460499DBF8002035
:10438000CB69019D13448B61002D3EF409ABFFF70F
:104390003EB90A2020F006FBB6F800B0824600289D
:1043A00000F000831BF0100F00F0E183274C94F81D
:1043B000D4A0BAF1000F7FF46EABDFF89C800D2023
:1043C00028F022FD012384F8D430B6F800B0BAF109
:1043D000000F7FF48BADFEF7ECBC94F8CC300122DB
:1043E00002FA0AF223EA020305F5FA7284F8CC30E5
:1043F000CBF80820FFF7EEBA039B1B780121D80702
:1044000084F8921000F1F38224F03CF8029B074EEE
:104410001B68FEF7E6BB0125FEF7D2BAA1500020CB
:10442000B07D0020A87D002088680020C49E002068
:1044300030A100207D680020587F0020ACA0002023
:10444000D34D621000007A4448960020EC2B0020E7
:104450006E8E0020E4A70020946600200021C8484A
:104460000AF0B5FB00287FF469AB322384F896008C
:10447000A4F89830FFF762BB0AF07CF839E40B46E9
:1044800000290CBF012002204AE7BE4B0022012078
:10449000BD49BE4C0B60227028F0C0FD029BBC4E93
:1044A0001B68FEF79EBB032024F0C0FC029B1B6828
:1044B000FEF797BB002024F0B9FC029B1B68FEF7B7
:1044C00090BB022024F0B2FC029B1B68FEF789BB64
:1044D000012024F0ABFC029B1B68FEF782BB9E2BE5
:1044E00000F01C849D2B00F01184AE2B00F006849C
:1044F000AD2B00F0FB83EF2B00F0F583FD2B00F0DC
:10450000E283FB2B00F02584FE2B00F01F84F72BA9
:1045100000F019847B2B00F0B183029B1B68FEF72F
:1045200060BBD4F8D0009B4A90F8368092789844CB
:10453000B8F1640FA8BF4FF0640828EAE87880F863
:104540003680002A40F022841FF020FBDBF8042094
:104550004BE4D4F8D0008F4A90F837809278984492
:10456000B8F1FE0FA8BF4FF0FE0828EAE87880F8FF
:104570003780002AE8D01620414620F05DFAD4F8B2
:10458000D000E1E70899834A91F801809844B8F592
:10459000967FA8BF4FF4967828EAE87881F80180E2
:1045A0009278002A40F0F783D4F8D000CCE7D4F812
:1045B000D000784A90F802809844B8F1C80FA8BF9C
:1045C0004FF0C80828EAE87880F802809278002A3C
:1045D000BAD01420414620F02FFAD4F8D000B3E727
:1045E000D4F8D0006B4A90F8048091789844B8F1E0
:1045F000C80FA8BF4FF0C80828EAE87880F8048000
:10460000002940F0DB83102E9ED090F80180984462
:10461000B8F1C80FA8BF4FF0C80828EAE87880F8BA
:1046200001809278002A8FD01320414620F004FAAE
:10463000D4F8D00088E7D4F8D000564A90F8038028
:1046400091789844B8F1C80FA8BF4FF0C80828EA7D
:10465000E87880F80380002940F0BB830F2E3FF4F8
:1046600073AF90F800809844B8F1C80FA8BF4FF01E
:10467000C80828EAE87880F800809278002A3FF499
:1046800063AF1220414620F0D7F9D4F8D0005BE7A1
:104690000899404A91F807809278984488F308086E
:1046A00081F80780002A3FF47FAF0520414620F0C3
:1046B000C3F9D4F8D00047E70898364A90F8068046
:1046C00091789844B8F1640FA8BF4FF0640828EAC5
:1046D000E87880F80680002940F028830D2E3FF40A
:1046E00063AF0898927890F805809844B8F1640F09
:1046F000A8BF4FF0640828EAE87880F80580002A0F
:104700003FF452AF0E20414620F096F9D4F8D00085
:104710001AE708991F4A91F8048009929844B8F161
:10472000640FA8BF4FF0640828EAE87881F8048095
:1047300020F09CF9099A9278002A3FF435AF0320C3
:10474000414620F079F9D4F8D000FDE6D4F8D00045
:10475000104A90F8088092789844B8F1C80FA8BF22
:104760004FF0C80828EAE87880F80880002A3FF46B
:10477000EBAE0B20414620F05FF9D4F8D000E3E621
:10478000A87D0020E4A10020C89E002008A80020E9
:10479000C49E0020AC8E0020D4F8D000BA4A90F815
:1047A000078092789844B8F1C80FA8BF4FF0C808A6
:1047B00028EAE87880F80780002A3FF4C5AE0A208E
:1047C000414620F039F9D4F8D000BDE6D4F8D00045
:1047D000AD4A90F8068092789844B8F1C80FA8BF07
:1047E0004FF0C80828EAE87880F80680002A3FF4ED
:1047F000ABAE0920414620F01FF9D4F8D000A3E663
:10480000D4F8D000A04A90F8058091789844B8F187
:10481000C80FA8BF4FF0C80828EAE87880F80580DC
:10482000002940F0C082112E7FF4C4AE8CE6D4F88B
:10483000D000954A15E7D4F8D000934AE5E6924AAD
:104840004FE70899904A91F800809844B8F1FA0F20
:10485000A8BF4FF0FA0828EAE87881F8008092783B
:10486000002A3FF4A1AE0120414620F0E5F8D4F83B
:10487000D00069E60899844A91F802809844B8F11A
:10488000640FA8BF4FF0640828EAE87881F8028036
:104890009278002A3FF488AE0220414620F0CCF8FE
:1048A000D4F8D00050E60C9AFFF789BB39F9111003
:1048B0009078B1F5617F4FF4966898FBF0F0C0F204
:1048C0008D8040F633088845A8BF88460C2EA8F591
:1048D000617898FBF0F85FFA88F800F02C81182EC8
:1048E00040F08E804146C829A8BFC821674CD4F843
:1048F000D00090F817C05FFA81FEE6453FF475AA34
:10490000B1EB0C01604A80F817E048BF0731C910CD
:1049100090784A1CD2B238B912B1104628F07EFB0A
:10492000DBF80420FFF761BA41461820099220F015
:1049300083F8099AF0E7564B56491A684FF47A7390
:10494000B3FBF2F3C3EB431203EB8202029B1B683F
:10495000D200A1F8A8201A067EF542A94E4A127884
:1049600097077EF53DA94D4A127D042A7EF638A9A7
:1049700018F0F2F8029B4A4E1B68FEF732B90F207E
:1049800028F042FAB4F8903084F89250FA3BA4F838
:104990009030029B424E1B68FEF723B9B0EE670AC7
:1049A000FFF7BDB91BF0100F40F02D810B201FF059
:1049B000F9FF002840F0F480DFF8FC801BF0200FA6
:1049C00040F03D81314C94F8D430002B3FF4F7ACEB
:1049D000BAF1000F7FF48AAAFEF7EBB90C2E00F0B3
:1049E0000F81182E0AD14FF0000841467EE72D496D
:1049F000029B0A601B682A4EFEF7F3B84FF00008CE
:104A0000224CFFF7F2B906F48056FEF75CBF264B46
:104A1000012202203CE5254A029B1E68136823F010
:104A200004031360049A012306F4805682F82130AF
:104A3000FEF749BF38EE678A1D4B1E491870FDEE20
:104A4000C87ACAF5FA63CDED007ABDF900201203E9
:104A500081FB0201D217C2EBA1121BB203FB02F3CE
:104A600043F30F33534407EE903AF8EEE77AC8ED7C
:104A7000037AFEF78DBAD4F8D0001FF087F84FF014
:104A8000FF38FFF7BEB900BFAC8E0020EC2B002032
:104A9000DCB00020ECA80020C69E0020EC580020CE
:104AA000C49E002030A1002032A20020C09E002021
:104AB000982E0020D34D6210946600200022BB2B5C
:104AC0000E9200F0FE80B72B00F0F880BE2B00F0B5
:104AD000F280BD2B7FF403AD13464FF6FE72C24940
:104AE000C8898D8903442A448A81CB8112F076F9E2
:104AF00009F078F812F05AF9F9F722F9012028F0B4
:104B00008DFAB4F89020029BFA3A00211B68A4F8B1
:104B1000902084F89210FEF764B8B44B0222032070
:104B2000B6E4B349029B0A781B68B24E42F0040215
:104B30000A70FEF756B84446AF494978A1423FF49F
:104B40005FAFAE4A0992204624F070F9099A927834
:104B50001AB141460C201FF06FFF621CD2B2A84C64
:104B6000DAE6F9F78DFA94F88E30FFF7F2B91020F3
:104B700006F090FC202006F075FCA249DFF8A08228
:104B8000081F14F0AFF8A04B02221A709C4C94F846
:104B9000D430002B00F0D380B6F800B0FFF7A6B9F0
:104BA0009A4BDFF87C825B8998ED007A07EE903AA9
:104BB000F8EEE77AB0EEC77AB4EEE77AF1EE10FAE3
:104BC0007FF5FCAE98ED017AB0EEC77AF4EEC77AC5
:104BD000F1EE10FA7FF7F2AE1BF0200F7FF4F2AE89
:104BE000202006F057FC94E80C0089490A6008462A
:104BF00041F8043F14F076F8834B01221A70C5E7A0
:104C00000024A04698E7102006F02CFC7E4BB6F856
:104C100000B083F800A04FF0010AC7E608231A4647
:104C2000FEF7A6BB07231A46FEF7A2BB794A029BF2
:104C3000704E1B684FF4C8711180FDF7D2BF202061
:104C400006F010FC704B00221A709FE702231A46F0
:104C5000FEF78EBB01231A46FEF78ABB06231A46CF
:104C6000FEF786BB05231A46FEF782BB04231A46CD
:104C7000FEF77EBB03231A46FEF77ABB4FF4FA61B8
:104C8000022023F0F1FF48E484F8941084F89500A2
:104C9000584EFEF745BF002D3DF490AF584C94F8A8
:104CA0008D30002B3DF4B6AE28F098F8002384F840
:104CB0008D30FDF7AFBE1346022210E74FF6FE73AC
:104CC0000DE702230BE70021012023F0CDFFB4F80C
:104CD0009020029B963A00211B68A4F8902084F84B
:104CE0009210FDF77EBF00210846EEE7FF2100206D
:104CF0001DF0CDFF94F88E30FFF7FDBB01210020A1
:104D00001DF0C5FF94F88E30FFF7F2BB0021FF20A5
:104D10001DF0BDFF94F88E30FFF7E7BB00210120A6
:104D20001DF0B5FF94F88E30FFF7DCBB41460D2037
:104D30000A9209931FF080FE0A9A099BCEE44FF075
:104D4000010AFFF73CBB00210420BEE7002103203D
:104D5000BBE700210220B8E70B2028F055F8029BA2
:104D6000244E1B68FDF73DBF254C23F0C7F884F89F
:104D70008D50FDF74FBE002B90D02749274A096878
:104D80004FF47A7000FB0313136087E74146172046
:104D90001FF052FE08E4152041461FF04DFED4F8E6
:104DA000D000FFF7D1BB112041460A9209931FF0B2
:104DB00043FED4F8D0000A9A099B34E510204146FE
:104DC0000A9209931FF038FED4F8D0000A9A099B82
:104DD00019E40F2041460A9209931FF02DFED4F8E2
:104DE000D0000A9A099B39E4387F002080A2002075
:104DF000C69E0020C49E002008A80020AC8E002083
:104E0000EC2B0020E46800200A690020986900204B
:104E1000AC28002042B30020E4A700202CA10020F1
:104E2000946600202DE9F047C74C636820469847F8
:104E3000002800F0C380C54B1B780122042B84F8A6
:104E40003C2000F0BD80B4F91610B4F91820B4F974
:104E50001A3021636263A363BD4B1B88002B69D0AA
:104E6000BC4DD4ED0C7AD5ED004A95ED050A95EDD3
:104E7000015A95ED067AD5ED035A95ED026AF8EEE2
:104E8000E76AD5ED047AA4EEA60AA5EE267A67EEC7
:104E9000C07AA5EEC07AE6EE267A85ED057AC5EDF4
:104EA000067A29F0C9FCD4ED0D6AD5ED094A95EDD5
:104EB0000E0A95ED0A5A95ED0F7AD5ED0D7AD5EDDE
:104EC0000C5A95ED0B6A2063F8EEE66AA4EEA60A8A
:104ED000A5EE267A67EEC07AA5EEC07AE6EE267ACF
:104EE00085ED0E7AC5ED0F7A29F0A6FCD4ED0E6A99
:104EF000D5ED124A95ED170A95ED135A95ED187AEE
:104F0000D5ED167AD5ED155A95ED146A6063F8EE75
:104F1000E66AA6EEA40AA6EE857A67EEC07AA0EE4F
:104F2000657AE6EE867A85ED177AC5ED187A29F06E
:104F300083FCA063884FA17F884810F093F93B88D9
:104F4000002B40F08480864ED6F8E450854B1B68D9
:104F50005B0743D4B5F90070216B636BA06B824A89
:104F6000824E92ED026AD2ED006AD2ED015AC91B5F
:104F70002163B5F90270DB1B6363B5F90470356812
:104F8000C01B07EE900AB8EEE75A07EE901AB8EE8B
:104F9000E77A07EE903AF8EEE77A36EE056A36EEF3
:104FA000877A77EEA57A0135A06382ED026A82EDF9
:104FB000007AC2ED017A3560BDE8F087BDE8F08780
:104FC0006B4BB4F91600B4F91810B4F91A20188014
:104FD0002063598061639A80A2633DE7B6F8982008
:104FE000322A00F08880002A66D196F89530002B8E
:104FF000B0D06048D6F800215F4980FB0273D21719
:10500000C2EB23122A80D6F8042180FB0273D21748
:10501000C2EB23126A80D6F80831A78A80FB03020C
:10502000DB17C3EB2213DB1BAB800023CB6086F8BE
:10503000953011F0D3FE08F0D5FD11F0B7FEF8F76A
:105040007FFE012027F0EAFFD6F8E45082E7444EC5
:10505000226BD6F8E450B3F5C87F4FF0000323630A
:105060002B80398818BFD6F8E800B7F8008008BF51
:105070000020B1F5C87F18BFD6F8EC30616B024450
:105080000B440020B8F5C87F6063C6F8E820C6F876
:10509000EC30688052D0D4F838E0D6F8F010A06335
:1050A0007144B8F1010FA880C6F8F01068D008F17B
:1050B000FF38A7F8008049E7D6F80001236B0021EC
:1050C0000344C6F8003121632980D6F80401636BDC
:1050D00061630344C6F804316980A36BD6F8080104
:1050E000A1630344012AC6F80831A98075D0013AAA
:1050F000A6F8982079E72B8820491F48276BA6F847
:10510000F4300023B5F802E0B5F804C0C0684B6085
:105110008B602363C6F800712B80616BC6F80411A5
:1051200063636B80A16BC6F80811A363A6F8F6E071
:10513000A6F8F8C0C6F8FC00AB80D8E7A36BC6F8A9
:10514000F030A063A880B2E77C9E0020A9960020E2
:10515000484D00204C4D002042B30020AC9E002062
:10516000EC2B0020ECB00020BC900020B890002078
:10517000AC9600201F85EB51387F0020EC2C0020DE
:10518000DFF88CC0DFF884E0C8328CFB02A9C8339A
:10519000D217C2EBE9128CFB03A9DB17C3EBE913AF
:1051A000C8316B802A808CFB013CA28ACB17C3EBF1
:1051B000EC139B1AAB80CEF80C0011F00FFE08F038
:1051C00011FD11F0F3FDF8F7BBFD404627F026FF77
:1051D000B7F80080D6F8E45069E70B2086F89A10FB
:1051E00086F8942027F010FED6F8E450074BB6F866
:1051F000F420B6F8F670B6F8F800D6F8FC102A805D
:105200006F80A880B6F89820D96070E7387F0020BA
:105210001F85EB512DE9F0478C4B1B78DB070746C8
:1052200044D58B4B8B4D1C788B4E012C59D01CD305
:10523000022C07D189498A4A09881288914201D9EA
:1052400001241C70EB7AE3B12B89D3B1854B1B7819
:10525000BBB106F0ABFC002800F09B802B7B8342A7
:105260002CBF0121002131700CE07C497E4A098865
:1052700010886A7B801A8842E2DAEB7A0024002BDD
:10528000E2D131782A79632A06D8022C774E00F0D1
:10529000BA803378002B5DD1754AAB7A8C4238BF27
:1052A0000C461470002B4CD1BDE8F0876B4B694D58
:1052B00019885B88E878CB1A83EAE3728142A2EB13
:1052C000E3721DD32B788B421AD3614B1C78E01EFE
:1052D000012861D96749097802294FD0012C5E4E17
:1052E000A5D15F4A5D491288687B0988121A9142EC
:1052F00039DD5D4A12888A42A4D200241C70A1E7DD
:10530000B1EB400FE1DC524B1C78E11E012940F269
:105310009480022ADEDC57494F4E0878DFF844813A
:10532000DFF844C1DFF838E100210324022834709B
:105330001C7088F80010ACF80010AEF8001081D195
:105340001FE0012C71D0022C0BD10720BDE8F047E3
:1053500027F05ABD7068381A474B984258DD727072
:105360009AE7BDE8F08702241C706BE7022AD2DDC1
:105370004049097802294FF0040464D13949364E76
:1053800009783E48022ACCBF00220122C2808180D7
:105390004BE70221317075E7022A9BDC95F800C0CB
:1053A00091FBFCFC0CF1010CBCF1080FDFF8B4A080
:1053B000304EA87895F801E096F800802A4CDFF886
:1053C000A090254EA8BF4FF0080C8AF800C01FFA25
:1053D0008CFA10FB0AF01EFB0AFE80B2DFF88CA0EC
:1053E0002080A9F800E000244FF0640EB8F1020F0D
:1053F00034701C70CAF804408AF801E07FF439AFB9
:105400000FFA8CF1BDE73078A0B9012377603370D3
:10541000C2F164021A4B00FB02F083FB0023C017A9
:10542000A0EBA3506430707036E70820BDE8F04769
:1054300027F0EABC7368F81A8EE7032C96D10D4961
:10544000097802299AD0044EFCE600BF6090002043
:10545000BC2F0020609E0020CC2F00207C66002006
:10546000C02F002092660020BE2F0020C42F0020F5
:1054700010800020A99600207F969800AC9600200E
:105480006BCA5F6B2DE9F04F2DED0C8BDFF8A89305
:1054900095B0D9F80420069048469047002875D06A
:1054A000B9F8A850002189F85110002D41F0568418
:1054B000D9F84820B9F93C70B9F93840D9F82060DA
:1054C000B9F93A00D9F82450DFF870B3BB1A83EA6F
:1054D000E371A1EBE371A41BB1F5804FC9F82C4037
:1054E000D9F8284099F85210DCBFC9F848703A46FC
:1054F000401B121BC9F83000B548C9F834200FF022
:10550000B1FEDBF80020910041F11C85D9ED0C5A69
:10551000DFF82CA3D9ED0B7AAE499AED406ADAEDAB
:10552000416A9AED427ADAF80C210968AA4B049391
:10553000B8EEE58AD9ED0D5AF8EEE77AF8EEE58A8D
:10554000013277EE867A38EE268A78EE878A8A42AA
:10555000CAED407A8AED418ACAED428ACAF80C2126
:1055600002F0DE811F78142F03F04E810023DAF859
:1055700014410593062C01F28381DFE814F0BD1479
:10558000FA15FA139115F1080B165A14924BDFF81D
:10559000B0A21C780493072C01F0C5819AF8213140
:1055A000089353B15F1E8AF82171012C01F0A78482
:1055B00015B0BDEC0C8BBDE8F08F884A5279002AFB
:1055C00001F02782864A1278013AD2B2072C8AF873
:1055D000212102F0A28200230A938249DAF82C21C9
:1055E000D1ED006A8049079106999FED806ADAED56
:1055F0004AAA7F4B7F4F1B68DFF848B29AED499A61
:105600009FED7DAADFED7DBA9FED7DCA9FED7DBA4E
:10561000DFF834827C4ECDF814B08A1A07EE902A57
:10562000F8EE677AB7EE007AC6EE279A002407F103
:105630001C02CAF82C11099225469B4677EE6A8A0D
:1056400068EEA68AF4EEC78AF1EE10FA88BFF0EE93
:10565000478A6E4B97ED008A2344D3ED007AF5EE2E
:10566000407AF1EE10FA17D0694B234493ED007A9B
:1056700078EE476AB0EEE66AF4EEC67AF1EE10FA1A
:1056800008D5F5EEC06AF1EE10FACCBF37EE878A86
:1056900037EE678A83ED008A5E4B1A8893073FD006
:1056A000022D3DD05C4B9BF82E1033F9153007EEE0
:1056B000103A099B07EE901A2344F8EEE76AB8EE19
:1056C000C77AD3ED007A4B42A6EEA77A680007EEC0
:1056D000903AF8EEE77AB4EEE77AF1EE10FA0AD4EF
:1056E00007EE901AF8EE677AF4EEC77AF1EE10FA48
:1056F00088BFF0EE477A494B49490344085EB3F945
:105700000C30C01A07EE100AB8EEC77AD007E7EEE1
:105710004A7A41F11281434B93ED008A27EE888A41
:10572000079B9AF86421234493ED01DA78EE4DCA81
:10573000002A00F0CB803C4BDAF8682106991B6800
:105740008A1A9A4240F3C2809BF84830022B02F03A
:105750002382022D04F01E84344B1B68990775D4F4
:10576000334B86ED00CA1B689342C0F2A980F7EE66
:10577000007AF4EEE7AAF1EE10FA40F1A78007995B
:105780002C4BD1ED017A93ED007AF0EEE77AF4EE4E
:10579000C77AF1EE10FA40F19980D1ED027AF0EE7D
:1057A000E77AB4EEE77AF1EE10FA40F38F80D1EDAC
:1057B000037AF0EEE77AB4EEE77AF1EE10FA40F30E
:1057C00085801A4B1B689A077AD51549134B5EE002
:1057D00018A90020104A0020A9960020C8B0002077
:1057E0002C7F002094950020DCB000200024744918
:1057F000C89E0020282E0020CDCCCC3DAE47813F56
:10580000000000000000C842387D0020889500207C
:10581000342E0020C49E0020402E0020387F00201F
:10582000749E0020709500209C950020709E0020A2
:1058300098950020A4950020ECA80020ECB0002052
:10584000F82C00202C7D0020447D0020D74BD84927
:10585000DFF8C8E331F915C09EED008ADFF8C0E338
:1058600086ED00CA03EB450028EE0A8AB0F90C0069
:10587000A0EB0C0007EE900AF8EEE77ADEF80000E5
:1058800027EE888A904278EE4DCABFF670AFB3F922
:105890000C20B1F900E0C748AEEB020E00688EEABA
:1058A000EE72A2EBEE72824210DAB3F90E30B1F969
:1058B0000220D21A82EAE273A3EBE273984205DD7A
:1058C000002318468AF86431F9F774FFBA4B234471
:1058D00093ED000A059B29EE000A022D20EE2C0A0A
:1058E000A3EC010A059304F0F782B44BD6ED006AED
:1058F00093ED007AB24BD3ED007AB24B93ED006A90
:10590000B14B67EE277A234427EEA87AD3ED007ACD
:1059100067EE277AF0EE665AECEEA75AB1EE467AB9
:10592000B4EEE57AF1EE10FA08DCF4EEC65AF1EEC8
:1059300010FA8CBFB0EE467AB0EE657A9AED4A6AFC
:10594000F7EE007AB4EEE76AF1EE10FAACBF01238D
:10595000002343B1F0EEE66AF0EEC77AF4EEE67AA1
:10596000F1EE10FA01D586ED007A022D04F08C825A
:10597000964A974B52F825001B68B0EE4D0A98479F
:10598000944A954B52F825001B6898479BF837308E
:1059900023B1924B1B88002B01F0D080B0EE4C8AD3
:1059A0008F4B38EE400A234493ED008A83ED000AC2
:1059B0009BF8483030EE480A20EE298A53B3894BD1
:1059C0001B78DB0740F1BF86F7EE007AF4EEE7AA1A
:1059D000F1EE10FA9AF86431C1F22085002B01F043
:1059E0006181DAF86831069AD31A7F4A12689A42BE
:1059F00010DD7E4BD3ED007AF0EEECCAF4EEE7CA90
:105A0000F1EE10FA42F1D180002318468AF8643191
:105A1000F9F7D0FE764B9AF87421234493ED000AEF
:105A200029EE000A20EE088A88ED008A32B9059B2B
:105A300086ED00CA03ED01CA88ED00CA0135032DC9
:105A400007F1040708F1040806F1040604F1040450
:105A50007FF4FFAD049B1A78072A01F0F584012A30
:105A600002F04980002307939AF87C21002A41F034
:105A70005382DFF8B0B15F4BDBF800201968D40423
:105A800091F82C0001F18680DFF89C815A4AB8F821
:105A90001A3092ED006A594A594CD2ED005AD4EDB1
:105AA000036A584A8AED636A07EE103A564B92ED44
:105AB000005AD3ED007AD3ED013AD3ED024A8AEDD4
:105AC000616AB8EEC77A35EEC64A012236EEC77A69
:105AD0008AED604ACAED645A8AF89421C7EE055AE5
:105AE0000A8D534206EE103A484BDFED496A93EDBA
:105AF000005A484B93ED004AB7EE007AF4EEC75ACD
:105B000035EE045AF1EE10FA88BFF0EE475A35EE42
:105B1000275AB8EEC66AF4EEE65AF1EE10FA07EE2E
:105B2000902AB4EEC65AB8BFF0EE665AF1EE10FAFB
:105B3000CAED675AB8EE677A01F15283B4EEC75ADC
:105B4000F1EE10FA88BFB0EE475A304BDFED326A03
:105B5000D3ED017A2F4B93ED014A77EE847A25EE4F
:105B6000265A77EEA37AB4EEE76AF1EE10FA08DC73
:105B7000B4EEE77AF1EE10FA8CBFB0EE676AB0EEE1
:105B8000476A224B4A8DD3ED027A9FED237A534226
:105B900004EE103A74EEA77AB8EEC44A26EE076A0D
:105BA000F4EEC47AF1EE10FA4BD43FE0387F0020D7
:105BB000749E0020A09500204495002098000020AD
:105BC000E8900020B895002050950020F09000202B
:105BD000EC9000204491002040910020C49E0020C1
:105BE000642E0020609000209C950020A895002045
:105BF0005C950020C89E0020C47D00201C7F0020F2
:105C00009466002050960020387D00202C7D0020D6
:105C100000000000447D00206F12833A7095002040
:105C200098950020ECB00020FC9C002007EE102A84
:105C3000B8EE474AB4EEE74AF1EE10FA88BFB0EE8C
:105C4000674AEB4ADFEDEB7A527824EE274A0AB92D
:105C5000B1EE444A002841F01486B7EE003AE64D12
:105C60002A78002A02F08186E449DFEDE57AD1ED59
:105C7000024AD1ED016A91ED037A66EE244AE5EE1F
:105C8000264AE4EE074A63EE244AF4EEE74AF1EED0
:105C900010FAB4BFF0EE673AF0EE643A98BFF0EE57
:105CA000647A012ACDED0C4A02F0B48691ED067AB1
:105CB000D1ED052AD1ED076A26EE077AA5EE227A04
:105CC000A4EE267A23EE077AB4EEE77AF1EE10FA24
:105CD000B4EEE37A8CBFF0EE676AF0EE476AF1EE5D
:105CE00010FA88BFF0EE676AB4BFF0EE637AF0EEA8
:105CF000477A022A8DED0D7A00F0DE8091ED0A7A66
:105D0000D1ED092AD1ED0B3A26EE077AA5EE227ADB
:105D1000A4EE237A23EE077AB4EEE67AF1EE10FAD7
:105D2000B4EEE77A8CBFF0EE663AF0EE473AF1EE69
:105D300010FA98BFF0EE636AA8BFF0EE477A032A24
:105D40008DED0E7A00F0B88091ED0E7AD1ED0D2A2E
:105D5000D1ED0F3A26EE077AA5EE227AA4EE237A49
:105D600023EE077AB4EEE67AF1EE10FAB4EEE77AB3
:105D70008CBFF0EE663AF0EE473AF1EE10FA98BFBB
:105D8000F0EE636AA8BFF0EE477A042A8DED0F7A31
:105D900000F09280D1ED123AD1ED112A91ED137AF3
:105DA00066EE233AE5EE223AE4EE073A63EE233A52
:105DB000F4EEE63AF1EE10FAF4EEE73A8CBFB0EE0C
:105DC000667AB0EE637AF1EE10FA98BFF0EE476AA9
:105DD000A8BFF0EE637A052ACDED103A6CD0D1ED74
:105DE000163AD1ED152A91ED177A66EE233AE5EED3
:105DF000223AE4EE073A63EE233AF4EEE63AF1EEA5
:105E000010FAF4EEE73A8CBFB0EE667AB0EE637A41
:105E1000F1EE10FA98BFF0EE476AA8BFF0EE637A91
:105E2000062ACDED113A47D0D1ED1A3AD1ED192A13
:105E300091ED1B7A66EE233AE5EE223AE4EE073A5C
:105E400063EE233AF4EEE63AF1EE10FAF4EEE73AB6
:105E50008CBFB0EE667AB0EE637AF1EE10FA98BFBE
:105E6000F0EE476AA8BFF0EE637A072ACDED123A4A
:105E700022D091ED1E7AD1ED1D2AD1ED1F3A26EEEA
:105E8000077AA5EE227AA3EE847A27EE037AB4EE9F
:105E9000E67AF1EE10FAB4EEE77A8CBFB0EE666AFD
:105EA000B0EE476AF1EE10FA8DED137A98BFF0EE7E
:105EB000466AA8BFF0EE477A77EEE67AF7EE006A18
:105EC000F4EEE67AF1EE10FACAED4A7A43F3A086D0
:105ED00086EEA77A022ADDED0D7A67EE244A67EE98
:105EE000877ACDED0C4ACDED0D7A2DD0DDED0E7A11
:105EF00067EE877A032ACDED0E7A25D0DDED0F7A95
:105F000067EE877A042ACDED0F7A1DD0DDED107A89
:105F100067EE877A052ACDED107A15D0DDED117A7E
:105F200067EE877A062ACDED117A0DD0DDED127A73
:105F300067EE877A072ACDED127A05D0DDED137A68
:105F400027EE877A8DED137A2E49096811F0805378
:105F5000059301F01882F6EE005ACAED675A002A3E
:105F600002F028859AF994319AED646A2649274E01
:105F70009AED635A264FB6F90660C878DBF8001030
:105F8000099607EE103ABDEEC66A224BB8F81A60C1
:105F90001C78214BD7ED004A0A9616EE10EABDEEAA
:105FA000C56A01F0100601F4805701F480010B91DD
:105FB0001B78DAED606ADAED617AB8EEC77A04F040
:105FC000010C16EE101A002840F0E8870B4C9DEDEE
:105FD0000C5A94ED006A002E41F0348325EE866A57
:105FE0000E48A5EE076AB0EE675AA6EE265A17E0ED
:105FF000687F00206F12833A65650020C0950020FD
:1060000000000000A87D0020886800206E8E00201F
:10601000BC9500206090002068550020607D002025
:10602000BDEEC56A16EE107A16EE106A7745A8BF67
:106030007646B942C8BF0E4606EE106AB8EEC66A8A
:10604000012A80ED006A00F0DC8094ED046A9DED89
:106050000D5A25EE866AA5EE076AB0EE675AA6EEDF
:10606000265ABDEEC56A16EE107A16EE106A77450E
:10607000A8BF7646B942C8BF0E4606EE106AB8EE13
:10608000C66A022A80ED016A00F0BB8094ED086ABE
:106090009DED0E5A25EE866AA5EE076AB0EE675AA8
:1060A000A6EE265ABDEEC56A16EE107A16EE106AF6
:1060B0007745A8BF7646B942C8BF0E4606EE106ABD
:1060C000B8EEC66A032A80ED026A00F09A8094ED69
:1060D0000C6A9DED0F5A25EE866AA5EE076AB0EEB2
:1060E000675AA6EE265ABDEEC56A16EE107A16EE6F
:1060F000106A7745A8BF7646B942C8BF0E4606EE7D
:10610000106AB8EEC66A042A80ED036A79D094ED6D
:10611000106A9DED105A25EE866AA5EE076AB0EE6C
:10612000675AA6EE265ABDEEC56A16EE107A16EE2E
:10613000106A7745A8BF7646B942C8BF0E4606EE3C
:10614000106AB8EEC66A052A80ED046A59D094ED4B
:10615000146A9DED115A25EE866AA5EE076AB0EE27
:10616000675AA6EE265ABDEEC56A16EE107A16EEEE
:10617000106A7745A8BF7646B942C8BF0E4606EEFC
:10618000106AB8EEC66A062A80ED056A39D094ED29
:10619000186A9DED125A25EE866AA5EE076AB0EEE2
:1061A000675AA6EE265ABDEEC56A16EE107A16EEAE
:1061B000106A7745A8BF7646B942C8BF0E4606EEBC
:1061C000106AB8EEC66A072A80ED066A19D094ED07
:1061D0001C6A9DED135A65EE865AE7EE055AE6EE07
:1061E000A57AFDEEE77A17EE904AA645A8BFA64627
:1061F000A142D8BF714607EE901AF8EEE77AC0EDDB
:10620000077ABCF1000F00F0D687D04A1268002A46
:1062100040F0DE87CE4A127882B1287858B1CD4E50
:10622000CD4F0024E0B23B68B6EC010A98472878CD
:1062300001348442F6DBC94A12689047049B1A78FD
:10624000072A01F0F0800025DBF80020570501F156
:106250002680C34B1B78BBB1C24AB8F81A30B2F9DA
:1062600006209A4210DCC04B1B78012B01F05A84A7
:10627000192B01F057840E2B06D0082B04D0BB4CF1
:106280000023A360CAF838319AF8A64124B1B84B6C
:106290001B889E0741F0D8839AF8AC31002B40F060
:1062A000A38798F81E60002E00F02086022E01F0D1
:1062B0001983032E41F01D8398F82020C2EB421170
:1062C00002EB8102D20092B298F81F700237FFB23F
:1062D000002B00F03C86002A00F03986A5490E68A4
:1062E000B2FBF6F216B2AAF8DC61002F03F0898146
:1062F00007EE906AF8EEE77AF7EE006A86EEA77A84
:106300009A4C012FDAED7C6AD4ED007A77EEE67ACA
:1063100067EE877ACAED787A21D0D4ED017ADAED8A
:106320007D6A77EEE67A022F67EE877ACAED797A90
:1063300015D0D4ED027ADAED7E6A77EEE67A032F95
:1063400067EE877ACAED7A7A09D0D4ED037ADAED6E
:106350007F6A77EEE67A67EE877ACAED7B7A049AEF
:106360001278092A03F0DF82002E40F3C5859FB31F
:106370009AED7C7ADAED787A77EE877A012FCAED9A
:106380007C7AC4ED007A21D09AED7D7ADAED797AC3
:1063900077EE877A022FCAED7D7AC4ED017A15D0A7
:1063A0009AED7E7ADAED7A7A77EE877A032FCAED64
:1063B0007E7AC4ED027A09D0DAED7F7A9AED7B7AA3
:1063C00077EE877ACAED7F7AC4ED037A013F022F18
:1063D000B8BF0227FAB20892002B089F18BF022705
:1063E000654BDFED6A6A1A68049B91781878137818
:1063F00007EE903AF8EEE77AB0EE007A67EEA67A0A
:10640000F4EEC77AF1EE10FA40F3E686DFED5C6A4F
:1064100037EEC77AB0EE676AA7EE266AF0EE466AF4
:1064200094ED007A9FED576A27EE066AF0EEC65AA1
:106430008AED536ACAED565A99B107EE101AB8EEB2
:10644000C75A9FED527A66EE064A25EE075AB7EE16
:10645000007A37EE457A64EEA54AA4EE857A26EEF8
:10646000076A9FED497A537926EE877A27EE067AF6
:10647000CBB1DFED466A9FED466A65EEA65A06EEA1
:10648000903AF8EEE66A65EEA65AF4EEC65AF1EED8
:1064900010FA01F3EC81B7EE006A76EE655AC6EEAB
:1064A000256A27EE267A0C289FED3A8ADFED3A6AB4
:1064B00000F09787B4EEC87AF1EE10FA98BFB0EE0C
:1064C000478AB4EEE68AF1EE10FAB8BFB0EE668AFB
:1064D0008AED4C8A002F00F00781B0EE007AF4EECE
:1064E000C77AF1EE10FA05DD37EEC77ADFED246AE0
:1064F000E7EE267A94ED017ADFED226A27EE267A1E
:10650000F0EEC75A8AED547ACAED575A99B106EEA1
:10651000901A9FED1E6AF8EEE66A27EE075A66EEBD
:10652000866AB7EE006A36EE666A25EE255AA5EE53
:10653000266A27EE067ADFED146A937967EEA67A6B
:1065400067EE877A002B3FD028E000BFE490002060
:1065500090580020607D00205C550020645500208C
:106560007D2200206E8E0020687F0020946600202F
:10657000C49E0020607F0020CC9E00200000C84206
:10658000D7A368416F12033B000048430AD7233C5E
:10659000A4707D3F00C0F94400C0F9C407EE103A72
:1065A000B8EEC77A1FED076A5FED076A27EE257A16
:1065B00027EE067AB4EEE67AF1EE10FA41F3458161
:1065C0005FED126A67EEA67A0C2800F0E3865FEDB5
:1065D0000F6A1FED0F7AF4EEE67AF1EE10FA88BF3B
:1065E000F0EE667AF4EEC77AF1EE10FAB8BFF0EE8C
:1065F000477A012FCAED4D7A76DD53785FED1D6A3B
:1066000007EE903AF8EEE77AB0EE007A67EEA67AF7
:10661000537AF4EEC77AF1EE10FA05DD37EEC77A59
:106620005FED296AE7EE267A94ED027A5FED2B6A38
:1066300027EE267AF0EEC75A8AED557ACAED585AF7
:106640009BB106EE903A1FED2F6AF8EEE66A27EE50
:10665000075A66EE866AB7EE006A36EE666A25EE7F
:10666000255AA5EE266A27EE067A5FED396AD379B8
:1066700067EEA67A67EE877AFBB107EE103AB8EEBE
:10668000C77A1FED3E6A5FED3E6A27EE257A27EE58
:10669000067AB4EEE67AF1EE10FA01F3E480B5EE94
:1066A000C07AF1EE10FA02F16F83B7EE006A36EEAF
:1066B000477AC6EE076A67EEA67A0C2800F089864C
:1066C0005FED4C6A1FED4C7AF4EEE67AF1EE10FACB
:1066D00088BFF0EE667AF4EEC77AF1EE10FAB8BF32
:1066E000F0EE477ACAED4E7A092800F03F8698F816
:1066F0002140002C40F0F48500238AF8AC31C64BD1
:106700001B689E0609D5C54B1B8803F0300323B1D7
:10671000C34B1B78DC0702F1B380C24B1B7823B953
:10672000C14CA778002F41F0A581049B1C78072C51
:106730007EF43BAFF8F70EFCBC4B049A401B147878
:10674000D880FEF732BF9AF86431002B3FF462A97B
:10675000002318468AF86431F9F72CF8FFF75AB984
:10676000B34A1178DAF81861B24B9FEDB37AF500AD
:106770005A1982ED007A002978D0B048B0EE476A05
:10678000F0EE476A0022F0EC017A013267EEA77A58
:1067900005EE902AB4EEE77AF1EE10FAF8EEE55A3B
:1067A000B8BFB0EE677A8A4276EEA76AA7EEA56A0E
:1067B000E9D1F5EEC06A5A19F1EE10FA82ED007ACD
:1067C00054DDC6EE265A9E4A9E490988F7EE007AA5
:1067D00075EEE75AD2ED007A65EEA77AFDEEE77A1C
:1067E00017EE902A812A42F346828A42A8BF0A46BF
:1067F00007EE902AF8EEE77A934AA81902EB800296
:1068000092ED057AD2ED003A92ED066A92ED014AD8
:10681000D2ED046AD2ED034A92ED025AA3EEA77AB2
:10682000A4EE276A66EEC76AA7EE646ABDEEC77A71
:10683000E5EE276A17EE100A812882ED056AC2ED9F
:10684000066A42F31C828142A8BF014607EE901AF5
:10685000F8EEE77AFCEEE77ACDED077ABDF81C207A
:1068600059198A8016B9132F03F0C081152F41F0F2
:10687000D3821D446D4BAA8823F81620DAF8144100
:10688000724A013482FB04321119E217C2EBA102F1
:10689000C2EBC202A41ACAF814416D48DAF81C21EE
:1068A000069B6C4C01682478CAF81C319A1A114472
:1068B0000160002C40F0DE8007EE902A664DDFF884
:1068C000B081664EB8EEE78A05F2447405F5F667C6
:1068D000F5EC017A99ED070AD9F86C37F8EEE77A0A
:1068E000204627EE800A9847A4F1E000D9F88C36BC
:1068F0009847A4F17000D9F8FC369847D5F85006AF
:10690000D9F8AC309847D6ED007AA8EC010AE0EE51
:10691000087A2434A742E6EC017AD9D1049B1C788A
:10692000072C7EF43BAEF8F715FB049A3F4B147826
:10693000069A801A1880FEF731BEB1F900209AED50
:10694000567AB1F90200DAED576A454982EAE273F4
:10695000A3EBE273F4EEC76A80EAE072F1EE10FA9C
:10696000A2EBE072B4BFB0EE476AB0EE666A934243
:10697000B8BF134607EE103A0B78B8EEC77A27EE89
:106980000A7A002B00F06181364B93ED005AB5EE88
:10699000C05AF1EE10FA40F3F284334BD3ED006AA3
:1069A000F5EEC06AF1EE10FA40F3E98436EEC77AEC
:1069B00066EE4B5A87EE266AC5EE856AB7EE007A18
:1069C000B4EEC76AF1EE10FA88BFB0EE476AB5EED2
:1069D000C06AF1EE10FA76EE876AB8BFB0EE4C6A84
:1069E00066EE266AF4EEC76AF1EE10FA88BFF0EEA2
:1069F000476AF5EEC06AF1EE10FAB8BFF0EE4C6AE5
:106A00001A4B93ED007A67EE877AA7EEA68AFEF717
:106A100087BE0122FEF7DABD709E0020C49E0020D2
:106A2000C69E002080540020AC8E0020AC96002032
:106A3000164A00200C4D002000000000F82C002019
:106A4000184A0020144A0020344C00209324499214
:106A5000A8900020084A002018A90020AC9000202F
:106A60007C9500207895002080950020749500206A
:106A7000E0B0002007EE902AA04BA14CA149A24F04
:106A8000CDF81CA0F8EEE78A059304F2D465984689
:106A900000268A46049BD9ED077A1B78172B6DD008
:106AA00094ED007AB8EEC78A082B28EE278A07D122
:106AB000B0EE480A089327F0BFFE089BA8F8000034
:106AC000DBF8002092000BD5002E03F04882B0EED8
:106AD000480AD9F86C3705F170009847B0EE408A43
:106AE000B0EE480AD9F88C36A5F170009847D9F86D
:106AF000FC3628469847049B1B78032BB0EE408A4F
:106B000037D0D4F85406D9F8AC30B0EE480A9847DC
:106B1000D7ED007AAAEC010AE0EE287A0136032EBE
:106B200005F1240508F1020804F10404E7EC017AF8
:106B3000B0D1049BDDF81CA01C78F1E6734B744ABD
:106B4000234493ED007AD2ED007A724B67EE277AF8
:106B5000F7EE006AF4EEE67AF1EE10FA93ED007AC1
:106B600088BFF0EE667A67EE877A27EE888AFEF7AE
:106B700017BF27F061FEA8F80000C2E794ED007A85
:106B800009EB4602B8EEC78A128FA8F8002028EE5B
:106B9000278A95E7604BDFF8C0811A785F4CD207EF
:106BA0005CBFB8F81820AAF888215D4AD4ED037AB2
:106BB000128807EE102AB8EEC77AF4EEC77AF1EE23
:106BC00010FA41F2DE85574C238807EE103AB8EEF2
:106BD000C77AF4EEC77AF1EE10FAC0F2AF87524AE4
:106BE000524C92ED006AD4ED006A9AF99421CAEDF4
:106BF000636A76EE665A012ACAED616ACAED605A86
:106C00008AED646A01F09884069BCAF898310024E2
:106C100037EEC77AFCEEE77A454D8AED677A17EED4
:106C2000902AAAF88821012295ED005A8AF8942129
:106C3000404A944241F2D5853F4BD3ED007AD3EDE3
:106C4000013AD3ED024AFEF749BF3C4BD3ED005A5F
:106C5000F4EEEB5AF1EE10FA40F1F186B7EE005A7D
:106C600075EE654ADFED366A9FED365A364B36EEE5
:106C7000C77A24EE855AD3ED006AE5EE075A65EE31
:106C8000A65AF5EEC05AF1EE10FA40F27883CBEE38
:106C9000256AB7EE007AF0EE475AE6EE665AF0EE55
:106CA000656A9FE6294AD2ED007AB0EEC87AB4EE62
:106CB000E77AF1EE10FA7EF7ADAE254AD2ED007A12
:106CC000B0EEEC7AB4EEE77AF1EE10FA7EF7A2AE0F
:106CD000204AD7ED007A92ED007AF0EEE77AF4EEF2
:106CE000C77AF1EE10FA7EF595AE01220699CAF840
:106CF00068118AF86421FEF778BE00BFAC960020C8
:106D000018A90020E0B00020AC900020502E0020F8
:106D10006C9500206895002060900020946600200B
:106D200054960020569600201C7F0020409600209C
:106D30005C9600208FD00300387D002084950020D1
:106D400000003443610BB63B78950020AC950020E1
:106D5000A8950020B0950020FC9C0020814C824B1F
:106D600082481A68477807932646814BB6F9060091
:106D700005944FF47A76B6FBF2F2C2EB421602EBC0
:106D80008602D600B6B2B54204931C7801F07A8729
:106D9000D9F87C30B9F93810D9F8602003F1010E28
:106DA00007EE901A0A44BEF1010FC9F87CE0C9F859
:106DB0006020F8EEE77A01F07287D9ED1B5AD9ED21
:106DC0001D6A07EE10EA37EEE56AB8EEC75A012DE4
:106DD00086EE057A37EE257A77EEC77A89ED1C7A4A
:106DE000E7EE866A89ED1B7AF0EE667AC9ED1E6AD7
:106DF000C9ED1D6A02F0D683D9F89030B9F93A107E
:106E0000D9F8642003F1010E07EE901A0A44BEF18E
:106E1000010FC9F890E0C9F86420F8EEE77A01F0B4
:106E20005987D9ED205AD9ED226A07EE10EA37EEDC
:106E3000E56AB8EEC75A012D86EE057A37EE257A57
:106E400077EEC77A89ED217AE7EE866A89ED207AB6
:106E5000F0EE667AC9ED236AC9ED226A02F0128269
:106E6000D9F8A430B9F93C10D9F8682003F1010E23
:106E700007EE901A0A44BEF1010FC9F8A4E0C9F860
:106E80006820F8EEE77A01F04087D9ED255AD9ED70
:106E9000276A07EE10EA37EEE56AB8EEC75A012D09
:106EA00086EE057A37EE257A77EEC77A89ED267A6F
:106EB000E6EE276A89ED257AF0EE667AC9ED286A52
:106EC000C9ED276A02F00682059BDFF8C4A0D880CE
:106ED000B9F8A820049B013A1C78A9F8A8200799C2
:106EE00000224A608A60CA60FEF755BBAAF8DC61DE
:106EF000002B3FF404AC1F4C0227FFF771BA1E4B66
:106F00001E4A19681288174BC96919805A8015B032
:106F1000BDEC0C8BBDE8F08F194B1A4D1A7812F0AE
:106F2000010F2A7840F0A482002A00F0A484920085
:106F300015491648DFF85CB0DFF85C8027F0A8FA46
:106F4000FFF763B90A4B0493DFF844A0A5E4BAF84D
:106F5000DC61013E36B2002EAAF8DC61C8DD054CCA
:106F6000FFF705BAAC960020DCB00020C8B00020C6
:106F7000A996002094660020ACA000207E4400204A
:106F8000609000206565002080440020607D002026
:106F9000F82C0020ECB00020FC9C0020002E01F01A
:106FA0004881BCF1000F42F07983C24C002B42F0C3
:106FB000AB8194ED006A9DED0C5ABF4825EE866AC0
:106FC000FDEEE44AA5EE076AB0EE675AA6EE265A31
:106FD00014EE901ABDEEC56A16EE107A16EE106A1F
:106FE0007745A8BF7646B942C8BF0E4606EE106A7E
:106FF000B8EEC66A012A80ED006A00F0DF8094EDE9
:10700000046A9DED0D5A25EE866AA5EE076AB0EE7C
:10701000675AA6EE265ABDEEC56A16EE107A16EE2F
:10702000106A7745A8BF76468F42B8BF0E4606EE77
:10703000106AB8EEC66A022A80ED016A00F0BE80CE
:1070400094ED086A9DED0E5A25EE866AA5EE076A54
:10705000B0EE675AA6EE265ABDEEC56A16EE107A55
:1070600016EE106A7745A8BF76468F42B8BF0E4627
:1070700006EE106AB8EEC66A032A80ED026A00F0D6
